:100000000C94FC1C0C942D1D0C942D1D0C942D1D7A
:100010000C942D1D0C942D1D0C942D1D0C942D1D38
:100020000C942D1D0C942D1D0C942D1D0C942D1D28
:100030000C942D1D0D94DC080C942D1D0C942D1D7D
:100040000C942D1D0C944BDB0C942D1D0C942D1D2C
:100050000C942D1D0C94D6DC0C94EEDB0D949C03BB
:100060000C942D1D0C942EDD0C9458DD0C942D1D3C
:100070000C942D1D0C942D1D0C942D1D0C942D1DD8
:100080000C942D1D0C942D1D0C942D1D0C942D1DC8
:100090000C942D1D0C942D1D0C942D1D0D94AA0156
:1000A0000C942D1D0C942D1D0C942D1D0C942D1DA8
:1000B0000C942D1D0C942D1D0C942D1D0C942D1D98
:1000C0000C942D1D0C942D1D0C942D1D0C942D1D88
:1000D0000C942D1D0C942D1D0C942D1D0C942D1D78
:1000E0000C942D1DDD95F595F595F595F595F59502
:1000F000F595F595F595F595F595F595F595F595B0
:10010000F595F595F595F595F595F595F595F5959F
:10011000F595F595F595F595CC957E95889502958F
:10012000F595AE95B895F595F5951395F094F595EB
:10013000A495F595C2959A959295F595F595F595B1
:1001400060956A957495F595F595F595F595F59500
:10015000F595F595F595F595CC957E95889502954F
:10016000F595AE95B895F595F5951395F094F595AB
:10017000A495F595C2959A959295F595F595F59571
:1001800060956A957495F5B286B319B46AB505C4DD
:1001900005C405C405C405C405C405C405C405C417
:1001A000B2B4EEB42CB505C405C405C405C405C479
:1001B00005C405C405C405C405C405C491B8F3B895
:1001C00053B9B3B913BA73BAD3BA05C44FBF57BB47
:1001D000CDBB40BCB2BC24BD96BD08BE75BEE2BE60
:1001E00005C405C405C405C405C414B7E1B737B7D1
:1001F00097BF04C070C0DDC0FEC040C172C1A4C1C1
:10020000FDC158C2B1C20AC32BC31FC105C405C476
:1002100005C405C405C405C405C405C405C405C496
:1002200005C405C4B4B6E3B605C405C405C405C415
:1002300005C405C405C405C4ADC305C4B0B705C431
:1002400005C405C455C383C305C405C405C405C49A
:10025000E8B205C405C4ADB550B694B639B8A0012E
:100260008A018601B001AC01B201A80182017A01C4
:10027000C601B8018001BA019001B2019C01A2013E
:100280009A017E01BC01C201A60192018C01BE014E
:100290008401AE018E0178019401980188018C01DE
:1002A000C801C001C40107634236B79BD8A71A39F9
:1002B000685618AEBAAB558C1D3CB7CC5763BD6DB4
:1002C000EDFD753EF6177231BF000000803F05A8B6
:1002D0004CCDB2D44EB93836A9020C50B9918688AB
:1002E000083CA6AAAA2ABE000000803F0D942A005E
:1002F0000D94D8040D9434030D942B000D94BF0479
:100300000D9452030D942C030D94CA040D9406030E
:100310000D94E6040D9401030D94F9040D94D40496
:100320000D946B030D94BB040D94DE040D945700E3
:100330000D94E2040D9489030D9475030D9400004F
:100340000D94FC020D947F030D9490050D94B5045B
:100350000D9424030D941B000D941A030D94D004E6
:100360000D9410030D9493030D94CB000D9408008D
:100370000D9448030D9461030D94C2040D94C604BA
:100380000D94F0040D94B1040D94F4040D943E0307
:100390000D94EC04436F6C64206578747275736916
:1003A0006F6E20646973616C6C6F77656400436F76
:1003B0006C6420657874727573696F6E20616C6C03
:1003C0006F776564004175746F72657472616374F0
:1003D0003A0053657474696E67206D6F746F722094
:1003E00063757272656E742E2E2E00536574204DE7
:1003F0006963726F7374657070696E6700547269B7
:1004000067676572696E67207761746368646F6798
:100410002E204966206163746976617465642C20BE
:10042000746865207072696E7465722077696C6C8F
:100430002072657365742E0053657474696E67204D
:100440005468726573686F6C6420546F3A00494E4B
:10045000542050494E3A20004D323531200020744E
:100460006F200053657420766F6C756D65747269CA
:100470006320657874727573696F6E20666F722081
:100480006578747275646572200044697361626C8A
:10049000656420766F6C756D65747269632065782C
:1004A00074727573696F6E20666F722065787472EE
:1004B0007564657220004D313134200048656174E7
:1004C000696E67204265640048656174696E6720E3
:1004D00045787472756465720050696E2063616E50
:1004E000206E6F7420626520736574206279204DE0
:1004F00034322C206D617920696E20696E76616CD2
:100500006964206F7220696E207573652E20004922
:100510006C6C6567616C20532076616C7565206634
:100520006F72204D3432005A2028432920746F778F
:10053000657220666C6F6F722073657420746F3AF9
:100540002000592028422920746F77657220666C3C
:100550006F6F722073657420746F3A2000582028E2
:10056000412920746F77657220666C6F6F722073FB
:10057000657420746F3A2000526F64205261646980
:1005800075732073657420746F3A200047313334DB
:100590002000506F7346726F6D53746570733A002C
:1005A000436F6D7044656C74613A0043616C6962BD
:1005B000726174696F6E206D6F76656D656E742003
:1005C0006973206C696D6974656420746F203130C3
:1005D0006D6D2E004669727374206D6F76652074A0
:1005E0006F20746F75636820617420782C793D30BA
:1005F0002C3020746F206175746F2D7365742072B8
:1006000061646975732E0043616C6962726174691B
:100610006F6E206D6F76656D656E74206973206CEA
:10062000696D6974656420746F2031306D6D2E00C2
:1006300043616E6E6F7420736574207261646975B6
:100640007320616E6420666C6F6F7220617420731A
:10065000616D652074696D652E0043616C6962721D
:100660006174696F6E20636F6465206973206C69C3
:100670006D6974656420746F20626F74746F6D208F
:10068000313025206F66205A2068656967687400DC
:1006900052656C617469766520706F736974696FF7
:1006A0006E696E67004162736F6C75746520706F60
:1006B000736974696F6E696E670047363920005A36
:1006C0003A2000593A2000583A20004F46465345F8
:1006D0005453204F464620425920544F4F204D55E9
:1006E0004348205F20545259494E472041474149D1
:1006F0004E3A200053657474696E672050726F62C1
:10070000652053656E736974697669747920546FD6
:100710003A005A2070726F6265206661696C656488
:10072000206F6E2073656E73697469766974793AA7
:10073000200053657474696E672050726F62652083
:1007400053656E736974697669747920546F3A00E1
:100750005A2070726F6265206661696C6564206FF3
:100760006E2073656E73697469766974793A2000D6
:1007700053657474696E672050726F6265205365AB
:100780006E736974697669747920546F3A005A20DF
:1007900070726F6265206661696C6564206F6E209F
:1007A00073656E73697469766974793A2000686557
:1007B0006865004E6577205261646975733A200060
:1007C0004F6C64205261646975733A200043616C18
:1007D00063756C6174656420526164697573206926
:1007E0007320626164203A0053657474696E6720F7
:1007F00050726F62652053656E73697469766974AF
:100800007920546F3A005A2070726F6265206661D9
:10081000696C6564206F6E2073656E7369746976A8
:100820006974793A200053657474696E6720507258
:100830006F62652053656E73697469766974792097
:10084000546F3A005A2070726F6265206661696C5D
:100850006564206F6E2073656E7369746976697460
:10086000793A2000473332200050524F42452D5AEA
:100870004F46465345543A0047333000536574742D
:10088000696E672050726F62652053656E7369747C
:10089000697669747920546F3A0050726F6265739B
:1008A00020646F206E6F74206D617463682E204F1A
:1008B0006666206279200047333020004D313137A1
:1008C0002043414C4942524154494F4E20434F4DE1
:1008D000504C4554450068656865004E6577204872
:1008E0006F72697A6F6E74616C205261646975739E
:1008F0003A20004F6C6420486F72697A6F6E7461A1
:100900006C205261646975733A200043616C6375B1
:100910006C61746564205261646975732069732029
:100920006261643A20004D3131372043414C4942E5
:10093000524154494F4E204641494C454400436181
:100940006C6962726174696F6E204661696C65647E
:100950000053657474696E672050726F626520532E
:10096000656E736974697669747920546F3A005AB8
:100970002070726F626520284852202D205A207402
:100980006F77657229206661696C6564206F6E20DF
:1009900073656E73697469766974793A20004E657F
:1009A00077205A204865696768743A004F6C642064
:1009B0005A204865696768743A004D3131372043E1
:1009C000414C4942524154494F4E204641494C45C1
:1009D000440043616C6962726174696F6E204661A4
:1009E000696C65640053657474696E672050726F3A
:1009F00062652053656E73697469766974792054F1
:100A00006F3A005A2070726F626520284852202D7C
:100A10002043656E74657220506F696E742920667C
:100A200061696C6564206F6E2073656E73697469AB
:100A3000766974793A200047363920005A3A200006
:100A4000593A2000583A20004D31313720456E6424
:100A500073746F70204F6666736574204572726F91
:100A600072004F464653455453204F464620425944
:100A700020544F4F204D5543482E2041626F7274D1
:100A8000696E672E2053656E73697469766974792F
:100A90003A20004D3131372043414C4942524154B4
:100AA000494F4E204641494C45440043616C6962C0
:100AB000726174696F6E204661696C65640053658C
:100AC0007474696E672050726F62652053656E732F
:100AD0006974697669747920546F3A005A2070728B
:100AE0006F626520285A20546F77657229206661ED
:100AF000696C6564206F6E2073656E7369746976C6
:100B00006974793A20004D3131372043414C4942D4
:100B1000524154494F4E204641494C45440043619F
:100B20006C6962726174696F6E204661696C65649C
:100B30000053657474696E672050726F626520534C
:100B4000656E736974697669747920546F3A005AD6
:100B50002070726F626520285920546F7765722962
:100B6000206661696C6564206F6E2073656E7369C1
:100B70007469766974793A20004D313137204341E8
:100B80004C4942524154494F4E204641494C4544FC
:100B90000043616C6962726174696F6E20466169BD
:100BA0006C65640053657474696E672050726F627F
:100BB000652053656E736974697669747920546F22
:100BC0003A005A2070726F626520285820546F775F
:100BD000657229206661696C6564206F6E2073659B
:100BE0006E73697469766974793A2000456E64732E
:100BF000746F70287329206E6F7420776F726B6921
:100C00006E672070726F7065726C79005A2000599F
:100C100020005820004572726F723A20004D313129
:100C20003720454E4453544F50204552524F5200A6
:100C30004D3130342053300A4D3134302053300A96
:100C40004D313037004D3131372049324320457224
:100C5000726F722E2041626F7274696E6700493242
:100C600043204572726F72202D2043616C6962725D
:100C70006174696F6E2041626F7274656400456EC5
:100C80006473746F70287329206E6F7420776F728D
:100C90006B696E672070726F7065726C79005A2094
:100CA000005920005820004572726F723A20004DA2
:100CB00031313720454E4453544F50204552524F06
:100CC00052006578656375746547436F6465202FCE
:100CD00020717565756544656C74614D6F7665202E
:100CE00072657475726E73206572726F72006969D5
:100CF0007332646820616363656C65726F6D6574DF
:100D0000657220696E697469616C697A696E672EB3
:100D10002E2E00616363656C65726F6D657465721C
:100D2000206932632072656376206661696C656450
:100D30002E00616363656C65726F6D65746572200A
:100D4000777269746520693263206661696C6564D5
:100D50002E00616363656C65726F6D6574657220EA
:100D600073656E6420693263206661696C65642E08
:100D70000000000100250030001D000C001E0024B2
:100D80000031001C000B00180023002F001B000A7C
:100D90000017000D0047000300040022002B001A7A
:100DA0000041004200000002003500206465672E0B
:100DB000204300206D656173757265642000457283
:100DC000726F723A436F756C64206E6F7420686F37
:100DD0006C642074656D7065726174757265200055
:100DE000206D730020616674657220004572726F19
:100DF000723A54656D702E20726169736564207457
:100E00006F20736C6F772E2052697365203D200030
:100E10004739310A4731452D313830463630303088
:100E20000A473930004D3131372045787472756486
:100E3000657220300A54300A4D38342050340A4745
:100E400039310A47314531373246363030300A477A
:100E5000314535463530300A473930001C151C14F1
:100E60000000002243141F1F70121C12AC115C11F1
:100E7000000000000000D410C80F780FFC0E800E98
:100E80000400081D900058091C01B007A801C806FD
:100E900034023006C002C0054C036805D8031805AB
:100EA0006404D004F00498047C056004080630044F
:100EB000940600042007D003AC07A8033808800379
:100EC000C408580350093003DC090803680AD80233
:100ED000F40AB002800B88020C0C6002980C3002FD
:100EE000240DF801B00DC0013C0E8001C80E300188
:100EF000540FB800B40F2800E00F00000400401D9C
:100F0000900060091C01B007A801D0063402380621
:100F1000C002C8054C036805D80318056404D8044A
:100F2000F00498047C05600408063004940600046C
:100F30002007D003AC07A80338088003C40858036F
:100F400050093003DC090803680AE002F40AB80219
:100F5000800B88020C0C6002980C3002240DF80102
:100F6000B00DC0013C0E8001C80E3001540FB80016
:100F7000B40F2800E00F000004000016D800C006DF
:100F8000AC0178058002C004540348042804E80337
:100F9000FC049803D0055003A40618037807D80270
:100FA0004C08A80220097002F4093802C80A080295
:100FB0009C0BD001700C9001440D5001180EF800EC
:100FC000EC0E8800C00F00000400681D4C00500BA0
:100FD00094005809DC0050082401A8076C01280778
:100FE000B401C006FC017006440228068C02F0051C
:100FF000D402B8051C03880564035805AC0330050A
:10100000F40310053C04E8048404C804CC04A804D8
:10101000140590045C057004A4055804EC0538041C
:10102000340620047C060804C406F0030C07D80329
:101030005407C8039C07B003E40798032C088003F7
:1010400074087003BC085803040948034C093003B2
:1010500094091803DC090803240AF0026C0AE00270
:10106000B40AC802FC0AB002440BA0028C0B88022E
:10107000D40B70021C0C5802640C4002AC0C280209
:10108000F40C10023C0DF001840DD801CC0DB80118
:10109000140E98015C0E7001A40E4801EC0E1801AC
:1010A000340FD8007C0F8800C40F0800FC0F00002C
:1010B0000000000000000000000000000000000030
:1010C0000000000000000000000000000000000020
:1010D000000000000000401F450060094F0010099B
:1010E0005C00C0086B0070087D0020089200D007EB
:1010F000AC008007CC003007DE00E006230190063C
:101100005E014006A601F005FF01A0056D02500535
:10111000F30200059603B0045A046004400510046D
:101120004806C0036E077003A8082003EB09D0022D
:10113000230B8002410C3002390DE001040E9001B6
:10114000A20E4001170FF000690FA000A20F50007F
:10115000C60F0000DD0FB0FFEB0F60FF0400700D45
:10116000D8004804AC0158038002D802540380021E
:1011700028043802FC040002D005C801A406980126
:10118000780770014C08480120091801F409F000A3
:10119000C80AC8009C0BA000700C7000440D3800F9
:1011A000180E0000EC0EA8FFC00FE8FE0400001BA4
:1011B00054006009640010097400C00884007008BD
:1011C0009C002008B800D007D80080070001300735
:1011D0002C01E00668019006AC0140060002F00513
:1011E0006802A005E0025005740300052404B00461
:1011F000F0046004DC051004E406C0030408700376
:1012000030092003780B8002600DE001A80E400138
:10121000680FA000C00F0000E80F60FF0400801AF4
:10122000D8009808AC012007800250065403C80576
:1012300028045805FC040005D005B004A406680481
:10124000780728044C08E8032009B003F409700368
:10125000C80A38039C0BF802700CB002440D6802F7
:10126000180E0802EC0E8801C00F8800F00F000075
:101270000000A00F5C006009690010097900C00837
:101280008C007008A2002008BD00D007DE00800797
:10129000050130073401E0066D019006B2014006F9
:1012A0000702F0056D02A005E80250057B0300056A
:1012B0002B04B004F8046004EB06C00335092003D6
:1012C0007F0B8002650DE001B00E40011D0FF000A4
:1012D000480FC8006C0FA000ED0F60FFFE0F48FE26
:1012E000000200002110422063308440A550C660F7
:1012F000E770088129914AA16BB18CC1ADD1CEE1D3
:10130000EFF13112100273325222B5529442F77249
:10131000D662399318837BB35AA3BDD39CC3FFF322
:10132000DEE36224433420040114E664C774A44459
:1013300085546AA54BB528850995EEE5CFF5ACC572
:101340008DD55336722611163006D776F666955629
:10135000B4465BB77AA719973887DFF7FEE79DD7C2
:10136000BCC7C448E5588668A778400861180228B9
:101370002338CCC9EDD98EE9AFF9488969990AA912
:101380002BB9F55AD44AB77A966A711A500A333A89
:10139000122AFDDBDCCBBFFB9EEB799B588B3BBB62
:1013A0001AABA66C877CE44CC55C222C033C600C19
:1013B000411CAEED8FFDECCDCDDD2AAD0BBD688DB2
:1013C000499D977EB66ED55EF44E133E322E511E69
:1013D000700E9FFFBEEFDDDFFCCF1BBF3AAF599F02
:1013E000788F8891A981CAB1EBA10CD12DC14EF1A2
:1013F0006FE18010A100C230E32004502540467008
:101400006760B9839893FBA3DAB33DC31CD37FE332
:101410005EF3B1029012F322D23235421452776257
:101420005672EAB5CBA5A89589856EF54FE52CD502
:101430000DC5E234C324A0148104667447642454A7
:101440000544DBA7FAB79987B8975FE77EF71DC712
:101450003CD7D326F2369106B016576676761546F7
:1014600034564CD96DC90EF92FE9C899E9898AB962
:10147000ABA94458654806782768C018E108823847
:10148000A3287DCB5CDB3FEB1EFBF98BD89BBBAB72
:101490009ABB754A545A376A167AF10AD01AB32A97
:1014A000923A2EFD0FED6CDD4DCDAABD8BADE89DC2
:1014B000C98D267C076C645C454CA23C832CE01CE7
:1014C000C10C1FEF3EFF5DCF7CDF9BAFBABFD98F52
:1014D000F89F176E367E554E745E932EB23ED10E37
:1014E000F01E7C3C3E5E2B3D3F2F5B5D3B2C2A2259
:1014F0005C004D617854656D703A004469616D65BA
:101500007465723A00416363656C65726174696FFA
:101510006E3A004D617853706565643A004A6572B1
:101520006B3A004D617842656454656D703A0050C5
:1015300072696E746572547970653A44656C746151
:10154000005A54726176656C416363656C3A005968
:1015500054726176656C416363656C3A00585472ED
:101560006176656C416363656C3A005A5072696ECE
:1015700074416363656C3A00595072696E744163DB
:1015800063656C3A00585072696E74416363656CB0
:101590003A005A53697A653A005953697A653A00B4
:1015A0005853697A653A005A4D61783A00594D614D
:1015B000783A00584D61783A005A4D696E3A0059B0
:1015C0004D696E3A00584D696E3A004A65726B5823
:1015D000593A005072696E746C696E654361636854
:1015E000653A00454550524F4D3A004175746F6C55
:1015F0006576656C3A005A50726F62653A004361D5
:1016000073654C69676874733A00537570706F72D4
:10161000744C6F63616C46696C616D656E74636870
:10162000616E67653A00537570706F727447313040
:101630004731313A005A486F6D654469723A005932
:10164000486F6D654469723A0058486F6D6544692A
:10165000723A00536F667477617265506F77657286
:101660005377697463683A004C43443A0046616EAC
:101670003A005344436172643A004865617465649A
:101680004265643A004D6978696E67457874727591
:101690006465723A004E756D457874727564657252
:1016A0003A00496E7075744275666665723A00421A
:1016B000617564726174653A004E6F206361736591
:1016C000206C6967687473004D31313420006465A3
:1016D0006C6179203130306D732E00686F6D65411B
:1016E0007869732000686F6D6541786973202F20D9
:1016F000717565756544656C74614D6F76652072B2
:10170000657475726E73206572726F7200486F6DCA
:10171000652044656C7461005072696E7465723A3C
:101720003A736574757020006D6F7665546F5265FD
:10173000616C202F20717565756544656C74614D11
:101740006F76652072657475726E73206572726F44
:1017500072006D6F7665546F202F20717565756509
:1017600044656C74614D6F76652072657475726E38
:1017700073206572726F72005374657070657220A9
:1017800044697361626C6564004B696C6C656400EC
:101790006973506F736974696F6E416C6C6F7765B4
:1017A0006420005344206572726F72206669786508
:1017B00064005344206572726F7220646964206E05
:1017C0006F74207265636F766572210053442052F6
:1017D000656164204572726F720055706C6F616450
:1017E000696E672E2E2E00005344207072696E744D
:1017F0002073746F707065642062792075736572F0
:101800002E005344206361726420696E73657274A4
:101810006564005344204361726420696E7365728D
:1018200074656400534420436172642072656D6F77
:1018300076656400534420636172642072656D6F45
:1018400076656400457874722E00436F6E66696732
:101850003A004F6E65206865617465722073656536
:101860006D73206465636F75706C65642066726F5C
:101870006D20746865726D6973746F72202D2064B9
:10188000697361626C696E6720616C6C20666F724F
:101890002073616665747921004865617465722002
:1018A0006465636F75706C6564004372656174692B
:1018B0006F6E206661696C6564004469726563746B
:1018C0006F727920637265617465640044656C654C
:1018D00074696F6E206661696C65640046696C6549
:1018E0002064656C6574656400446F6E6520736187
:1018F00076696E672066696C652E00577269746937
:101900006E6720746F2066696C653A20006F7065A1
:101910006E206661696C65642C2046696C653A20AE
:10192000004E6F74205344207072696E74696E6744
:10193000005344207072696E74696E672062797416
:1019400065200066696C652E6F70656E2066616942
:101950006C65640046696C652073656C65637465CD
:1019600064002053697A653A0046696C65206F709F
:10197000656E65643A00456E642066696C65206C2E
:1019800069737400426567696E2066696C65206CD6
:10199000697374006572726F722077726974696E10
:1019A0006720746F2066696C6500534420696E6916
:1019B00074206661696C00616476616E6365204CB9
:1019C000205B303D6F66665D006578747275646596
:1019D0007220636F6F6C6572207370656564205B45
:1019E000302D3235355D0064697374616E63652036
:1019F000746F2072657472616374207768656E20FD
:101A000068656174696E67205B6D6D5D0074656DFE
:101A1000702E20666F722072657472616374696FD4
:101A20006E207768656E2068656174696E67205BFB
:101A3000435D0074656D702E2073746162696C691A
:101A40007A652074696D65205B735D00592D6F6642
:101A500066736574205B73746570735D00582D6FD9
:101A60006666736574205B73746570735D005049BE
:101A700044206D61782076616C7565205B302D3275
:101A800035355D0050494420442D6761696E005032
:101A9000494420492D6761696E0050494420502D0A
:101AA0006761696E2F646561642D74696D650050AE
:101AB0004944206472697665206D696E005049441E
:101AC000206472697665206D6178006865617420B4
:101AD0006D616E61676572205B302D335D006163FF
:101AE00063656C65726174696F6E205B6D6D2F73D9
:101AF0005E325D0073746172742066656564726144
:101B00007465205B6D6D2F735D006D61782E2066AE
:101B100065656472617465205B6D6D2F735D007324
:101B20007465707320706572206D6D00426564206D
:101B3000504944206D61782076616C7565205B307A
:101B40002D3235355D004265642050494420442DD6
:101B50006761696E004265642050494420492D67E1
:101B600061696E004265642050494420502D6761D0
:101B7000696E00426564205049442064726976654C
:101B8000206D696E0042656420504944206472698A
:101B90007665206D61780042656420486561742037
:101BA0004D616E61676572205B302D335D00436F60
:101BB00072722E20646961676F6E616C2043205BD6
:101BC0006D6D5D00436F72722E20646961676F6E88
:101BD000616C2042205B6D6D5D00436F72722E2040
:101BE000646961676F6E616C2041205B6D6D5D00A3
:101BF0004D6178207072696E7461626C65207261EB
:101C000064697573205B6D6D5D00546F776572203C
:101C10005A20656E6473746F70206F6666736574A6
:101C2000205B73746570735D00546F776572205923
:101C300020656E6473746F70206F666673657420C0
:101C40005B73746570735D00546F77657220582004
:101C5000656E6473746F70206F6666736574205B65
:101C600073746570735D005365676D656E74732F73
:101C70007320666F722074726176656C00536567BD
:101C80006D656E74732F7320666F72207072696E4B
:101C900074696E6700486F72697A6F6E74616C2048
:101CA000726F642072616469757320617420302CD6
:101CB00030205B6D6D5D00446961676F6E616C2003
:101CC000726F64206C656E677468205B6D6D5D007B
:101CD000486F6D696E672066656564726174652022
:101CE0005B6D6D2F735D004D61782E2066656564B8
:101CF00072617465205B6D6D2F735D005374657048
:101D00007320706572206D6D0054726176656C2071
:101D1000616363656C65726174696F6E205B6D6D84
:101D20002F735E325D00416363656C657261746937
:101D30006F6E205B6D6D2F735E325D004D61782E8E
:101D4000206A65726B205B6D6D2F735D005A206D8C
:101D50006178206C656E677468205B6D6D5D0059FD
:101D6000206D6178206C656E677468205B6D6D5DB9
:101D70000058206D6178206C656E677468205B6D1B
:101D80006D5D005A20686F6D6520706F73205B6D0C
:101D90006D5D005920686F6D6520706F73205B6DFD
:101DA0006D5D005820686F6D6520706F73205B6DEE
:101DB0006D5D0053746F7020737465707065722070
:101DC000616674657220696E61637469766974799D
:101DD000205B6D732C303D6F66665D004D61782E23
:101DE00020696E6163746976652074696D65205B36
:101DF0006D732C303D6F66665D005072696E746560
:101E00007220616374697665205B735D0046696C5E
:101E1000616D656E74207072696E746564205B6DAF
:101E20005D00416476616E63656420557365720080
:101E30004261756472617465004550523A33200006
:101E40004550523A3220004550523A312000455018
:101E5000523A30200050726F746F636F6C20766559
:101E60007273696F6E206368616E6765642C20759C
:101E70007067726164696E6700436F6E666967754B
:101E8000726174696F6E20726573657420746F205F
:101E900064656661756C74732E00436F6E66696766
:101EA00075726174696F6E206C6F61646564206621
:101EB000726F6D20454550524F4D2E00436F6E6638
:101EC000696775726174696F6E2073746F7265648F
:101ED00020746F20454550524F4D2E004175746F50
:101EE0006C6576656C206163746976652028312F96
:101EF0003029005A2D70726F6265205933005A2DB7
:101F000070726F6265205833005A2D70726F62656F
:101F1000205932005A2D70726F6265205832005A73
:101F20002D70726F6265205931005A2D70726F6288
:101F300065205831005A2D70726F626520782D79B6
:101F40002D7370656564205B6D6D2F735D005A2D78
:101F500070726F6265207370656564205B6D6D2FB4
:101F6000735D005A2D70726F6265206F66667365CF
:101F7000742079205B6D6D5D005A2D70726F626503
:101F8000206F66667365742078205B6D6D5D004D13
:101F900061782E207A2D70726F6265202D20626527
:101FA0006420646973742E205B6D6D5D005A2D7022
:101FB000726F626520686569676874205B6D6D5D2E
:101FC0000077616974005072696E7465722068658B
:101FD000696768743A005A2D70726F626520666195
:101FE000696C6564005472616E73666F726D6174C2
:101FF000696F6E206D61747269783A004175746F13
:102000006C6576656C696E672064697361626C6586
:1020100064004175746F6C6576656C696E672065E8
:102020006E61626C6564004175746F6C6576656C99
:10203000206D617472697820726573657400004761
:1020400032382F6E47315A32352F6E005A2D70724A
:102050006F62652073746174653A005265736574CC
:10206000205A20686569676874005A2D70726F6223
:102070006520617665726167652068656967687467
:102080003A00205374657020566172696174696FFB
:102090006E2066726F6D2050726F626520746F20C3
:1020A0006265642044697374616E63653A005A2DF9
:1020B00070726F62653A005072696E746572207357
:1020C000657420696E746F206472792072756E2059
:1020D0006D6F646520756E74696C207265737461D0
:1020E000727421003A20776F726B696E67003A2034
:1020F00074656D702073656E736F722064656665BC
:102100006374006578747275646572200068656137
:1021100074656420626564004D54454D503A00502A
:102120004944204175746F74756E652066696E69E7
:1021300073686564202120506C6163652074686554
:10214000204B702C204B6920616E64204B6420630F
:102150006F6E7374616E747320696E20746865208D
:10216000436F6E66696775726174696F6E2E682061
:102170006F7220454550524F4D00504944204175E3
:10218000746F74756E65206661696C656421207476
:10219000696D656F757400504944204175746F74A2
:1021A000756E65206661696C6564212054656D708B
:1021B0006572617475726520746F20686967680064
:1021C000204B643A2000204B693A2000204B703AA3
:1021D000200020436C6173736963205049440020E0
:1021E00054753A2000204B753A2000206D61783AF2
:1021F0002000206D696E3A200020643A20002062A1
:102200006961733A2000504944204175746F7475B8
:102210006E652073746172740054617267657442F4
:1022200065643A0054617267657445787472004E53
:102230006F206D6F766520696E2064656C74612017
:102240007365676D656E742077697468203E203110
:10225000207365676D656E742E20546869732073F2
:10226000686F756C64206E65766572206861707049
:10227000656E20616E64206D6179206361757365A0
:1022800020612070726F626C656D210044656C7412
:10229000612052616469757320432830293A0044F3
:1022A000656C74612052616469757320422830291D
:1022B0003A0044656C746120526164697573204111
:1022C0002830293A00416C70686120432839302950
:1022D0003A00416C706861204228333330293A005B
:1022E000416C706861204128323130293A00546FC6
:1022F00077657220333A00546F77657220323A0066
:10230000546F77657220313A00496E76616C69646A
:102310002064656C746120636F6F7264696E6174B0
:1023200065202D206D6F76652069676E6F7265641C
:10233000006C696E656172204C3A00454550524F01
:102340004D2075706461746564002C207370656540
:10235000643D00206C696E656172207374657073F2
:102360003A004A65726B3A007A5F6D61783A00799B
:102370005F6D61783A00785F6D61783A004C2000BB
:10238000482000206973200020746F20005365747A
:10239000206F75747075743A20004D53312C4D5375
:1023A000322050696E730045313A0045303A005A88
:1023B0003A00593A0020002C00206D696E00206818
:1023C0006F7572732000206461797320006D2000A6
:1023D0005072696E74696E672074696D653A005059
:1023E00072696E7465642066696C616D656E743ABD
:1023F0000046616E73706565643A00482E20526134
:10240000646975733A00466C6F774D756C746970CA
:102410006C793A0053706565644D756C7469706CC5
:10242000793A00202F002F003A0020524157002017
:1024300042403A0020403A0020423A00543A0020FC
:10244000453A00205A3A0020593A0020583A00589C
:102450003A00467265652052414D3A00556E6B6EEA
:102460006F776E20636F6D6D616E643A00536F66B7
:102470007477617265205265736574005761746387
:1024800068646F672052657365740042726F776E7F
:10249000206F757420526573657400457874657299
:1024A0006E616C20526573657400506F776572556C
:1024B0007000737461727400424C4B2000736B693E
:1024C00070200020676F7420004572726F723A6549
:1024D00078706563746564206C696E652000534490
:1024E0002072656164206572726F72002052002054
:1024F0004A0020490020500020530020460020457B
:1025000000205A00205900205800446F6E6520704A
:1025100072696E74696E672066696C6500466F72D9
:102520006D6174206572726F720057726F6E6720F2
:10253000636865636B73756D004563686F3A00523D
:102540006573656E643A005761726E696E673A0032
:10255000496E666F3A004572726F723A00494E4694
:10256000004E414E006F6B004649524D5741524557
:102570005F4E414D453A52657065746965725F30D2
:102580002E39322E32204649524D574152455F4432
:102590004154453A3230313731313133204D4143A6
:1025A00048494E455F545950453A4F52494F4E2085
:1025B00044656C7461200052657175657374506177
:1025C0007573653A004D31313720494E53455254A9
:1025D0002053442043415244004D3131372053446D
:1025E0002043415244204552524F520055495F41C9
:1025F0004354494F4E5F5345545F4D4541535552E7
:1026000045445F4F524947494E20004E6F20534486
:1026100020436172640053687574204F66662041E0
:102620004C4C204865617473005072656865617434
:1026300020414253005072656865617420504C41DE
:102640000055495F414354494F4E5F484F4D455FE8
:102650005A200055495F414354494F4E5F484F4D02
:10266000455F59200055495F414354494F4E5F48EB
:102670004F4D455F58200055495F414354494F4EE7
:102680005F484F4D45414C4C200055495F414354F4
:10269000494F4E5F5A504F534954494F4E5F464140
:1026A00053545F4E4F54455354200055495F4143A6
:1026B00054494F4E5F5A504F534954494F4E5F4E05
:1026C0004F54455354200055495F414354494F4EA0
:1026D0005F45504F534954494F4E200055495F4183
:1026E0004354494F4E5F5A504F534954494F4E5FE0
:1026F00046415354200055495F414354494F4E5F72
:1027000059504F534954494F4E5F4641535420004E
:1027100055495F414354494F4E5F58504F534954B8
:10272000494F4E5F46415354200055495F41435441
:10273000494F4E5F5A504F534954494F4E20005510
:10274000495F414354494F4E5F59504F5349544993
:102750004F4E200055495F414354494F4E5F5850FA
:102760004F534954494F4E200042616E6742616E9B
:102770006700536C6F7742616E6700446561642047
:1027800054696D650050494400003A002064617945
:1027900073200050657263656E74205072696E74A8
:1027A00065643A00206465662000465720446174E1
:1027B00065203230313731313133004F52494F4E7D
:1027C0002044656C7461005365654D65434E43005C
:1027D0004F52494F4E2044656C74610076342C345E
:1027E000C2336533416374696F6E3A256C610004CE
:1027F0000003004E6F00596573004E2F41004F6675
:1028000066004F6E000000003FCDCC4C3D0AD7A3C0
:102810003B6F12033A5265706574696572207620C9
:10282000302E39322E3200004014548025000040F2
:10283000380000004B00008070000000960000C0CF
:10284000DA000000E10000002C010008B2010000E5
:10285000C2010000F401000084030090D0030000D6
:10286000E803000008070020A1070000100E004048
:10287000420F0060E3160000000000110A0411047A
:102880000A1111001C1F11111F0000040A0A0A0E70
:102890001F1F0E001F1111111F0000001F1F1F1FFF
:1028A0001F0000040A040000000000040E15041CB0
:1028B0000000000200000600BA28EC302029A12DFB
:1028C000F328F42D62290200000700CD28EC30DB4C
:1028D00028A12DF328F42D2C2D0729E22802A22E61
:1028E00000005072696E7465722053657474696E6D
:1028F000677300FA2802902F000041646A757374B0
:102900002054656D7073000E29023829000041645F
:1029100076616E6365642053657474696E677300D5
:10292000272902BB2E00005072696E746572205315
:10293000657474696E67730002000009003F29EC3A
:10294000304D2A392A292A192A5129022AEA2962CC
:1029500029582902CF2C0000446562756767696EAB
:102960006700692902CD2F000043616C69627261C2
:1029700074696F6E204D656E75000310270200812B
:10298000298C29852993290000000000A429000032
:102990000000006C6F6164656420662E2045455020
:1029A000524F4D00436F6E66696775726174696F4F
:1029B0006E000310270200B929C429BD29CB2900C4
:1029C00000000000DC29000000000073746F7265D5
:1029D0006420696E20454550524F4D00436F6E662E
:1029E000696775726174696F6E00F12903070400ED
:1029F000004C6F61642066726F6D20454550524FE8
:102A00004D00092A030604000053746F7265207498
:102A10006F20454550524F4D00202A025C2A00008D
:102A2000457874727564657200302A02632C000068
:102A3000466565647261746500402A028F2C00004F
:102A4000416363656C65726174696F6E00542A023C
:102A5000AF2B000047656E6572616C0002000010CC
:102A600000632AEC309B2B872B752B642B4F2B207C
:102A70002B382B092BF62AE22AD12AC02AAB2A9618
:102A80002A832A8A2A042F040000504944204D61D9
:102A9000783A255844009D2A0426040000447269AF
:102AA0007665204D61783A25584D00B22A042504F8
:102AB00000004472697665204D696E3A25586D00B4
:102AC000C72A042404000050494420443A2558648D
:102AD00000D82A042304000050494420493A2558CC
:102AE0006900E92A042204000044542F504944207C
:102AF000503A25587000FD2A042D040000436F6EE3
:102B000074726F6C3A25586800102B04460400005C
:102B1000416476616E6365206C696E3A25586C007D
:102B2000272B044D0400005761697420556E6974A9
:102B3000733A2558556D6D003F2B044C0400005727
:102B40006169742054656D702E25585402430056F7
:102B50002B042E040000537461622E54696D653A93
:102B6000255877006B2B042A040000416363656CD1
:102B70003A255841007C2B042B0400004D6178203D
:102B800046523A255846008E2B042C0400005374FC
:102B90006172742046523A25586600A22B0429041B
:102BA000000053746570732F4D4D3A255365000234
:102BB00000000400B62BEC30EB2BD32BBE2BC52B27
:102BC00002FF2B00004D61782E20496E616374690D
:102BD000766500DA2B02312C000053746570706545
:102BE0007220496E61637469766500F22B041004EB
:102BF000000042617564726174653A256F63000379
:102C000058040200062C112C0A2C182C000000007D
:102C100000222C00000000005B735D20303D4F66F9
:102C200066004469732E2041667465723A256970A6
:102C3000000320040200382C432C3C2C4A2C0000BA
:102C4000000000542C00000000005B735D20303D4C
:102C50004F6666004469732E2041667465723A259A
:102C600069730002000003006A2CEC30802C702C89
:102C7000772C0413040000486F6D653A25665A00EE
:102C8000872C04160400004D61783A25667A00020C
:102C900000000400962CEC30BE2CAE2C9E2CA52CF3
:102CA000040E0400004A65726B3A25616A00B52C77
:102CB000040D0400004D6F76653A25615A00C52C5D
:102CC000040A0400005072696E743A25617A0002A9
:102CD00000000500D62CEC30192D062DF32CE02C2D
:102CE000E72C03350400004472792072756E3A2592
:102CF000646400FA2C03340400004572726F72732E
:102D0000203A256465000D2D0333040000496E66EA
:102D10006F2020203A25646900202D033204000032
:102D20004563686F2020203A25646F00332D0240F0
:102D30002D000053442043617264204D656E750080
:102D40000200000600472DEC30A12D8E2D782D6657
:102D50002D532D5A2D03F403010244656C657465EF
:102D60002066696C65006D2D02C02D020053746FE2
:102D700070205072696E74007F2D03F703040043C6
:102D80006F6E74696E7565205072696E7400952D52
:102D900003F60302045061757365205072696E7406
:102DA00000A82D03F503010253656C65637420537D
:102DB000442046696C65000100000100BE2DEC3026
:102DC0000200000300C72DE22DD82DCD2DD42D03F8
:102DD0005424020059657300DF2D03E80300004E00
:102DE0006F00E92D010000000053746F70205072D5
:102DF000696E7400FB2D020C2E000041646A75732D
:102E0000742046616E2073706565640002000007DF
:102E100000132EEC308A2E762E612E4C2E372E216A
:102E20002E282E031E0400005365742046616E2078
:102E3000313030252525003E2E031D04000053654A
:102E4000742046616E20373525252500532E031C3E
:102E50000400005365742046616E20353025252519
:102E600000682E031B0400005365742046616E2029
:102E70003235252525007D2E031A0408005475726D
:102E80006E2046616E204F666600912E045204004B
:102E90000046616E2073706565643A25467325258A
:102EA00025000200000A00A92EEC30072FEE2E6547
:102EB0002F522F382FD830202F782F0200000A00F1
:102EC000C22EEC30072FEE2E652F522F382FD83020
:102ED000D62E202F782FDD2E03B20F0000556E6CFA
:102EE0006F636B2046756C6C204D656E7500F52E1A
:102EF0000448040000466C6F772020526174653AE4
:102F0000256F66252525000E2F041F040000537031
:102F100065656420526174653A256F6D252525002D
:102F2000272F034204001044697361626C652053CB
:102F300074657070657273003F2F0338040000538E
:102F4000687574204F666620414C4C20486561745A
:102F50007300592F0347040000507265686561745F
:102F600020414253006C2F03370400005072656803
:102F700065617420504C41007F2F033604000041EE
:102F8000545820706F776572206F6E2F6F666600E1
:102F90000200000400972FEC30B52F9D2FA42F04C2
:102FA0003C0400004245442054656D703A202025C1
:102FB0004562024300BC2F043D0400004E4F5A20DE
:102FC00054656D703A202025453002430002000010
:102FD0000600D42FEC300A30E02FD830A230F62F84
:102FE000E72F0421040000482E20526164697573A4
:102FF000203A256F6800FD2F03AC0F000053657465
:10300000205A204F726967696E0011300222300029
:103010000046756C6C2043616C6962726174696F03
:103020006E0002000004002930EC305F304A30317D
:1030300030383003B10F0000426567696E2043618C
:103040006C6962726174696F6E00513003B50F0074
:10305000004245442041524520434C45414E0066C4
:103060003003B40F00004D414B45205355524520CD
:103070004E4F5A5A4C452026000200000600803070
:10308000EC30D830C630B430A2308C3093300205EA
:10309000310000457874722E20706F736974696F07
:1030A0006E00A93002663200005A20506F736974B6
:1030B000696F6E00BB3002BB3200005920506F7345
:1030C0006974696F6E00CD300210330000582050D3
:1030D0006F736974696F6E00DF3003FD0300004891
:1030E0006F6D65205072696E74657200F33003E88D
:1030F00003000050726576696F75732053637265C3
:10310000656E20010003F00304000C3129312231E7
:103110001B311431303100000000003E310000004E
:1031200000004F3100000000005E31000000000090
:10313000255566206D207072696E746564002045A7
:103140003A2565632F25456302437E256F43003191
:1031500020636C69636B203D2031206D6D00453A22
:10316000257833206D6D0003FC0304006E318B3134
:1031700084317D31763192310000000000933100BE
:1031800000000000A3310000000000B33100000087
:103190000000004D617820656E6473746F703A258D
:1031A000735A004D696E20656E6473746F703A25B2
:1031B000737A005A3A257832206D6D0003FB0304C0
:1031C00000C331E031D931D231CB31E731000000D9
:1031D0000000E8310000000000F8310000000000AD
:1031E00008320000000000004D617820656E6473B5
:1031F000746F703A257359004D696E20656E647363
:10320000746F703A25737900593A257831206D6DC5
:103210000003FA030400183235322E3227322032EE
:103220003C3200000000003D3200000000004D3242
:1032300000000000005D320000000000004D6178D9
:1032400020656E6473746F703A257358004D696E13
:1032500020656E6473746F703A25737800583A2550
:103260007830206D6D0003EF0304006D328A3283E5
:10327000327C327532913200000000009232000040
:10328000000000A2320000000000B2320000000086
:1032900000004D617820656E6473746F703A257319
:1032A0005A004D696E20656E6473746F703A2573B1
:1032B0007A005A3A257832206D6D0003EE0304003F
:1032C000C232DF32D832D132CA32E63200000000D8
:1032D00000E7320000000000F732000000000007A5
:1032E000330000000000004D617820656E64737447
:1032F0006F703A257359004D696E20656E64737462
:103300006F703A25737900593A257831206D6D0038
:1033100003ED030400173334332D3326331F333BBF
:103320003300000000003C3300000000004C33007C
:10333000000000005C330000000000004D617820B8
:10334000656E6473746F703A257358004D696E2012
:10335000656E6473746F703A25737800583A2578F7
:1033600030206D6D0000000004006C33893382331F
:103370007B3374339033000000000096330000006C
:103380000000AA330000000000AE3300000000007F
:10339000255566206D00546F74616C2046696C6120
:1033A0006D656E7420557365640025557400546F07
:1033B00074616C205072696E74696E672054696D17
:1033C00065000000000400C933E633DF33D833D191
:1033D00033ED330000000000F93300000000000767
:1033E000340000000000193400000000004F524972
:1033F0004F4E2044656C7461005072696E74657242
:10340000204D6F64656C00465720446174653A2016
:1034100032303137313131330046572056657273BF
:10342000696F6E3A20302E39322E320000000004CF
:103430000033345034493442343B345734000000B4
:1034400000005B3400000000006434000000000055
:103450006D340000000000256F73005A3A25783261
:10346000206D6D00593A257831206D6D00583A2550
:103470007830206D6D0000000004007D349A349394
:10348000348C348534A1340000000000A5340000E1
:10349000000000BE340000000000D1340000000035
:1034A00000256F730053706565643A256F6D25259F
:1034B0002520466C6F773A256F6625252500424505
:1034C000443A256562205461726765743A25456205
:1034D000004E4F5A3A256563205461726765743A0D
:1034E000254563000000000000000000000000FF10
:1034F00000000100000000000000000000000000CB
:103500000000000024F403D950C38EB1C2A23D963E
:10351000828B3582127AE372816CCB66A861015D81
:10352000C758EB546151204E1E4B5648C145594374
:103530001A41013F093D2F3B7139CD374036C9341F
:1035400065331432D430A32F802E6B2D632C672B60
:10355000752A8E29B028DC2710274B268F25D924E1
:103560002B248223E0224322AC211A218D20042027
:10357000801F001F841E0C1E971D261DB81C4E1C8C
:10358000E61B821B201BC11A641A0A1AB2195D19A4
:103590000A19B9186A181C18D11788174017FA1693
:1035A000B51673163116F115B31576153A150015C3
:1035B000C7148F1458142214EE13BA138813561319
:1035C0002513F612C71299126C1240121512EB1144
:1035D000C1119811701148112111FB10D610B110B2
:1035E0008D106910461024100210E10FC00FA00FBB
:1035F000800F610F420F230F060FE80ECB0EAF0EA8
:10360000930E770E5C0E410E270E0D0EF30DDA0DA4
:10361000C10DA80D900D780D600D490D320D1B0DDB
:10362000050DEF0CD90CC30CAE0C990C850C700C6D
:103630005C0C480C350C210C0E0CFB0BE80BD60B6C
:10364000C40BB20BA00B8E0B7D0B6B0B5A0B4A0BF2
:10365000390B290B180B080BF80AE90AD90ACA0A10
:10366000BB0AAC0A9D0A8E0A800A710A630A550ACF
:10367000470A390A2C0A1E0A110A040AF709EA093C
:10368000DD09D009C409B709AB099F099209870967
:103690007B096F09630958094C09410936092B094F
:1036A000200915090A090009F508EB08E008D60801
:1036B000CC08C208B808AE08A4089A089008870881
:1036C0007D0874086B08610858084F0846083D08D3
:1036D00034082C0823081A08120809080108F807FA
:1036E000F007E807E007D807D007C807C007B80702
:1036F000B007A807A1070000420FA1071605D003D5
:103700000D038B022E02E801B2018601630145011F
:103710002C0117010401F4004F52494F4E2052650D
:10372000616479004F52494F4E20526561647900BF
:103730004F52494F4E20526561647900207A3A0019
:1037400020793A0020783A00696E207175657565B8
:1037500044656C74614D6F766520746F2063616C95
:1037600063756C61746544656C746153756253650F
:10377000676D656E74732072657475726E73206503
:1037800072726F722E00432068697420666C6F6FCE
:10379000720043706F7320782073717561726520B9
:1037A0000043706F7320782073746570732000433A
:1037B000706F73207920737175617265200043709A
:1037C0006F732079207374657073200042206869DC
:1037D0007420666C6F6F720042706F732078207374
:1037E0007175617265200042706F73207820737468
:1037F000657073200042706F73207920737175615A
:103800007265200042706F73207920737465707345
:103810002000412068697420666C6F6F72004170EF
:103820006F73207820737175617265200041706F2D
:10383000732078207374657073200041706F73205B
:103840007920737175617265200041706F73207902
:1038500020737465707320006D6F766552656C61BE
:103860007469766544697374616E6365496E5374F7
:10387000657073202F20717565756544656C746182
:103880004D6F76652072657475726E732065727205
:103890006F720000000A0B02090C0D0E08070304EA
:1038A0000100000000000000000000000000000017
:1038B00000000000000000000000000000000012F6
:1038C00011100000000000000000000000000000D7
:1038D0000000000000000000000102102020080885
:1038E0001020401020408002010201080402010162
:1038F000020408102040808040201008040201804B
:1039000004020180402010080402010804020101A1
:1039100002040810204080010204081020408005A5
:10392000050505070508080808020202020A0A0838
:10393000080404040401010101010101010303035E
:103940000303030303040707070C0C0C0C0C0C0CFB
:103950000C0202020206060606060606060B0B0B02
:103960000B0B0B0B0B000020002300260029002C62
:10397000002F0032000001000003010601090100D0
:10398000002200250028002B002E00310034000208
:10399000010000050108010B01000021002400279F
:1039A000002A002D0030003300010100000401074F
:1039B000010A01024E414E494E495459494E46CDE5
:1039C000CCCC3D0AD7233C17B7D13877CC2B3295D6
:1039D00095E6241FB14F0A000020410000C84200B4
:1039E000401C4620BCBE4CCA1B0E5AAEC59D74007E
:1039F0004590829F08DEB40111241FBECFEFD1E2B3
:103A0000DEBFCDBF00E00CBF13E0A0E0B2E0EEEA05
:103A1000F4E202E00BBF02C007900D92A638B10796
:103A2000D9F72EE1A6E8B3E001C01D92AE37B20788
:103A3000E1F719E3C8EFD9E300E006C022970109D6
:103A4000FE010BBF0F94D00DC03FD10780E00807E7
:103A5000A9F70F943C090D9455120C940000CF93D4
:103A6000DF9300D01F92CDB7DEB744E050E0BC0139
:103A7000CE0101960F94111269817A818B819C810C
:103A80000F900F900F900F90DF91CF91089580913C
:103A9000EA0283FB882780F90895179A0895169AF9
:103AA0000895159A089580B182FB882780F90895BA
:103AB00080B186958170089588E493E0D0CFCF924D
:103AC000DF92EF92FF92CF93DF9300D01F921F926D
:103AD000CDB7DEB76B017C0160936D0770936E0705
:103AE00080936F07909370070E94E374C982DA8213
:103AF000EB82FC8244E050E065E773E0CE01019682
:103B00000F94331223E0B701A60188E795E00E94E5
:103B10009DA10E9440CF682F88E690E06D830F94AE
:103B200021126D81681721F088E690E00F943C1215
:103B30000F900F900F900F900F90DF91CF91FF900B
:103B4000EF90DF90CF900895CF93DF931F92CDB782
:103B5000DEB7BC018DE793E00F944F120E9440CF77
:103B6000682F88E690E069830F94211269816817B5
:103B700039F088E690E00F90DF91CF910D943C12E0
:103B80000F90DF91CF910895CF93DF931F92CDB720
:103B9000DEB7BC018FE793E00F944F120E9440CF35
:103BA000682F88E690E069830F9421126981681775
:103BB00039F088E690E00F90DF91CF910D943C12A0
:103BC0000F90DF91CF910895CF93DF931F92CDB7E0
:103BD000DEB7BC0181E893E00F944F120E9440CF02
:103BE000682F88E690E069830F9421126981681735
:103BF00039F088E690E00F90DF91CF910D943C1260
:103C00000F90DF91CF910895CF93C82F80919C049E
:103C10008823D1F010929C040E94085A9091DF02F0
:103C200091509093DF02911109C08091E00283309E
:103C300010F40E94955985E08093DF026C2F8CE68A
:103C40009AE0CF910C9475CACF9108958091210C80
:103C5000882349F00E94629880E0D6DF8CE69AE0E3
:103C60000E9474CAF3CF08954F925F926F927F9231
:103C70008F929F92AF92BF92CF92DF92EF92FF927C
:103C80000F931F93CF93DF9300D01F92CDB7DEB772
:103C90008C018091E7079091E807A091E907B09126
:103CA000EA0789839A83AB83BC83C090EB07D090EB
:103CB000EC07E090ED07F090EE078090EF07909012
:103CC000F007A090F107B090F2079C01AD01BC0194
:103CD000CD010F94020D81110FC149805A806B8074
:103CE0007C80E89477F82FEF3FEF4FE75FE7C30161
:103CF000B2010F94020D81110BC02FEF3FEF4FE780
:103D00005FE7C301B2010F94AF0918160CF4F4C0B9
:103D1000A7019601C701B6010F94020D8111ECC0F5
:103D200026013701E89477F82FEF3FEF4FE75FE781
:103D3000C301B2010F94020D81110BC02FEF3FEFB1
:103D40004FE75FE7C301B2010F94AF0918160CF4F7
:103D5000D3C0A5019401C501B4010F94020D8111D6
:103D6000CBC024013501E89477F82FEF3FEF4FE700
:103D70005FE7C301B2010F94020D81110BC02FEF59
:103D80003FEF4FE75FE7C301B2010F94AF09181689
:103D90000CF4B2C02091BF073091C0074091C10719
:103DA0005091C20769817A818B819C810F944B0964
:103DB0002B013C012091C3073091C4074091C507F6
:103DC0005091C607C701B6010F944B096B017C01E6
:103DD0002091C7073091C8074091C9075091CA0781
:103DE000C501B4010F944B094B015C018091470858
:103DF000882329F020E732E441E25DE304C020E0BB
:103E000030E040E85FE3C301B2010F94570CAB010F
:103E1000BC0122E08FE494E20E94DAA1809147087D
:103E2000882329F020E732E441E25DE304C020E08A
:103E300030E040E85FE3C701B6010F94570CAB01D7
:103E4000BC0122E087E494E20E94DAA18091470855
:103E5000882329F020E732E441E25DE304C020E05A
:103E600030E040E85FE3C501B4010F94570CAB01AB
:103E7000BC0123E083E494E20E94DAA16091FF0791
:103E80007091000880910108909102080F94820AB5
:103E900020914308309144084091450850914608CC
:103EA0000F94570C20914708222329F020E732E491
:103EB00041E25DE304C020E030E040E85FE30F94BE
:103EC000570CAB01BC0124E08FE394E20F900F90FC
:103ED0000F900F90DF91CF911F910F91FF90EF9076
:103EE000DF90CF90BF90AF909F908F907F906F901A
:103EF0005F904F900C949DA1C8010E94BF9F4ACF34
:103F0000CF92DF92EF92FF92CF93DF93EC01893152
:103F100091053CF0C53F81E0D8072CF0C4EFD1E01B
:103F200002C0C9E1D0E0BE01882777FD8095982FB7
:103F30000F94820A6B017C016091F7067091F8067C
:103F4000882777FD8095982F0F94820A9B01AC01FA
:103F5000C701B6010F94B6099B01AC016091F90647
:103F60007091FA068091FB069091FC060F94570C15
:103F70006093F9067093FA068093FB069093FC0613
:103F8000D093F806C093F706BE0184E194E2DF9176
:103F9000CF91FF90EF90DF90CF900C9483A0CF92C1
:103FA000DF92EF92FF926B017C0120E030E040E76E
:103FB00052E40F94AF0987FD11C020E030E046E1E4
:103FC00053E4C701B6010F94E30B18166CF4C12C2F
:103FD000D12C86E1E82E83E4F82E06C0C12CD12C2A
:103FE00090E7E92E92E4F92EC0926D07D0926E0709
:103FF000E0926F07F092700722E0B701A6018BEF05
:1040000093E2FF90EF90DF90CF900C949DA18F9260
:104010009F92AF92BF92CF92DF92EF92FF92CF9397
:10402000DF93EC018931910534F0893C91052CF046
:10403000C8ECD0E002C0C9E1D0E0D093F606C0934E
:10404000F506E0918603F0918703E258FF4FC080A8
:10405000D180E280F38020E030E0A901C701B60101
:104060000F94AF09AE01662757FD6095762F18169D
:104070005CF0CB01BA010F94820A2AE037ED43E2EB
:104080005CE30F94570C24C0CB01BA010F94820A51
:104090002AE037ED43E25CE30F94570C20E030E078
:1040A00040E850E40F94570C4B015C01A7019601C6
:1040B000C701B6010F94570C2BED3FE049E450E4E3
:1040C0000F94570C9B01AC01C501B4010F94B609C4
:1040D0006093E5027093E6028093E7029093E80212
:1040E000BE0186E094E2DF91CF91FF90EF90DF90E8
:1040F000CF90BF90AF909F908F900C9483A0CF9360
:10410000DF932091BB0797FD0DC0EC018F3F910518
:1041100019F014F0CFEFD0E0209721F02860209321
:10412000BB0705C0277F2093BB07C0E0D0E061112B
:104130008DDD80917A1D90E0C817D90729F0BE0166
:1041400081EF93E20E9483A0C0937A1DDF91CF910B
:1041500008954F925F926F927F928F929F92AF924B
:10416000BF92CF92DF92EF92FF92CF93DF9300D076
:104170001F92CDB7DEB72FE632E143E85AE36091F4
:10418000DF067091E0068091E1069091E2060F94BF
:10419000570C6B017C0181E890E061DC9B01AC0174
:1041A000C701B6010F944B09AB01BC0122E08FEDB2
:1041B00093E20E94DAA18DEC93E20E94859FE09148
:1041C0000A02F0910B0220E030E040E751E4638501
:1041D0007485858596850F94E30B18160CF46BC0D7
:1041E00020E030E0A9018DE790E029833A834B83FA
:1041F0005C830F9429124B015C0129813A814B8128
:104200005C81820E931EA41EB51EC501B40120E878
:1042100031E541E050E00F94830D60E87EEA8EEFD7
:104220009FEF0F941E0D6B017C01C80CD91CEA1C7A
:10423000FB1CBA01A90180ED93E20E94A9A0C7016D
:10424000B60120E13EE040E050E00F94830D4901CB
:104250005A01BA01A90186EC93E20E94A9A0A0EF3D
:10426000B1EFA50194010F94CC0D6C0D7D1D8E1D39
:104270009F1D2CE330E040E050E00F94830DBA0125
:10428000A9018EEB93E20E94A9A089EB93E20F9023
:104290000F900F900F90DF91CF91FF90EF90DF90F4
:1042A000CF90BF90AF909F908F907F906F905F90D6
:1042B0004F900C949E9F0F94E603C090E306D0901D
:1042C000E406E090E506F090E6066C197D098E099B
:1042D0009F0928EE33E040E050E00F94610D83CF5A
:1042E000811102C08EE207C0813011F48DE203C05B
:1042F000823019F48CE20D94D8020895EAE0F1E0DE
:1043000080818860808380818061808380818062F9
:1043100080836CE370E08EE20F94D8026CE370E06F
:104320008DE20F94D80262E870E08CE20F94D8021C
:10433000E1E2F1E08081887F81608083089567FDFC
:1043400043C08230E9F028F4882341F0813061F0E5
:104350003BC0833009F1843059F136C0662311F037
:10436000A19A69C0A19867C080910801662311F0E5
:10437000806801C08F778093080147FF3AC05FC013
:1043800080910801662311F0806401C08F7B8093C7
:10439000080147FF34C055C080910801662311F021
:1043A000886001C0877F8093080147FF32C046C004
:1043B00080910501662311F0806401C08F7B80939A
:1043C000050147FF2EC03CC047FD3BC08230B9F01D
:1043D00028F4882341F0813061F008958330C9F0DA
:1043E0008430F9F00895442311F0A09A0895A0981C
:1043F0000895442311F0A29A0895A29808958091F7
:104400000801442311F0806201C08F7D8093080170
:10441000089580910801442311F08061F7CF8F7EC9
:10442000F5CF80910501442311F0806401C08F7B9A
:1044300080930501089547FFD6CF08950895089504
:1044400008950895643079F028F4613041F06230C5
:1044500041F00895683051F0603141F0089540E036
:1044600003C040E004C041E060E002C041E061E020
:1044700066CFCF93DF938AE993E20E949E9F62B357
:104480006695617070E08FE494E20E9477A062B359
:10449000617070E087EB93E20E9483A0C6E0D1E0F8
:1044A0008881992787FD9095692F661F6627661F6B
:1044B00070E082EB93E20E9477A062B362FB662712
:1044C00060F970E087EB93E20E9483A0688166FB4D
:1044D000662760F970E08FEA93E20E9477A0688116
:1044E00065FB662760F970E087EB93E20E9483A08A
:1044F000688163FB662760F970E08BEA93E20E94B3
:1045000077A068816295617070E087EB93E20E940A
:1045100083A0C3E0D1E0688166FB662760F970E0A4
:1045200087EA93E20E9477A0688166FB662760F9BC
:1045300070E087EB93E2DF91CF910C9483A0FF9220
:104540000F931F93CF93DF9300D01F921F92CDB78D
:10455000DEB785E0E7E4F3E0DE01119601900D920D
:104560008A95E1F7989A9A9A8091070180628093E0
:104570000701809107018061809307018091040108
:104580008064809304018E010F5F1F4FF12CF801AE
:1045900061918F018F2D56DFF394F5E0FF12F7CF75
:1045A0000F900F900F900F900F90DF91CF911F9170
:1045B0000F91FF9008950C94D9DA0E94C4DA2091EB
:1045C0000802309109028217930724F4909309029C
:1045D0008093080208956091080270910902809109
:1045E0000602909107026817790744F47093070256
:1045F0006093060282E594E20C9483A00895CF9321
:10460000C82F69E170E085E89DE10F94B6006C2F3A
:1046100085E89DE10F94570060E085E89DE10F94E7
:10462000B700882329F082E59DE0CF910C949E9FEE
:10463000CF910895CF93DF93D82FC62F69E170E013
:1046400085E89DE10F94B6006D2F85E89DE10F94FC
:1046500057006C2F85E89DE10F94570085E89DE198
:104660000F94C900882331F082E39DE0DF91CF9160
:104670000C949E9FDF91CF910895C1DF41E050E0FF
:1046800069E170E085E89DE10F94AA0085E89DE16D
:104690000F940000892B31F085E89DE10F9408000C
:1046A00081E0089583E19DE00E949E9F80E008954F
:1046B0008EEE9CE00E949E9F85E89DE10F94950000
:1046C0008FE0DBDF81E3D9DF80E2D7DF6CE980E2D6
:1046D000B1DF80E2D2DF82E2D0DF60E482E2AADFF3
:1046E00082E2CBDF85E2C9DF60E085E2A3DF85E21D
:1046F000C4DF83E2C2DF60E383E29CDF83E2BDDFED
:1047000084E2BBDF6AE484E295DF84E2B6DF80E323
:10471000B4DF60E280E38EDF80E3AFDF81E3ADDF13
:1047200082E3ABDF64E182E385DF82E3A6DF83E33C
:10473000A4DF60E083E37EDF83E39FDF84E39DDF2C
:1047400060E084E377DF84E398DF86E396DF62E36B
:1047500086E370DF86E391DF87E38FDF60E087E346
:1047600069DF87E38ADF88E388DF60E188E362DF6F
:1047700088E383DF89E381DF8AE37FDF62E38AE323
:1047800059DF8AE37ACFCF9381E377DFC82F85E3C0
:1047900074DF811101C0C0E089E36FDF811101C0C6
:1047A000C0E08DE26ADF811101C0C0E08C2FCF91A3
:1047B00008956DE08FE29BE00E9478D96AE08FE275
:1047C0009BE00C9478D9CF93C82FE0918603F091A9
:1047D000870342A953A964A975A922E08CE394E256
:1047E0000E94DAA1E0918603F091870346A957A9B8
:1047F00060AD71AD20E083E294E20E94DAA10E94F4
:104800009951AB01BC0122E088E394E20E94DAA155
:104810004091190250911A0260911B0270911C0282
:1048200020E083E294E20E94DAA1CC2391F061E0DF
:1048300070E08AE294E20E9477A06CEF7FE08091C2
:10484000110290911202681B790B88E294E20E9497
:1048500077A0E0910E02F0E0E958F24E608170E03E
:104860008FE294E20E9477A0E091DE02EF3F29F40C
:10487000E0918603F0918703E081F0E0E958F24E81
:10488000608170E084E394E20E9477A0CF9191CFA1
:104890002F923F924F925F926F927F928F929F9250
:1048A000AF92BF92CF92DF92EF92FF920F931F933E
:1048B000CF93DF93CDB7DEB729970FB6F894DEBF5D
:1048C0000FBECDBF5C01DC0116968D919C911797B0
:1048D0008C38910509F48AC608F0E7C08235910545
:1048E00009F42FC408F08AC08A31910509F4D1C2B5
:1048F00008F03FC08531910509F449C278F482314E
:10490000910509F423C28431910509F424C2419729
:1049100011F00C944B3517981698D0C58731910536
:1049200009F46DC208F44FC28831910509F495C2AB
:10493000499711F00C944B3560E088E199E0299695
:104940000FB6F894DEBF0FBECDBFDF91CF911F91A0
:104950000F91FF90EF90DF90CF90BF90AF909F901E
:104960008F907F906F905F904F903F902F900C941E
:10497000579B8E31910509F4E9C218F58C319105E8
:1049800009F4BCC210F00C94843588E199E02996B2
:104990000FB6F894DEBF0FBECDBFDF91CF911F9150
:1049A0000F91FF90EF90DF90CF90BF90AF909F90CE
:1049B0008F907F906F905F904F903F902F900C94CE
:1049C0009E9E8A32910509F41BC328F4809709F44E
:1049D000EAC20C944B358035910509F49DC38135AD
:1049E000910511F00C944B3531D99B9A8091BD07FC
:1049F0008F7B8093BD07A39A0C9484358B369105E9
:104A000011F40C94792E38F58C35910509F4A4C471
:104A100060F48435910509F49DC308F496C3853587
:104A2000910509F475C40C944B358836910509F449
:104A300048C530F48336910509F4F2C40C944B3523
:104A40008936910509F425C68A36910511F40C942E
:104A5000682E0C944B358337910511F40C94CA2EB3
:104A600080F48F36910511F40C949A2E82379105BB
:104A700011F40C94E82E8D36910511F00C944B3501
:104A80002AC68537910511F40C94EB2E10F40C9482
:104A9000F22D8737910511F40C94162F8837910564
:104AA00011F40C945D2F0C944B358530B1E09B07CD
:104AB00011F40C946B3208F0B0C08F3C910511F4E6
:104AC0000C94053108F041C08A3C910511F40C9416
:104AD000343070F4883C910511F40C94832F10F05D
:104AE0000C94D62F8E3B910509F4CBC70C944B3513
:104AF0008C3C910511F40C948B3010F40C947930AB
:104B00008D3C910511F40C94EB308E3C910511F025
:104B10000C944B35C50129960FB6F894DEBF0FBE35
:104B2000CDBFDF91CF911F910F91FF90EF90DF905C
:104B3000CF90BF90AF909F908F907F906F905F903D
:104B40004F903F902F900C94E1D58F3D910511F43B
:104B50000C94C03188F48C3D910511F40C946D31A6
:104B60008D3D910511F40C949531813D910511F025
:104B70000C944B350C944D31893E910511F40C94F5
:104B8000D53140F5883E910511F00C944B3560917C
:104B90007F1D7091801D83E593E20E9477A0409174
:104BA0007B1D50917C1D60917D1D70917E1D22E0CA
:104BB0008AE493E20E949DA11092801D10927F1DB5
:104BC00010927B1D10927C1D10927D1D10927E1DF7
:104BD0000C9484358B3F910511F40C940E32843083
:104BE000914011F00C944B3529960FB6F894DEBF26
:104BF0000FBECDBFDF91CF911F910F91FF90EF902E
:104C0000DF90CF90BF90AF909F908F907F906F90EC
:104C10005F904F903F902F904BCD8E3521E09207C3
:104C200011F40C94C333C0F58E3241E0940711F4B3
:104C30000C940E3398F48931A1E09A0711F40C9486
:104C4000C3328C32B1E09B0711F40C94D33286301E
:104C5000914011F00C944B350C948D328034F1E07E
:104C60009F0711F40C94813338F48F32914011F482
:104C70000C944D330C944B35813441E0940711F47E
:104C80000C9485338234914011F00C944B3580E0C4
:104C90000E94178C0C949A338239A1E09A0711F480
:104CA0000C94AE3498F58836E1E09E0711F40C942C
:104CB0007A3438F48336914011F40C9434340C94E3
:104CC0004B35803931E0930711F40C9494348139D9
:104CD000914011F00C944B3529960FB6F894DEBF35
:104CE0000FBECDBFDF91CF911F910F91FF90EF903D
:104CF000DF90CF90BF90AF909F908F907F906F90FC
:104D00005F904F903F902F900C948F86853F51E09D
:104D1000950711F40C94DE3460F4843F914011F057
:104D20000C944B3580E00E9457CF8CEB9EE10C94A5
:104D3000E934863FE1E09E0711F40C9403358C388A
:104D4000934011F40C941D350C944B350E944D1D6D
:104D50000E944F1D8CC288E199E029960FB6F89405
:104D6000DEBF0FBECDBFDF91CF911F910F91FF909E
:104D7000EF90DF90CF90BF90AF909F908F907F90FB
:104D80006F905F904F903F902F900C94E79D88E13B
:104D900099E029960FB6F894DEBF0FBECDBFDF9124
:104DA000CF911F910F91FF90EF90DF90CF90BF9028
:104DB000AF909F908F907F906F905F904F903F90BB
:104DC0002F900C94DB9A88E199E029960FB6F8941D
:104DD000DEBF0FBECDBFDF91CF911F910F91FF902E
:104DE000EF90DF90CF90BF90AF909F908F907F908B
:104DF0006F905F904F903F902F900C94E09AD50168
:104E00008D919C9197FD02C00C94843560E088E1FF
:104E100099E00E942A67F501EE5AFF4F6081718187
:104E200040E088E199E029960FB6F894DEBF0FBE06
:104E3000CDBFDF91CF911F910F91FF90EF90DF9049
:104E4000CF90BF90AF909F908F907F906F905F902A
:104E50004F903F902F900C94189E88E199E02996EE
:104E60000FB6F894DEBF0FBECDBFDF91CF911F917B
:104E70000F91FF90EF90DF90CF90BF90AF909F90F9
:104E80008F907F906F905F904F903F902F900C94F9
:104E9000469BF5018081918192FD02C00C9484357E
:104EA000468D578D60A171A180918209882311F4EC
:104EB0000C9484354093790950937A0960937B0967
:104EC00070937C0988E599E029960FB6F894DEBFC7
:104ED0000FBECDBFDF91CF911F910F91FF90EF904B
:104EE000DF90CF90BF90AF909F908F907F906F900A
:104EF0005F904F903F902F900C947065D5018D91ED
:104F00009C9197FD02C00C948435F501EE5AFF4F39
:104F10006081718188E199E029960FB6F894DEBF2F
:104F20000FBECDBFDF91CF911F910F91FF90EF90FA
:104F3000DF90CF90BF90AF909F908F907F906F90B9
:104F40005F904F903F902F900C94BF9EF501808111
:104F5000918197FD02C00C94843560E088E199E06E
:104F60000E942A67F501EE5AFF4F6081718188E146
:104F700099E029960FB6F894DEBF0FBECDBFDF9142
:104F8000CF911F910F91FF90EF90DF90CF90BF9046
:104F9000AF909F908F907F906F905F904F903F90D9
:104FA0002F900C94219FD5018D919C9197FD02C06B
:104FB0000C94843560E088E199E00E942A67F5014D
:104FC000EE5AFF4F6081718188E199E029960FB612
:104FD000F894DEBF0FBECDBFDF91CF911F910F912F
:104FE000FF90EF90DF90CF90BF90AF909F908F9009
:104FF0007F906F905F904F903F902F900C944F9FB9
:10500000F5012081318133FD02C00C94843512A159
:10501000E12EF3A0E1E7FDE0449150E04E155F057D
:1050200009F45EC032964DE0E53EF407A9F7F7FCBF
:1050300057C032FF2CC0D5015E964D915D916D91A8
:105040007C9191974F3F51056105710509F0E0F49E
:1050500061E0812F0F94FA04F501668D812F0F9482
:105060003305D5015E966D917C915F97812F0F94EA
:10507000D802B7018DE893E20E9477A0F501668D12
:10508000778D88E893E212C08FE095E02BC062E054
:10509000812F0F94FA04B70188E893E20E9477A069
:1050A000812F0F946805BC0183E893E229960FB61F
:1050B000F894DEBF0FBECDBFDF91CF911F910F914E
:1050C000FF90EF90DF90CF90BF90AF909F908F9028
:1050D0007F906F905F904F903F902F900C9483A0A3
:1050E00089ED94E029960FB6F894DEBF0FBECDBFD0
:1050F000DF91CF911F910F91FF90EF90DF90CF90B4
:10510000BF90AF909F908F907F906F905F904F90E7
:105110003F902F900C94BF9F0E94261E0F94E60391
:105120006093811D7093821D8093831D9093841DD5
:105130009B9A8091BD0780648093BD07A3980C94CF
:105140008435109203080C94843581E08093030821
:105150000C948435D5018D919C91119792FF14C0C8
:105160005E962D913D914D915C919197A8EEB3E0A3
:105170000F94C00D60933E0370933F0380934003F0
:10518000909341030C94843593FFA5C0F50182A14F
:1051900093A1A4A1B5A182309105A105B10509F49F
:1051A00066C02CF50097A105B10509F446C001972A
:1051B000A105B10511F00C94843529960FB6F89429
:1051C000DEBF0FBECDBFDF91CF911F910F91FF903A
:1051D000EF90DF90CF90BF90AF909F908F907F9097
:1051E0006F905F904F903F902F900C944F1D8330A5
:1051F0009105A105B10509F454C00497A105B105B5
:1052000011F00C94843529960FB6F894DEBF0FBECA
:10521000CDBFDF91CF911F910F91FF90EF90DF9065
:10522000CF90BF90AF909F908F907F906F905F9046
:105230004F903F902F900C94B05129960FB6F89450
:10524000DEBF0FBECDBFDF91CF911F910F91FF90B9
:10525000EF90DF90CF90BF90AF909F908F907F9016
:105260006F905F904F903F902F900C944D1D29961A
:105270000FB6F894DEBF0FBECDBFDF91CF911F9167
:105280000F91FF90EF90DF90CF90BF90AF909F90E5
:105290008F907F906F905F904F903F902F900C94E5
:1052A000511D29960FB6F894DEBF0FBECDBFDF911A
:1052B000CF911F910F91FF90EF90DF90CF90BF9013
:1052C000AF909F908F907F906F905F904F903F90A6
:1052D0002F900C94A2510E94261E81E029960FB6B1
:1052E000F894DEBF0FBECDBFDF91CF911F910F911C
:1052F000FF90EF90DF90CF90BF90AF909F908F90F6
:105300007F906F905F904F903F902F900C947474AB
:10531000D5018D919C91119792FF14C05E962D91AD
:105320003D914D915C919197A8EEB3E00F94C00D23
:105330006093420370934303809344039093450327
:105340000C9484351092420310924303109244034C
:10535000109245030C948435F501808183FF0CC0C5
:1053600082859385A485B585809327039093280330
:10537000A0932903B0932A03D5018C9184FF0EC01A
:105380001E968D919D910D90BC91A02D80932B0325
:1053900090932C03A0932D03B0932E03F5018081ED
:1053A00085FF0CC082899389A489B58980932F03D6
:1053B00090933003A0933103B09332030E94E374BF
:1053C000D5018C9186FD02C00C9484352091860312
:1053D0003091870356968D919D910D90BC91A02D93
:1053E000F90181879287A387B487808129960FB6B8
:1053F000F894DEBF0FBECDBFDF91CF911F910F910B
:10540000FF90EF90DF90CF90BF90AF909F908F90E4
:105410007F906F905F904F903F902F900C94DF4F54
:10542000D501ED91FC911197F2FF0DC05E962D9183
:105430003D914D915C919197A8EEB3E00F94C00D12
:105440006B017C0106C040E1C42E47E2D42EE12C62
:10545000F12CE3FD0E944D1DF501808184FD0E9429
:105460004F1DD5018C9185FD0E94511D0F94E603BF
:105470002B013C014C0C5D1C6E1C7F1C0F94E60341
:10548000A3019201261B370B480B590BDA01C90106
:10549000803A9648A140B10518F40E94D979EECF20
:1054A000D5018C9183FD1798F501808184FD1698B4
:1054B000D5018C9185FD02C00C94843515980C940F
:1054C00084350E94C65981110C9484350F94E603EB
:1054D0006093811D7093821D8093831D9093841D22
:1054E0000E94471D81110C948435F50180819181C2
:1054F00093FF02C00C946E3592FF0AC0868D978D83
:10550000A0A1B1A1892B8A2B8B2B11F40C946E35A1
:10551000D5018D919C91119792FD02C00C94843518
:105520009C012227317091FF23C0232B89F011E0C9
:1055300020E030E0A9015A966D917D918D919C916A
:105540005D970F94E30B18160CF010E0212F01C0AB
:1055500020E085010C5A1F4FF501668D778D80A1E3
:1055600091A129870F94820A2985D8014C9124C0E2
:10557000232B81F011E020E030E0A901F501628DDC
:10558000738D848D958D0F94E30B18160CF010E03D
:10559000212F01C020E00091860310918703D501DF
:1055A0005E966D917D918D919C91919729870F9435
:1055B000820A2985F801408129960FB6F894DEBF4A
:1055C0000FBECDBFDF91CF911F910F91FF90EF9054
:1055D000DF90CF90BF90AF909F908F907F906F9013
:1055E0005F904F903F902F900C9416550E94C65993
:1055F00081110C9484350F94E6036093811D7093A0
:10560000821D8093831D9093841D0E94471D8111EC
:105610000C948435D5018D919C91119792FD02C017
:105620000C94843590FF11C011E020E030E0A90116
:105630005A966D917D918D919C915D970F94E30B9E
:1056400018160CF010E0412F01C040E0F501668D06
:10565000778D80A191A149870F94820A4985299667
:105660000FB6F894DEBF0FBECDBFDF91CF911F9173
:105670000F91FF90EF90DF90CF90BF90AF909F90F1
:105680008F907F906F905F904F903F902F900C94F1
:10569000DF55D5018D919C9133E0969587953A958C
:1056A000E1F7817029960FB6F894DEBF0FBECDBF2B
:1056B000DF91CF911F910F91FF90EF90DF90CF90EE
:1056C000BF90AF909F908F907F906F905F904F9022
:1056D0003F902F9078C80E94C65981110C94843550
:1056E0000F94E6036093811D7093821D8093831D48
:1056F0009093841D0E94471D81110C94843540E0D5
:1057000068EC74E08CE69AE00E9494AB8CE69AE038
:105710000E94E8AE0E94261E2090860330908703E8
:10572000F5018081918191FF09C0EC5AFF4F2081E2
:10573000211104C02BE5222E22E0322E92FF1EC042
:1057400090FF0FC011E020E030E0A901D5015A968A
:105750006D917D918D919C915D970F94E30B18163F
:105760000CF010E0F501668D778D80A191A10F946A
:10577000820A212FD1014C910E941655F10126A9D0
:1057800037A940AD51AD62A973A984A995A90F9419
:105790004A092B013C0120E030E0A9010F94E30B02
:1057A000181664F420E030E040EA50E4C301B2018E
:1057B0000F94AF0987FF0EC00C94843520E030E0D1
:1057C00040EA50ECC301B2010F94E30B181614F435
:1057D0000C94843599249394D101D0962D913C91C9
:1057E000D1979E968D919C919F97821793070CF06D
:1057F000912C0F94E6036D837E838F83988710E04E
:10580000412C512C32010F94E60369837A838B83F8
:105810009C836093811D7093821D8093831D909360
:10582000841DDC01CB012D813E814F815885821B77
:10583000930BA40BB50B893E9340A105B10558F01D
:1058400080E00E94E32389819A81AB81BC818D83B2
:105850009E83AF83B88781E00E94041E80918603F7
:10586000909187032816390609F064C0D1019396F8
:10587000ED90FC9094971E141F040CF05BC0111166
:1058800058C0992009F477C091966D917C919297B8
:10589000882777FD8095982F0F94820A9B01AC0191
:1058A000F10162A973A984A995A90F94E30B1816B5
:1058B00014F00C947B35662777276E197F098827AB
:1058C00077FD8095982F0F94820A209133033091B1
:1058D000340340913503509136030F94570C0F94C5
:1058E0004F0A1F921F92D10152962C9152972F93DB
:1058F00051962C9151972F9350962C9150972F930E
:105900001F962C912F935B016C01E12CF12C8701E8
:1059100020E030E0A90160E070E0CB010E9407F8D0
:105920000F900F900F900F900F900F9011E00C942C
:105930007B3511E0411451046104710409F050C039
:105940009920F1F020E030E040E85FE3F10166A942
:1059500077A980AD91AD0F944A099B01AC01D101AB
:10596000D2966D917D918D919C91D5970F94E30B7B
:1059700087FF1FC045CF411451046104710481F5B4
:1059800020E030E040E85FE3F10166A977A980AD4F
:1059900091AD0F944B099B01AC01D101D2966D9151
:1059A0007D918D919C91D5970F94AF0918160CF4A9
:1059B00027CFF101A78DB0A128EE33E00F94BA0DE7
:1059C0002B013C0129813A814B815C81420E531E9F
:1059D000641E751E411451046104710409F413CF4F
:1059E000D301C20129813A814B815C81821B930BD7
:1059F000A40BB50B81159449A543B74708F403CF11
:105A0000112309F4E2C08091860390918703281640
:105A1000390609F0DAC0D10193966D917C91949783
:105A2000882777FD8095982F0F94820A2091330361
:105A30003091340340913503509136030F94570C45
:105A40000F944F0A1F921F92F10122892F932189EF
:105A50002F9320892F9327852F935B016C01E12CD5
:105A6000F12C870120E030E0A90160E070E0CB017B
:105A70000E9407F80F900F900F900F900F900F90CB
:105A8000A4C00E94471D81110C94843540E06CEB4A
:105A900074E08CE69AE00E9494AB8CE69AE00E9457
:105AA000E8AE0E94261ED5018D919C91119792FF20
:105AB0001FC090FF11C011E020E030E0A9015A960C
:105AC0006D917D918D919C915D970F94E30B1816CC
:105AD0000CF010E0412F01C040E0F501668D778D9C
:105AE00080A191A149870F94820A49850E94DF55C0
:105AF0002091190230911A0240911B0250911C0210
:105B0000609115027091160280911702909118020F
:105B10000F944A092B013C0120E030E0A9010F94C9
:105B2000E30B18165CF420E030E040EA50E4C301D7
:105B3000B2010F94AF0987FF0CC0E6C720E030E048
:105B400040EA50ECC301B2010F94E30B18160CF4B9
:105B5000DBC70F94E6032B013C0120E030E040E07E
:105B60005FE3609115027091160280911702909187
:105B700018020F944B092091190230911A0240919A
:105B80001B0250911C020F94AF0987FF1EC00F9497
:105B9000E6036419750986099709693E7340810512
:105BA000910578F080E00E94E3230F94E6032B0137
:105BB0003C016093811D7093821D8093831D90939F
:105BC000841D81E00E94041EC8CF1092D50A0F9454
:105BD000E6036093811D7093821D8093831D9093D3
:105BE000841D92C70E94471D81118EC70F94E60342
:105BF0002B013C010F94E603641975098609970986
:105C0000693E73408105910538F080E00E94E323EE
:105C10000F94E6032B013C0181E00E94041E0091D9
:105C20000A0210910B02D8011B968D909D90AD90A9
:105C3000BC901E9720E030E040EF51E4C501B40174
:105C40000F94E30B1816BCF4F801278130854185C9
:105C50005285C501B4010F944A099F7701E020E005
:105C600030E040E85FE30F94E30B18160CF000E01F
:105C700011E0102701C011E0E0900C02F0900D023D
:105C8000D7011B968D909D90AD90BC901E9720E003
:105C900030E040EF51E4C501B4010F94E30B181656
:105CA0009CF4F7012781308541855285C501B401F7
:105CB0000F944A099F7720E030E040E85FE30F94BB
:105CC000E30B18160CF496CF112309F493CF1CC7DD
:105CD000D5018D919C91119793FB662760F992FFF6
:105CE00005C05E968D919C915F970AC08FEF90E002
:105CF00007C0F501618163FB662760F980E090E0F1
:105D000029960FB6F894DEBF0FBECDBFDF91CF91BD
:105D10001F910F91FF90EF90DF90CF90BF90AF90C9
:105D20009F908F907F906F905F904F903F902F90BB
:105D30000C947F20D5018D919C91119792FF04C006
:105D40005E962C912093EA0293FF12C0F50182A186
:105D500093A1A4A1B5A12091EA02181619061A066A
:105D60001B0614F4822B02C0815082238093EA0226
:105D70000E94471D882309F4C7C620E040E060E088
:105D800070E0CB010E94165520E040E060E070E03A
:105D9000CB0112CC88E695E20E949E9F29960FB611
:105DA000F894DEBF0FBECDBFDF91CF911F910F9151
:105DB000FF90EF90DF90CF90BF90AF909F908F902B
:105DC0007F906F905F904F903F902F900C94A92000
:105DD00086EB94E066C3D5018D919C9197FF94C6A4
:105DE000F501EE5AFF4F6081718140E08CE69AE048
:105DF0000E940DAC8CE69AE029960FB6F894DEBFAF
:105E00000FBECDBFDF91CF911F910F91FF90EF900B
:105E1000DF90CF90BF90AF909F908F907F906F90CA
:105E20005F904F903F902F900C94E8AE0E94261EFA
:105E300086E793E20E94859F379903C08DE793E23E
:105E400002C080E893E20E94859F8FE693E20E9461
:105E5000859F0E94531D882319F080E893E202C0B9
:105E60008DE793E20E94859F88E693E20E94859FDA
:105E70000E94581D882319F080E893E202C08DE744
:105E800093E20E94859F29960FB6F894DEBF0FBE5D
:105E9000CDBFDF91CF911F910F91FF90EF90DF90D9
:105EA000CF90BF90AF909F908F907F906F905F90BA
:105EB0004F903F902F900C94D923F50180819181D0
:105EC00088279C7081159C4009F01EC6F50162A1CF
:105ED000868D29960FB6F894DEBF0FBECDBFDF9139
:105EE000CF911F910F91FF90EF90DF90CF90BF90D7
:105EF000AF909F908F907F906F905F904F903F906A
:105F00002F900C94B0A2E0918603F091870320813A
:105F1000D5018D919C9191FF06C0F501EC5AFF4F80
:105F20008081882311F0822F01C080E0F5019281E9
:105F300092FF05C046A457A460A871A803C0412CD5
:105F4000512C320193FF07C0D501D2964D905D9040
:105F50006D907C90D597082F10E0B3E88B9FF001EF
:105F60001124E752FD4F4082518262827382821374
:105F700006C08091F5069091F6060E94072020E069
:105F800030E0A901C301B2010F94AF09B80181113A
:105F900003C08AE894E08AC883E694E00E9477A070
:105FA00022E0B301A2018EE594E05DC1F50180819C
:105FB00083FF0CC082859385A485B5858093FB0201
:105FC0009093FC02A093FD02B093FE02D5018C9148
:105FD00084FF0EC01E968D919D910D90BC91A02DB9
:105FE0008093FF0290930003A0930103B0930203F8
:105FF000F501808185FF0CC082899389A489B589C8
:106000008093030390930403A0930503B0930603C6
:10601000D5018C9186FF0EC056968D919D910D9065
:10602000BC91A02D8093070390930803A0930903CC
:10603000B0930A0329960FB6F894DEBF0FBECDBF0A
:10604000DF91CF911F910F91FF90EF90DF90CF9054
:10605000BF90AF909F908F907F906F905F904F9088
:106060003F902F900C94E374F501808183FF0CC066
:1060700082859385A485B5858093EB029093EC028D
:10608000A093ED02B093EE02D5018C9184FF0EC077
:106090001E968D919D910D90BC91A02D8093EF0245
:1060A0009093F002A093F102B093F202F501808187
:1060B00085FF0CC082899389A489B5898093F302F6
:1060C0009093F402A093F502B093F602D5018C915F
:1060D00086FFB0CF56968D919D910D90BC91A02DCD
:1060E0008093F7029093F802A093F902B093FA021A
:1060F000A1CFF5018081918192FF06C5868D978D94
:10610000A0A1B1A1181619061A061B060CF481E00D
:106110008093E002F9C4E0918603F0918703BB9677
:10612000D5012D913C91119732FF11C05E968D9152
:106130009D910D90BC91A02DB7FDE6C4892B8A2BB3
:106140008B2B19F0EEE0F2E002C0E6E8F2E023FF6C
:106150000BC0D5011A964D915D916D917C911D9763
:10616000428F538F648F758FD5018C9184FF0AC045
:106170001E964D915D916D917C915197468F578FF1
:1061800060A371A3D5018C9185FF0AC052964D91F1
:106190005D916D917C91559742A353A364A375A320
:1061A000CF0129960FB6F894DEBF0FBECDBFDF91A9
:1061B000CF911F910F91FF90EF90DF90CF90BF9004
:1061C000AF909F908F907F906F905F904F903F9097
:1061D0002F900C94114F29960FB6F894DEBF0FBE86
:1061E000CDBFDF91CF911F910F91FF90EF90DF9086
:1061F000CF90BF90AF909F908F907F906F905F9067
:106200004F903F902F900C948ED7F501208123FF63
:106210000CC082859385A485B5858093F106909303
:10622000F206A093F306B093F40626FF11C0209166
:10623000860330918703F50186899789A08DB18DFA
:10624000F901878B908FA18FB28F80810E94DF4FE1
:106250004091F1065091F2066091F3067091F406B8
:1062600022E082E693E229960FB6F894DEBF0FBED5
:10627000CDBFDF91CF911F910F91FF90EF90DF90F5
:10628000CF90BF90AF909F908F907F906F905F90D6
:106290004F903F902F900C949DA1D5018D919C9192
:1062A000119792FF31C461E05E968D919D910D90A2
:1062B000BC91A02D2091BC07892B8A2B8B2B21F41C
:1062C00060E0822F8D7F02C0822F82608093BC07A6
:1062D00070E085EC93E00C945628F5018081918163
:1062E00092FF05C0868D978DA0A1B1A104C084E660
:1062F00090E0A0E0B0E029960FB6F894DEBF0FBEA4
:10630000CDBFDF91CF911F910F91FF90EF90DF9064
:10631000CF90BF90AF909F908F907F906F905F9045
:106320004F903F902F900C94801FD5018D919C91A0
:10633000119792FF07C05E968D919D910D90BC9133
:10634000A02D04C084E690E0A0E0B0E029960FB64E
:10635000F894DEBF0FBECDBFDF91CF911F910F919B
:10636000FF90EF90DF90CF90BF90AF909F908F9075
:106370007F906F905F904F903F902F900C940720EC
:10638000F5018081918192FFBFC34FB7F89480914E
:10639000480890914908268D378D820F931F90935E
:1063A0004908809348084FBFAFC3F5018081209111
:1063B00086033091870384FF09C086859785A0896D
:1063C000B189F90185A396A3A7A3B0A7D901959692
:1063D0004D915D916D917C91989722E081E393E2DC
:1063E0000E94DAA10E94D92329960FB6F894DEBF45
:1063F0000FBECDBFDF91CF911F910F91FF90EF9016
:10640000DF90CF90BF90AF909F908F907F906F90D4
:106410005F904F903F902F900C94C9742091EF079C
:106420003091F0074091F1075091F2076091010718
:106430007091020780910307909104070F944A0915
:1064400060930107709302078093030790930407FA
:106450001092FB071092FC071092FD071092FE07A6
:106460000E94E37467E078E083EF97E00E94F3EC2A
:1064700080E00E94EC8040910107509102076091FA
:1064800003077091040722E086EC9FE10E949DA122
:1064900080E00E9457CF8BE393E20E949E9F88E5A5
:1064A00094E029960FB6F894DEBF0FBECDBFDF9102
:1064B000CF911F910F91FF90EF90DF90CF90BF9001
:1064C000AF909F908F907F906F905F904F903F9094
:1064D0002F900C94341E80E10F946805BC018EE46B
:1064E00094E00E9483A029960FB6F894DEBF0FBEF9
:1064F000CDBFDF91CF911F910F91FF90EF90DF9073
:10650000CF90BF90AF909F908F907F906F905F9053
:106510004F903F902F900C94C32382E30E943D2321
:10652000F5018081918192FFEFC2468D578D60A168
:1065300071A188E394E00E94C1A0D5015E966C91A0
:1065400082E30E941A23F501668D8AE30E941A23D2
:1065500082E329960FB6F894DEBF0FBECDBFDF9160
:10656000CF911F910F91FF90EF90DF90CF90BF9050
:10657000AF909F908F907F906F905F904F903F90E3
:106580002F900C943D238DEF93E00E94B59F80E007
:106590000E94747468EC70E080E090E00F94150441
:1065A0008FB7F894FFCFD5018D919C91119792FFF1
:1065B00005C05E966D917C915F9702C061E070E0CE
:1065C00093FF04C0F50102A113A102C008EE13E07D
:1065D00020E030E0A90184E50F94B805B80180E01F
:1065E00090E00F94150484E529960FB6F894DEBF69
:1065F0000FBECDBFDF91CF911F910F91FF90EF9014
:10660000DF90CF90BF90AF909F908F907F906F90D2
:106610005F904F903F902F900D94C908D5018D91B8
:106620009C91119792FF0EC021E05E968D919D91F5
:106630000D90BC91A02D892B8A2B8B2B09F420E087
:10664000822F01C081E09091BD07882311F09068EE
:1066500001C09F779093BD07882319F08EEA93E0DD
:1066600002C084E993E029960FB6F894DEBF0FBE0E
:10667000CDBFDF91CF911F910F91FF90EF90DF90F1
:10668000CF90BF90AF909F908F907F906F905F90D2
:106690004F903F902F900C949E9FF50100811181A7
:1066A00012FF03C0668D778D02C066E970E013FFAC
:1066B0000DC0D5019296ED90FC909397B2E0EB1649
:1066C000F10434F082E0E82EF12C02C0E12CF12C30
:1066D000A3E016950795AA95E1F70170882777FD45
:1066E0008095982F0F94820AAB01BC01F701EE0F41
:1066F000FF1FE65FFD4F2E2D808191810E94605625
:1067000003C281E00E94C38715C080E00E94C38756
:10671000D5018D919C91119792FFF6C15E968D9156
:106720009D910D90BC91A02D0097A105B10509F098
:10673000D9C1EAC1F5018081918192FFE5C1868DC1
:10674000978DA0A1B1A1892B8A2B8B2B09F4DCC1D9
:1067500080E029960FB6F894DEBF0FBECDBFDF9163
:10676000CF911F910F91FF90EF90DF90CF90BF904E
:10677000AF909F908F907F906F905F904F903F90E1
:106780002F900C9457CF8BEE93E00E949E9FD501E3
:106790008D919C9192FD0FC0F501808183FF16C001
:1067A000F50162857385848595850F94540A80E090
:1067B0000E9422220BC010E0D5015E966C91812FC1
:1067C0000E9422221F5F1530B9F7E6CFD5018C91C8
:1067D00084FF0BC01E966D917D918D919C91519778
:1067E0000F94540A81E00E942222F501808185FFE6
:1067F00009C062897389848995890F94540A82E05B
:106800000E942222D5018C9186FF0BC056966D9175
:106810007D918D919C9159970F94540A83E00E9429
:106820002222F5018081918193FF04C062A184E05E
:106830000E94222229960FB6F894DEBF0FBECDBF6C
:10684000DF91CF911F910F91FF90EF90DF90CF904C
:10685000BF90AF909F908F907F906F905F904F9080
:106860003F902F900C943922D5018D919C911197D6
:1068700092FF26C081E05E964D915D916D917C9175
:106880009197452B462B472B09F480E029960FB6AC
:10689000F894DEBF0FBECDBFDF91CF911F910F9156
:1068A000FF90EF90DF90CF90BF90AF909F908F9030
:1068B0007F906F905F904F903F902F900C944090FE
:1068C00029960FB6F894DEBF0FBECDBFDF91CF91F2
:1068D0001F910F91FF90EF90DF90CF90BF90AF90FE
:1068E0009F908F907F906F905F904F903F902F90F0
:1068F0000C94419029960FB6F894DEBF0FBECDBF21
:10690000DF91CF911F910F91FF90EF90DF90CF908B
:10691000BF90AF909F908F907F906F905F904F90BF
:106920003F902F900C944F9029960FB6F894DEBFAD
:106930000FBECDBFDF91CF911F910F91FF90EF90D0
:10694000DF90CF90BF90AF909F908F907F906F908F
:106950005F904F903F902F900C94261EF501808100
:10696000918190FF05C0E28CF38C048D158D08C0D9
:10697000E090F906F090FA060091FB061091FC06F3
:106980009C0146E0369527954A95E1F72170AC01C8
:1069900065E0569547956A95E1F74170BC01E4E0E2
:1069A00076956795EA95E1F76170F3E0969587959E
:1069B000FA95E1F781700E94F086A6C00E94B4D1DA
:1069C000E0918603F091870380810E94DF4F8AE97E
:1069D0009EE129960FB6F894DEBF0FBECDBFDF91C2
:1069E000CF911F910F91FF90EF90DF90CF90BF90CC
:1069F000AF909F908F907F906F905F904F903F905F
:106A00002F900C94B59F29960FB6F894DEBF0FBE59
:106A1000CDBFDF91CF911F910F91FF90EF90DF904D
:106A2000CF90BF90AF909F908F907F906F905F902E
:106A30004F903F902F900C945CCD82ED93E00E949C
:106A40009E9FD5018D919C9188279C7081159C40BB
:106A500009F05AC0D5015E966D917C915F97929630
:106A60008C9129960FB6F894DEBF0FBECDBFDF9193
:106A7000CF911F910F91FF90EF90DF90CF90BF903B
:106A8000AF909F908F907F906F905F904F903F90CE
:106A90002F900C9470218091EA0282FF35C08CE522
:106AA00094E20E94859FC50129960FB6F894DEBF37
:106AB0000FBECDBFDF91CF911F910F91FF90EF904F
:106AC000DF90CF90BF90AF909F908F907F906F900E
:106AD0005F904F903F902F900C946F970E94261ECE
:106AE0000C94882A0397A105B10509F031CE80E006
:106AF0000E94178C2DCE411451046104710411F4CD
:106B00000C94A22C0C94F02C29960FB6F894DEBFAE
:106B10000FBECDBFDF91CF911F910F91FF90EF90EE
:106B2000DF90CF90BF90AF909F908F907F906F90AD
:106B30005F904F903F902F9008952F923F924F92E9
:106B40005F926F927F928F929F92AF92BF92CF92FD
:106B5000DF92EF92FF920F931F93CF93DF93CDB706
:106B6000DEB7EC970FB6F894DEBF0FBECDBF1C01A9
:106B7000DC0118968D919C9119978032910509F44A
:106B800069C358F58531910509F45EC198F48430E4
:106B9000910509F41BC128F4029708F4EBC00C948A
:106BA0007644449711F00C94764481E08093470832
:106BB0000C9481448D31910509F4AEC128F44C97B1
:106BC00009F446C10C9476448E31910509F41DC236
:106BD0004F9709F42CC30C9476448C35910511F42D
:106BE0000C94A04040F58534910509F492C7B8F49F
:106BF0008434910511F00C9476448091F9069091BB
:106C0000FA06A091FB06B091FC068D879E87AF87A0
:106C1000B88B44E1442E512C612C712CA5C58A35CA
:106C2000910511F40C9485408B35910511F40C9469
:106C300091400C9476448438910511F40C943743B8
:106C400008F05DC08436910511F40C9482418338BC
:106C5000910511F00C9476446091E7077091E80774
:106C60008091E9079091EA072091EB073091EC07BA
:106C70004091ED075091EE07E090EF07F090F0079C
:106C80000091F1071091F2074090F9065090FA0632
:106C90006090FB067090FC061092ED061092EE06D6
:106CA0001092EF061092F0061092E9061092EA0692
:106CB0001092EB061092EC06E0910E03EF93E09138
:106CC0000D03EF93E0910C03EF93E0910B03EF932F
:106CD000E0EFAE2EE3E2BE2EE4E7CE2EE9E4DE2EB8
:106CE0000E942F7E4092F9065092FA066092FB06AF
:106CF0007092FC0680E00E94EC800C943243853850
:106D0000910511F40C94C6438638910511F00C944A
:106D100076444091070850910808609109087091E5
:106D20000A0880EA95E00E94A9A040910B085091C2
:106D30000C0860910D0870910E0887EB93E20E9499
:106D4000A9A040910F08509110086091110870910E
:106D5000120887EB93E20E94C1A080E00E94EC80C1
:106D600082E995E00E94859F8CE895E00E94341EA0
:106D70000C948144F1018081918192FF11C0868D34
:106D8000978DA0A1B1A12091BD07892B8A2B8B2BB8
:106D900019F0822F806202C0822F8F7D8093BD0701
:106DA000C1010E946382882359F041E061E081E0E3
:106DB0000E94D7F2811104C082EC9CE00E94AB9F3C
:106DC00061E081E00E94D8EC0C9481440E94261E70
:106DD000D1018D919C91119793FF07C092968D9050
:106DE0009D90AD90BC90959703C0812C912C54013F
:106DF00092FF0BC0F101268D378D40A151A1A8EE65
:106E0000B3E00F94C00D4B015C010F94E6036B01DE
:106E10007C01C80CD91CEA1CFB1C0F94E603A701DB
:106E20009601261B370B480B590BDA01C901811556
:106E30009449A543B74710F00C9481440E9462988E
:106E400081E00E94041EE9CF109247080C9481440F
:106E5000D1018D919C91AC01487355274115510585
:106E600051F49C0166E0369527956A95E1F7B1E00B
:106E70002B27217001C020E086FF08C01092FF0779
:106E8000109200081092010810920208211117C0F8
:106E9000452BD1F0AC0125E0569547952A95E1F7B1
:106EA000BC0134E0769567953A95E1F753E0969505
:106EB00087955A95E1F761704170817003C061E078
:106EC00041E081E00E94DD8780E00E94EC803799FC
:106ED00002C00C94A4448FEA9CE00E94289687EAA2
:106EE0009CE00E94859F379B04C084EA9CE00E943E
:106EF000859F0E94531D882321F081EA9CE00E9417
:106F0000859F0E94581D882321F08EE99CE00E94F5
:106F1000859F8EE79CE075C00E94C323811111C03C
:106F20006AEF70E080E090E00F9415040E94C323A4
:106F3000811107C08EE59CE00E949E9F85E49CE045
:106F400072C180E39CE00E9428962091F90630915E
:106F5000FA064091FB065091FC06298F3A8F4B8F21
:106F60005C8F80E090E00E94A41D80E090E00E9491
:106F7000C41D80E090E00E94E41D80E00E9457CF95
:106F80000E94B4D184E190E0A0E0B0E0898B9A8BBC
:106F9000AB8BBC8B86E1482E512C612C712C1DA231
:106FA00029893A894B895C892D873E874F87588B81
:106FB00041E061E081E00E94DD87379902C00C94D6
:106FC000AF448DE19CE00E94289685E19CE00E9400
:106FD000859F379B04C082E19CE00E94859F0E94B0
:106FE000531D882321F08FE09CE00E94859F0E9422
:106FF000581D882321F08CE09CE00E94859F8CEE38
:107000009BE00E949E9F0C948144D1012D913C9164
:10701000119732FD02C00C94BA495E968D919D91F4
:107020000D90BC91A02D0297A105B10511F00C9413
:10703000BA490C94334A81E99BE00E949E9F89E7FC
:107040009BE00E94289686ED9FE10E94BF9FEDA1E4
:10705000E1110C94814481E00E94EC80298D3A8DED
:107060004B8D5C8D2093F9063093FA064093FB0616
:107070005093FC0687E39AE00E94341E8EE390E270
:107080000E942896212C312C80916D0790916E07DB
:10709000A0916F07B0917007898B9A8BAB8BBC8BDB
:1070A00080E00E9457CF0E94B4D181E00E94C38744
:1070B00041E061E081E00E94DD8780E00E94C387BB
:1070C0008FE390E20E9428960E945C1D9F938F930D
:1070D0007F936F93B0EFAB2EB3E2BB2EB4E7CB2E12
:1070E000B9E4DB2E8601750120E030E0A901CA0178
:1070F000B9010E949A8520E041E060E081E00E94B1
:107100006C886B017C0120E041E060E081E00E943E
:107110006C884B015C019B01AC01C701B6010F9467
:107120004A092B013C010F900F900F900F902DEC0E
:107130003CEC4CEC5DE30F94E30B181614F00C944C
:10714000D0474D855E856F85788983E09AE00E94FF
:10715000C1A02D853E854F855889283231054105CE
:10716000510514F00C94DC4782E30E943D238D8589
:107170009E85AF85B8890296A11DB11D8D879E871A
:10718000AF87B88BAC01BD0185EE99E00E94C1A02C
:107190006D8582E30E941A236D858AE30E941A237B
:1071A00082E30E943D23B4E02B1631040CF46CCF33
:1071B00081E00E94C38781E00E94EC8086ED98E028
:1071C0000E94341E8EE390E20E942896298D3A8D0B
:1071D0004B8D5C8D2093F9063093FA064093FB06A5
:1071E0005093FC0641E061E081E00E94DD8780E091
:1071F0000E9457CF41E06CE473E088E199E00E947F
:10720000189E882371F088E199E00E94769B6CE4D7
:1072100073E088E199E00E94219F88E199E00E9453
:10722000AA9A8CEB98E00E9428960C9481448CE4F6
:1072300090E20E94859F8091000181FD02C068E478
:1072400001C06CE48FE29BE00E9478D90E94D923B0
:107250000C9481448FE390E20E9428961092C70715
:107260001092C8071092C9071092CA071092C3075C
:107270001092C4071092C5071092C6071092BF075C
:107280001092C0071092C1071092C20780E00E94BE
:10729000C3872091F9063091FA064091FB06509180
:1072A000FC0629A33AA34BA35CA30E945C1D162FE6
:1072B000072FF82EE92E84E393E00E942F1D9B01F7
:1072C000AC0180E393E029AF3AAF4BAF5CAF0E94D3
:1072D0002F1DEF92FF920F931F9350EFA52E53E2B5
:1072E000B52E54E7C52E59E4D52E8601750129AD7A
:1072F0003AAD4BAD5CAD0E949A8520E041E060E084
:1073000081E00E946C882B013C010F900F900F9040
:107310000F9020E030E0A9010F94AF0987FF02C071
:107320000C9481440E945C1D162F072FF82EE92E25
:107330008CE393E00E942F1D9B01AC0188E393E056
:1073400029AF3AAF4BAF5CAF0E942F1DEF92FF9277
:107350000F931F938601750129AD3AAD4BAD5CAD1E
:107360000E949A8521E041E060E080E00E946C8804
:107370006D877E878F87988B0F900F900F900F905F
:1073800020E030E0A9010F94AF0987FF02C00C9400
:1073900081440E945C1D162F072FF82EE92E84E4ED
:1073A00093E00E942F1D9B01AC0180E493E029AF84
:1073B0003AAF4BAF5CAF0E942F1DEF92FF920F933D
:1073C0001F938601750129AD3AAD4BAD5CAD0E94AE
:1073D0009A8521E041E061E080E00E946C884B01E9
:1073E0005C010F900F900F900F9020E030E0A9010A
:1073F0000F94AF0987FF02C00C948144850174018A
:107400002D853E854F855889C301B2010E94128E99
:107410008091930790919407A0919507B09196075A
:107420008D879E87AF87B88B2091A7073091A807DB
:107430004091A9075091AA07298B3A8B4B8B5C8B03
:10744000C0909B07D0909C07E0909D07F0909E070E
:1074500080919F079091A007A091A107B091A207EA
:107460008D8B9E8BAF8BB88F2091F7073091F807EB
:107470004091F9075091FA072DA33EA34FA358A7B7
:1074800080913B0890913C08A0913D08B0913E0846
:1074900089A79AA7ABA7BCA72091A3073091A407FF
:1074A0004091A5075091A6072D8F3E8F4F8F58A36F
:1074B0008091970790919807A0919907B0919A07AA
:1074C000898F9A8FAB8FBC8F2091F3073091F4078F
:1074D0004091F5075091F6072DA73EA74FA758AB4F
:1074E0008091370890913808A0913908B0913A08F6
:1074F00089AB9AABABABBCAB1092FD061092FE060B
:107500001092FF0610920007D1018D919C91119766
:1075100092FFDCC05E968D919D910D90BC91A02D47
:10752000AC01BD0141505109610971094230510559
:107530006105710548F00397A105B10509F0C6C0C2
:1075400080E00E9457CFC2C029893A894B895C8963
:107550006D857E858F8598890F94570C2B013C0192
:107560002D893E894F89588DC701B6010F94570C5C
:107570009B01AC01C301B2010F944A092B013C01EC
:107580006DA17EA18FA198A50F94820A9B01AC01E9
:10759000C301B2010F94570C29A53AA54BA55CA5D0
:1075A0000F94570C2B013C012D8D3E8D4F8D58A112
:1075B000C701B6010F94570C6B017C0129893A89E8
:1075C0004B895C89698D7A8D8B8D9C8D0F94570CBE
:1075D0009B01AC01C701B6010F944A096B017C0104
:1075E0006DA57EA58FA598A90F94820A9B01AC0179
:1075F000C701B6010F94570C29A93AA94BA95CA958
:107600000F94570C9B01AC01C301B2010F944B09BD
:107610006B017C01F7FAF094F7F8F0942D893E891C
:107620004F89588D698D7A8D8B8D9C8D0F94570C59
:107630002B013C012D8D3E8D4F8D58A16D857E8592
:107640008F8598890F94570C9B01AC01C301B2013F
:107650000F944A099B01AC01C701B6010F94B6090A
:107660009B01AC01C501B4010F944B092091EF07B8
:107670003091F0074091F1075091F2070F944A09B9
:1076800020910107309102074091030750910407B0
:107690000F944B09AB01BC014093010750930207C3
:1076A000609303077093040722E086EC9FE10E9439
:1076B0009DA181E00E94C387F101868D978DA0A1D5
:1076C000B1A10297A105B10509F43ACF81E00E946A
:1076D000C3870E94E37481E00E94EC8084E698E016
:1076E0000E94341E41E061E081E00E94DD8729A113
:1076F0003AA14BA15CA12093F9063093FA0640937E
:10770000FB065093FC060C9481442DEC3CEC4CECB5
:107710005DEBC701B6010F94AF0987FF85C0B301C8
:10772000A20184E498E00E94C1A038E2431651040B
:1077300061047104CCF482E30E943D2342E0440ED4
:10774000511C611C711CB301A20186E298E00E94E9
:10775000C1A0642D82E30E941A23642D8AE30E9453
:107760001A2382E30E943D2320916D0730916E071A
:1077700040916F0750917007298F3A8F4B8F5C8F24
:1077800080E00E9457CF0E94B4D141E061E081E0E7
:107790000E94DD878FE390E20E94289680E00E949D
:1077A000C3870E945C1D9F938F937F936F9330EFED
:1077B000A32E33E2B32E34E7C32E39E4D32E860151
:1077C000750120E030E0A901CA01B9010E949A8543
:1077D00020E041E060E081E00E946C88698B7A8B58
:1077E0008B8B9C8B20E041E060E081E00E946C8804
:1077F0006D8B7E8B8F8B988F9B01AC0169897A8909
:107800008B899C890F944A096B017C010F900F9022
:107810000F900F902DEC3CEC4CEC5DE30F94E30BE0
:1078200018160CF072CF7BCF0E945C1D162F072F0D
:10783000F82EE92E84E493E00E942F1D9B01AC01F9
:1078400080E493E029AF3AAF4BAF5CAF0E942F1DAD
:10785000EF92FF920F931F9320EFA22E23E2B22EFE
:1078600024E7C22E29E4D22E8601750129AD3AAD56
:107870004BAD5CAD0E949A8521E041E061E080E083
:107880000E946C884B015C0121E041E061E080E0F6
:107890000E946C886B017C019B01AC01C501B401A5
:1078A0000F944A096D8F7E8F8F8F98A30F900F9042
:1078B0000F900F902DEC3CEC4CEC5DE30F94E30B40
:1078C000181664F02DEC3CEC4CEC5DEB6D8D7E8D70
:1078D0008F8D98A10F94AF0987FF13C0B301A20148
:1078E00086E098E00E94C1A082E30E943D2352E01E
:1078F000450E511C611C711CB301A20188EE97E07A
:1079000026CF29893A894B895C896D897E898F893F
:10791000988D0F944B0920E030E040E05FE30F9436
:10792000570C698B7A8B8B8B9C8B20E030E0A90104
:107930000F94AF0987FD18CFA5019401C701B601C7
:107940000F944B0920E030E040E05FE30F94570CC8
:107950009B01AC0169897A898B899C890F944A09BA
:1079600020E030E040EA52E40F94570C6B017C01B8
:1079700020E030E0A9010F94AF0987FF31C0F7FA8A
:10798000F094F7F8F09422E0B701A6018AE690E2BD
:107990000E949DA120916D0730916E0740916F0765
:1079A00050917007C701B6010F94B6099B01AC0155
:1079B0000F944B096B017C0122E0AB01BC018AE60C
:1079C00090E20E949DA1A701960160916D077091C0
:1079D0006E0780916F07909170070F944A0918C045
:1079E00080906D0790906E07A0906F07B090700721
:1079F000A5019401C701B6010F94B6099B01AC0122
:107A00000F944B099B01AC01C501B4010F944B09C4
:107A100060936D0770936E0780936F079093700764
:107A200022EC35EF41EB52E460916D0770916E07E7
:107A300080916F07909170070F94B6096B017C01DC
:107A40002DEC3CEC4CE85FE30F94E30B181654F07C
:107A500026E636E646E65FE3C701B6010F94AF09B6
:107A600087FF12C082EC95EFA1EBB2E480936D0723
:107A700090936E07A0936F07B093700722E0AC015C
:107A8000BD018DEC97E014C022E0498D5A8D6B8DBD
:107A90007C8D80EC97E00E949DA140916D075091F4
:107AA0006E0760916F077091700722E083EB97E09B
:107AB0000E949DA18D859E85AF85B8898093F9062A
:107AC0009093FA06A093FB06B093FC0681E00E9417
:107AD000C38781E00E94EC808EEA97E00E94341E0A
:107AE0008EE390E20E9428962D853E854F85588929
:107AF0002093F9063093FA064093FB065093FC0658
:107B000041E061E081E00E94DD8780E00E9457CF84
:107B1000F8C68091F9069091FA06A091FB06B09103
:107B2000FC068D8F9E8FAF8FB8A324E130E040E03C
:107B300050E02D873E874F87588BD1018D919C91C6
:107B4000119792FF0CC05E968D919D910D90BC9106
:107B5000A02D0297A105B10511F40C947F4B41E0D3
:107B600061E081E00E94DD878FE390E20E94289629
:107B700080E00E94C3870E945C1D162F072FF82EFD
:107B8000E92E84E393E00E942F1D9B01AC0180E36A
:107B900093E029AF3AAF4BAF5CAF0E942F1DEF923D
:107BA000FF920F931F9300EFA02E03E2B02E04E785
:107BB000C02E09E4D02E8601750129AD3AAD4BAD3A
:107BC0005CAD0E949A8520E041E060E081E00E9487
:107BD0006C88698F7A8F8B8F9C8F20E041E060E00A
:107BE00081E00E946C8869A37AA38BA39CA39B016C
:107BF000AC01698D7A8D8B8D9C8D0F944A096B0138
:107C00007C010F900F900F900F902DEC3CEC4CEC02
:107C10005DE30F94E30B181654F02DEC3CEC4CECA8
:107C20005DEBC701B6010F94AF0987FF2BC04D85EF
:107C30005E856F8578898EE897E00E94C1A02D85CA
:107C40003E854F85588928323105410551050CF094
:107C500074CF82E30E943D23D1018D919C9192FFCC
:107C60006CCF2D853E854F8558892E5F3F4F4F4FF6
:107C70005F4F2D873E874F87588BBA01A90180E758
:107C800097E086C08DE793E00F942E129A8B898B34
:107C90000E945C1D162F072FF82EE92E8CE393E02F
:107CA0000E942F1D9B01AC0188E393E029AF3AAFFE
:107CB0004BAF5CAF0E942F1DEF92FF920F931F936B
:107CC00010EFA12E13E2B12E14E7C12E19E4D12E2C
:107CD0008601750129AD3AAD4BAD5CAD0E949A8528
:107CE00021E041E060E080E00E946C886DA37EA30B
:107CF0008FA398A721E041E060E080E00E946C88BB
:107D000069A77AA78BA79CA79B01AC016DA17EA157
:107D10008FA198A50F944A096B017C010F900F90D9
:107D20000F900F902DEC3CEC4CEC5DE30F94E30BCB
:107D3000181654F02DEC3CEC4CEC5DEBC701B60191
:107D40000F94AF0987FF32C04D855E856F857889B6
:107D500080E597E00E94C1A08D859E85AF85B8899A
:107D60008897A105B1050CF0E8CE82E30E943D237F
:107D70002D853E854F8558892E5F3F4F4F4F5F4F72
:107D80002D873E874F87588BBA01A90182E397E080
:107D90000E94C1A06D8582E30E941A236D858AE34B
:107DA0000E941A2382E30E943D23C7CE8FE793E00F
:107DB0000F942E129E8B8D8B0E945C1D162F072F09
:107DC000F82EE92E84E493E00E942F1D9B01AC0164
:107DD00080E493E029AF3AAF4BAF5CAF0E942F1D18
:107DE000EF92FF920F931F93B0EFAB2EB3E2BB2E37
:107DF000B4E7CB2EB9E4DB2E8601750129AD3AAD8F
:107E00004BAD5CAD0E949A8521E041E061E080E0ED
:107E10000E946C884B015C0121E041E061E080E060
:107E20000E946C886B017C019B01AC01C501B4010F
:107E30000F944A092B013C010F900F900F900F9067
:107E40002DEC3CEC4CEC5DE30F94E30B181654F076
:107E50002DEC3CEC4CEC5DEBC301B2010F94AF098F
:107E600087FF25C04D855E856F85788982E197E023
:107E70000E94C1A08D859E85AF85B8898897A10590
:107E8000B1050CF05ACE82E30E943D232D853E853C
:107E90004F8558892E5F3F4F4F4F5F4F2D873E874D
:107EA0004F87588BBA01A90184EF96E071CFA501E5
:107EB0009401C701B6010F944B0920E030E040E087
:107EC0005FE30F94570C6DA77EA78FA798AB81E84F
:107ED00093E00F942E128C01D1018D919C911197FA
:107EE00092FF0CC05E968D919D910D90BC91A02D3E
:107EF000892B8A2B8B2B11F00C94924B298D3A8D68
:107F00004B8D5C8D69A17AA18BA19CA10F944B092B
:107F100020E030E040E05FE30F94570C698F7A8FE8
:107F20008B8F9C8F2D8D3E8D4F8D58A12093F90600
:107F30003093FA064093FB065093FC0681E00E94C2
:107F4000C387D1018D919C91119792FFABC05E9632
:107F50008D919D910D90BC91A02D0297A105B10529
:107F600009F0A0C020E030E040EA52E4698D7A8D4B
:107F70008B8D9C8D0F94570C20E030E048EC54E43E
:107F80000F944A090F944F0A6B017C0129893A89A1
:107F9000442737FD4095542F298B3A8B4B8B5C8BB4
:107FA0002DA13EA14FA158A569A57AA58BA59CA599
:107FB0000F944B0920E030E040E05FE30F94570C52
:107FC00020E030E040EA52E40F94570C20E030E02B
:107FD00048EC54E40F944A090F944F0A2B013C01DA
:107FE0008D899E89AA2797FDA095BA2F8D8B9E8B90
:107FF000AF8BB88F20E030E040EA52E46DA57EA55B
:108000008FA598A90F94570C20E030E048EC54E479
:108010000F944A090F944F0A4B015C01222717FD68
:108020002095322FC414D504E604F70414F00C9400
:10803000AA4BC814D904EA04FB0414F00C94D24BE4
:108040004C185D086E087F088D899E89AF89B88DB0
:10805000480E591E6A1E7B1E8C189D08AE08BF086C
:10806000800E911EA21EB31EC2010E94C41DC40137
:108070000E94E41DC12CD12C7601A1E94A16A1E091
:108080005A066104710414F00C94064CB1E98B1685
:10809000B1E09B06A104B10414F00C94064C80E0FE
:1080A0000E9457CF20E030E0A901698D7A8D8B8D39
:1080B0009C8D0F94AF0987FD40CD20E030E0A901F1
:1080C0006DA57EA58FA598A90F94AF0987FD35CD25
:1080D00081E00E94EC808AEB96E00E94341E8EE3E1
:1080E00090E20E9428962D8D3E8D4F8D58A12093B1
:1080F000F9063093FA064093FB065093FC0641E0E4
:1081000061E081E00E94DD87FCC310920408F10168
:10811000EB5AFF4F8081882309F4F3C385EA96E088
:108120000CC081E080930408F101EB5AFF4F80817D
:10813000882309F4E6C380E996E00E94B59FE1C375
:108140008090BF079090C007A090C107B090C20771
:108150004090C3075090C4076090C5077090C60751
:10816000C090C707D090C807E090C907F090CA0731
:10817000D1011C9113FF2BC01A96EC911A971B96F4
:10818000FC911B971C960C911C971D96BC9080919E
:108190004708882361F023E333E34BEC51E4BF014C
:1081A000802F9B2D0F94570CFB01DC0102C0A02FE8
:1081B000BB2D2091E7073091E8074091E9075091E6
:1081C000EA07BF01CD010F944A094B015C0114FF7E
:1081D0002CC0D1011E96EC911E971F96FC911F9703
:1081E00050960C91509751967C9080914708882327
:1081F00061F023E333E34BEC51E4BF01802F972D73
:108200000F94570CFB01DC0102C0A02FB72D209169
:10821000EB073091EC074091ED075091EE07BF015D
:10822000CD010F944A092B013C0115FF2CC0D1014F
:108230005296EC9152975396FC91539754961C91F9
:10824000549755960C9180914708882361F023E359
:1082500033E34BEC51E4BF01812F902F0F94570C67
:10826000FB01DC0102C0A12FB02F2091EF0730915C
:10827000F0074091F1075091F207BF01CD010F9433
:108280004A096B017C0187017601A3019201C501B6
:10829000B4010E94B879F101808186FF32C3E6897A
:1082A000D1015796FC91579758961C91589759961B
:1082B0000C9180914708882361F023E333E34BEC72
:1082C00051E4BF01812F902F0F94570CFB01DC016B
:1082D00002C0A12FB02F209133033091340340917D
:1082E000350350913603BF01CD010F94570C0F9405
:1082F0004F0A6093FF0770930008809301089093E2
:108300000208FFC28090EF079090F007A090F1075D
:10831000B090F207209101073091020740910307C6
:1083200050910407C501B4010F94B6092DEC3CEC43
:108330004CEC5DE30F94E30B18162CF48AE596E001
:108340000E94BF9FDEC2F10122818081918122FFC4
:108350000CC083FF02C00C94224C80739927892B98
:1083600011F00C94224C0C94284C83FF6FC0C284F3
:10837000D384E484F58420E030E0A901C701B6018C
:108380000F94E30B181664F420E030E040E251E46F
:10839000C701B6010F94AF0918160CF459C00AC0F2
:1083A00020E030E040E251ECC701B6010F94E30B4E
:1083B00087FD4EC0A5019401C701B6010F944B097A
:1083C0009B01AC0160910D0770910E0780910F0722
:1083D000909110070F944B0960930D0770930E074F
:1083E00080930F07909310070E94E37440910D074C
:1083F00050910E0760910F077091100723E08DE5F3
:1084000095E00E949DA180910D0790910E07A0918B
:108410000F07B091100789879A87AB87BC8744E024
:1084200050E065E870E0CE0109960F9433120E9487
:1084300040CF682F88E690E069AF0F94211269ADB4
:10844000681721F088E690E00F943C1210E001C01C
:1084500011E0F101808184FF71C0C684D784E08877
:10846000F18820E030E0A901C701B6010F94E30BC9
:10847000181664F420E030E040E251E4C701B60190
:108480000F94AF0918160CF458C00AC020E030E071
:1084900040E251ECC701B6010F94E30B87FD4DC0DC
:1084A000A5019401C701B6010F944B099B01AC01D2
:1084B0006091050770910607809107079091080762
:1084C0000F944B0960930507709306078093070785
:1084D000909308070E94E3744091050750910607A6
:1084E000609107077091080723E082E495E00E94FD
:1084F0009DA18091050790910607A0910707B09173
:1085000008078D839E83AF83B88744E050E069E815
:1085100070E0CE0105960F9433120E9440CF682F71
:1085200088E690E069AF0F94211269AD681731F0C9
:1085300088E690E00F943C1201C011E0D1018C91CB
:1085400085FF74C05296CD90DD90ED90FC905597CC
:1085500020E030E0A901C701B6010F94E30B181623
:108560005CF420E030E040E251E4C701B6010F9432
:10857000AF0918165CF00EC020E030E040E251EC8C
:10858000C701B6010F94E30B87FF04C08BEA95E0A7
:108590000C94244CA5019401C701B6010F944B091A
:1085A0009B01AC016091FD067091FE068091FF0673
:1085B000909100070F944B096093FD067093FE069F
:1085C0008093FF06909300070E94E3744091FD069C
:1085D0005091FE066091FF067091000723E087E24C
:1085E00095E00E949DA18091FD069091FE06A091CC
:1085F000FF06B091000789839A83AB83BC8344E074
:1086000050E06DE870E0CE0101960F9433120E94A5
:1086100040CF682F88E690E069AF0F94211269ADD2
:10862000681721F088E690E00F943C121111AECF4C
:1086300089E48F9384E78F9383E28F9380EF8F9306
:10864000F0EFAF2EF3E2BF2EF4E7CF2EF9E4DF2EEA
:10865000E12CF12C00E411E4A6019501C601B5015D
:108660000E949A850F900F900F900F904AC180E062
:108670000E94C3871092BF071092C0071092C107D3
:108680001092C2071092C3071092C4071092C50738
:108690001092C6071092C7071092C8071092C90718
:1086A0001092CA076091130370911403809115030F
:1086B000909116030E943B7A80913D0790913E076E
:1086C000A0913F07B0914007409135075091360780
:1086D0006091370770913807C0903907D0903A07FA
:1086E000E0903B07F0903C075A01F62FE72F481720
:1086F00059076A077B071CF45C01FA2FEB2F8501F1
:108700002F2F3E2F0C151D052E053F0514F4970144
:108710008601480159018C189D08AE08BF08680100
:108720007901C41AD50AE60AF70A28013901481A5C
:10873000590A6A0A7B0AB501A40180E093E20E940B
:10874000C1A0B701A60187EF92E20E94C1A0B301C8
:10875000A2018EEE92E20E94C1A0F101808191817E
:1087600092FFCDCC868D978DA0A1B1A118161906C8
:108770001A061B060CF0C3CCC4010E94A41DC6013E
:108780000E94C41DC2010E94E41DB9CC7090BE07B6
:1087900075FA772470F880E00E94C3871092F3077F
:1087A0001092F4071092F5071092F6071092F7074F
:1087B0001092F8071092F9071092FA071092FB072F
:1087C0001092FC071092FD071092FE071092BF074F
:1087D0001092C0071092C1071092C2071092C307EF
:1087E0001092C4071092C5071092C6071092C707CF
:1087F0001092C8071092C9071092CA071092070872
:10880000109208081092090810920A0810920B089A
:1088100010920C0810920D0810920E0810920F087A
:108820001092100810921108109212086091130310
:108830007091140380911503909116030E943B7A66
:1088400000912107109122072091230730912407DE
:108850008091150790911607A0911707B0911807FE
:10886000081B190B2A0B3B0B08511C4F2F4F3F4F76
:108870008091350790913607A0913707B09138075E
:1088800048015901881A990AAA0ABB0A80913D0732
:1088900090913E07A0913F07B09140076801790190
:1088A000C81AD90AEA0AFB0A8091390790913A0757
:1088B000A0913B07B0913C07B901A801481B590B97
:1088C0006A0B7B0B80E093E20E94C1A0B501A4017A
:1088D00087EF92E20E94C1A0B701A6018EEE92E25C
:1088E0000E94C1A0872D0E94C38709CC8091EA0213
:1088F00082FF07C08CE594E20E94859FC1010E941F
:108900006F970F94E6036093811D7093821D80938F
:10891000831D9093841DEC960FB6F894DEBF0FBEB6
:10892000CDBFDF91CF911F910F91FF90EF90DF901E
:10893000CF90BF90AF909F908F907F906F905F90FF
:108940004F903F902F9008950E94531D81110C94D9
:108950006B370E94581D81110C946B37D2CF0E9447
:10896000531D81110C94E1370E94581D81110C9404
:10897000E1378FE390E20E94289680E00E94C3874F
:108980000E945C1D162F072FF82EE92E84E393E03A
:108990000E942F1D9B01AC0180E393E029AF3AAF09
:1089A0004BAF5CAF0E942F1DEF92FF920F931F936E
:1089B00050EFA52E53E2B52E54E7C52E59E4D52E1F
:1089C0008601750129AD3AAD4BAD5CAD0E949A852B
:1089D00020E041E060E081E00E946C8869A77AA70E
:1089E0008BA79CA720E041E060E081E00E946C88BA
:1089F00069A37AA38BA39CA39B01AC0169A57AA56B
:108A00008BA59CA50F944A096B017C010F900F90D8
:108A10000F900F902DEC3CEC4CEC5DE30F94E30BCE
:108A2000181654F02DEC3CEC4CEC5DEBC701B60194
:108A30000F94AF0987FF1AC049895A896B897C89CD
:108A400082EC9BE00E94C1A089899A89AB89BC898C
:108A50008897A105B10511F40C941B3882E30E949C
:108A60003D23B301A20184EA9BE01BC18DE793E0A3
:108A70000F942E129E8B8D8BD1018D919C9111970D
:108A800092FF0BC05E968D919D910D90BC91A02D93
:108A90000297A105B10509F453C40E945C1D162F6D
:108AA000072FF82EE92E8CE393E00E942F1D9B01E7
:108AB000AC0188E393E029AF3AAF4BAF5CAF0E94C3
:108AC0002F1DEF92FF920F931F9300EFA02E03E252
:108AD000B02E04E7C02E09E4D02E8601750129AD21
:108AE0003AAD4BAD5CAD0E949A8520E041E060E07C
:108AF00081E00E946C886DA77EA78FA798AB20E0CD
:108B000041E060E081E00E946C8869AB7AAB8BAB9E
:108B10009CAB9B01AC016DA57EA58FA598A90F9478
:108B20004A096B017C010F900F900F900F902DEC74
:108B30003CEC4CEC5DE30F94E30B181654F02DEC79
:108B40003CEC4CEC5DEBC701B6010F94AF0987FF1D
:108B500021C049895A896B897C898FE49BE00E94F6
:108B6000C1A029893A894B895C89283231054105A0
:108B7000510541F082E30E943D23B301A20181E34C
:108B80009BE08FC08EE19BE00E949E9F86E09BE071
:108B90000C9421388FE793E00F942E129E8F8D8FC7
:108BA000D1018D919C91119792FF0BC05E968D9192
:108BB0009D910D90BC91A02D0297A105B10509F4DE
:108BC000CCC30E945C1D162F072FF82EE92E84E4DB
:108BD00093E00E942F1D9B01AC0180E493E029AF3C
:108BE0003AAF4BAF5CAF0E942F1DEF92FF920F93F5
:108BF0001F9310EFA12E13E2B12E14E7C12E19E43A
:108C0000D12E8601750129AD3AAD4BAD5CAD0E9408
:108C10009A8520E041E060E081E00E946C886B0171
:108C20007C0120E041E060E081E00E946C886DAB57
:108C30007EAB8FAB98AF9B01AC01C701B6010F941F
:108C40004A094B015C010F900F900F900F902DEC93
:108C50003CEC4CEC5DE30F94E30B181654F02DEC58
:108C60003CEC4CEC5DEBC501B4010F94AF0987FF00
:108C700042C049895A896B897C898CED9AE00E94AF
:108C8000C1A029893A894B895C892832310541057F
:108C9000510549F182E30E943D23B301A2018EEB0D
:108CA0009AE00E94C1A0642D82E30E941A23642DE1
:108CB0008AE30E941A2382E30E943D23F2E04F0ED2
:108CC000511C611C711C29893A894B895C892E5F72
:108CD0003F4F4F4F5F4F298B3A8B4B8B5C8B31E073
:108CE0003DA30C94D0378BEA9AE00E949E9F83E9C3
:108CF0009AE00C94213829A13AA14BA15CA169A565
:108D00007AA58BA59CA50F944B0920E030E040E0AC
:108D10005FE30F94570C20E030E040EA52E40F94F8
:108D2000570C20E030E048EC54E40F944A090F94CB
:108D30004F0A4B015C018D899E89AA2797FDA0955A
:108D4000BA2F8D8B9E8BAF8BB88F29A93AA94BA9CF
:108D50005CA96DA57EA58FA598A90F944B0920E06D
:108D600030E040E05FE30F94570C20E030E040EA51
:108D700052E40F94570C20E030E048EC54E40F9498
:108D80004A090F944F0A2B013C012D8D3E8D44273B
:108D900037FD4095542F2D8F3E8F4F8F58A32DA90F
:108DA0003EA94FA958ADC701B6010F944B0920E069
:108DB00030E040E05FE30F94570C20E030E040EA01
:108DC00052E40F94570C20E030E048EC54E40F9448
:108DD0004A090F944F0A6B017C0181E893E00F94DC
:108DE0002E129C01442737FD4095542F29A33AA306
:108DF0004BA35CA380E00E94EC800E94E3748BE5AF
:108E000090E20E94B59F4091010750910207609146
:108E100003077091040722E086EC9FE10E949DA168
:108E2000898D9A8DAB8DBC8D8093F9069093FA064F
:108E3000A093FB06B093FC0684149504A604B70423
:108E400014F58C149D04AE04BF040CF042C0481805
:108E500059086A087B082D8D3E8D4F8D58A1420E12
:108E6000531E641E751EC818D908EA08FB0889A19C
:108E70009AA1ABA1BCA1C80ED91EEA1EFB1E812C73
:108E8000912C540152C0481459046A047B040CF517
:108E90004C145D046E047F04E4F484189508A6085D
:108EA000B7082D893E894F89588D820E931EA41EC6
:108EB000B51EC418D508E608F70889A19AA1ABA188
:108EC000BCA1C80ED91EEA1EFB1E412C512C32013A
:108ED00025C0C814D904EA04FB0404F5C414D5045D
:108EE000E604F704DCF48C189D08AE08BF082D8951
:108EF0003E894F89588D820E931EA41EB51E4C18B4
:108F00005D086E087F088D8D9E8DAF8DB8A1480ECF
:108F1000591E6A1E7B1EC12CD12C760191E989163F
:108F200091E09906A104B10474F4A1E94A16A1E004
:108F30005A06610471043CF4B1E9CB16B1E0DB06DA
:108F4000E104F104FCF049895A896B897C8982E645
:108F50009AE00E94C1A088E49AE00E942896B50198
:108F6000A40184E49AE00E94C1A0B301A20180E4BC
:108F70009AE00E94C1A0B701A6018CE39AE00E948A
:108F8000C1A0BFCCC4010E94A41DC2010E94C41D87
:108F9000C6010E94E41D80E00E9457CF0C942B383C
:108FA0002DEC3CEC4CEC5DEBC301B2010F94AF092E
:108FB00087FF09C00C94A13882ED99E00E949E9F22
:108FC0008AEB99E0D0C09FEF291A390AA5019401D4
:108FD000C701B6010F944B0920E030E040E05FE3A9
:108FE0000F94570C2B013C0140910107509102074F
:108FF000609103077091040722E08CEA99E00E94D7
:109000009DA12091EF073091F0074091F107509119
:10901000F207C301B2010F944A099B01AC016091B0
:1090200001077091020780910307909104070F9444
:109030004B09609301077093020780930307909395
:1090400004070E94E3744091010750910207609168
:1090500003077091040722E08EE999E00E949DA128
:109060000E945C1D162F072FF82EE92E84E493E052
:109070000E942F1D9B01AC0180E493E029AF3AAF21
:109080004BAF5CAF0E942F1DEF92FF920F931F9387
:10909000A0EFAA2EA3E2BA2EA4E7CA2EA9E4DA2EE4
:1090A0008601750129AD3AAD4BAD5CAD0E949A8544
:1090B00020E041E060E081E00E946C886B017C016F
:1090C00020E041E060E081E00E946C886D8B7E8B47
:1090D0008F8B988F9B01AC01C701B6010F944A0991
:1090E0004B015C010F900F900F900F902DEC3CEC1A
:1090F0004CEC5DE30F94E30B181654F02DEC3CECB4
:109100004CEC5DEBC501B4010F94AF0987FF33C090
:109110004D855E856F8578898FE699E00E94C1A0B4
:109120002D853E854F8558892832310541055105E9
:10913000A4F482E30E943D238D859E85AF85B88986
:109140000296A11DB11D8D879E87AF87B88BAC019C
:10915000BD0181E599E00C94C6388EE399E00E9448
:109160009E9F86E299E00E94289686ED9FE10E94EC
:10917000BF9F0C94D8382D893E894F89588DC701DF
:10918000B6010F944B0920E030E040E05FE30F941C
:10919000570C9B01AC01C301B2010F944A0920E0B6
:1091A00030E040EA52E40F94570C6B017C0120E060
:1091B00030E0A9010F94AF0987FF27C0C701B601AE
:1091C000905820916D0730916E0740916F07509134
:1091D00070070F94B6099B01AC010F944B096B010A
:1091E0007C0122E0AB01BC018AE690E20E949DA1D5
:1091F000A701960160916D0770916E0780916F07CE
:10920000909170070F944A0918C080906D07909054
:109210006E07A0906F07B0907007A5019401C70179
:10922000B6010F94B6099B01AC010F944B099B0149
:10923000AC01C501B4010F944B0960936D077093A5
:109240006E0780936F0790937007C0906D07D09062
:109250006E07E0906F07F090700722EC35EF41EB5E
:1092600052E4C701B6010F94B6094B015C012DEC25
:109270003CEC4CE85FE30F94E30B181654F026E641
:1092800036E646E65FE3C501B4010F94AF0987FFF8
:1092900013C022E0B701A6018BE099E00E949DA1D6
:1092A00082EC95EFA1EBB2E480936D0790936E078B
:1092B000A0936F07B093700722E049895A896B89A0
:1092C0007C8983EF98E00E949DA140916D075091A9
:1092D0006E0760916F077091700722E08BED98E048
:1092E0000E949DA194E02916310414F00C94D83802
:1092F00029893A894B895C8960916D0770916E0765
:1093000080916F07909170070F944A096B017C015F
:109310002DEC3CEC4CEC5DE30F94E30B181614F4CD
:109320000C9444382DEC3CEC4CEC5DEBC701B601E1
:109330000F94AF0987FF02C00C9444380C94D838BE
:1093400041E061E081E00E94DD878FE390E20E94CE
:10935000289680E00E94C387A0CB41E061E081E0D5
:109360000E94DD878FE390E20E94289680E00E94B1
:10937000C38727CCC90188719927489709F474C11C
:1093800020E041E060E081E00E946C882091EF07DE
:109390003091F0074091F1075091F2070F944A097C
:1093A0004B015C0120E041E061E080E00E946C88BC
:1093B0002091EF073091F0074091F1075091F207AB
:1093C0000F944A092B013C019B01AC01C501B4017A
:1093D0000F944A096B017C012DEC3CEC4CEC5DE3F5
:1093E0000F94E30B181654F02DEC3CEC4CEC5DEBB9
:1093F000C701B6010F94AF0987FF21C022E0B70172
:10940000A6018AE998E00E949DA182E30E943D2383
:1094100046E150E060E070E08CE798E00E94C1A077
:1094200066E182E30E941A2366E18AE30E941A231E
:1094300082E30E943D2388E798E00C941339A3014E
:109440009201C501B4010F944B0920E030E040E0E7
:109450005FE30F94570CAB01BC0122E089E698E072
:109460000E949DA14ECA8091F9069091FA06A091A2
:10947000FB06B091FC068D879E87AF87B88BF10104
:109480008081918192FF09C0868D978DA0A1B1A1A5
:109490000297A105B10509F4AEC041E061E081E0A9
:1094A0000E94DD878FE390E20E94289680E00E9470
:1094B000C3870E945C1D9F938F937F936F93F0EF00
:1094C000AF2EF3E2BF2EF4E7CF2EF9E4DF2E8601B4
:1094D000750120E030E0A901CA01B9010E949A8516
:1094E00020E041E060E081E00E946C884B015C017B
:1094F00020E041E060E081E00E946C886B017C012B
:109500009B01AC01C501B4010F944A092B013C0138
:109510000F900F900F900F902DEC3CEC4CEC5DE316
:109520000F94E30B181654F02DEC3CEC4CEC5DEB77
:10953000C301B2010F94AF0987FF05C086ED9FE11B
:109540000E94BF9F9CCFA5019401C701B6010F9453
:109550004B0920E030E040E05FE30F94570C6B01D3
:109560007C0120E030E040E85FE30F94AF0987FD25
:1095700086CFD1018D919C91119792FF0BC05E9681
:109580008D919D910D90BC91A02D892B8A2B8B2BB9
:1095900009F043C02D853E854F8558892093F906F3
:1095A0003093FA064093FB065093FC0681E00E943C
:1095B000C387D1018D919C91119792FF0BC05E964C
:1095C0008D919D910D90BC91A02D0297A105B105A3
:1095D00009F446C081E00E94EC8087EB98E00E948D
:1095E000341E8EE390E20E9428962D853E854F859D
:1095F00058890C94774020E030E046E653E420930D
:10960000010730930207409303075093040780E05B
:109610000E9457CF0E94B4D140CF2091EF073091E4
:10962000F0074091F1075091F207C701B6010F947E
:109630004A099B01AC01609101077091020780917A
:109640000307909104070F944B09609301077093EF
:10965000020780930307909304070E94E3749ACF54
:1096600080E00E9457CFB6CF30FF27C0D1011E96B1
:109670002D913D914D915C9151971A966D917D91EF
:109680008D919C911D975D96EC915D97EF935C9603
:10969000EC915C97EF935B96EC915B97EF935A9606
:1096A000EC91EF93E0EFAE2EE3E2BE2EE4E7CE2E98
:1096B000E9E4DE2E860175011BC00E945C1DF101EC
:1096C0002685378540895189428453846484758412
:1096D0009F938F937F936F9360EFA62E63E2B62ED6
:1096E00064E7C62E69E4D62E86017501C301B20176
:1096F0000E949A850F900F900F900F9041CE80E0BE
:1097000090E00E94A41D80E090E00E94C41D80E0D3
:1097100090E00E94E41D80E00E9457CF0E94B4D1E7
:109720000C94AF3D80E00E94EC800E94E3748BE5D6
:1097300090E20E94B59F409101075091020760910D
:1097400003077091040722E086EC9FE10E949DA12F
:109750000C947E3F4C145D046E047F041CF5481489
:1097600059046A047B04F4F4C418D508E608F70821
:1097700089899A89AB89BC89C80ED91EEA1EFB1E4D
:1097800084189508A608B708800E911EA21EB31E65
:10979000C6010E94A41DC4010E94E41D412C512C4D
:1097A00032012BC08C149D04AE04BF0434F5841424
:1097B0009504A604B7040CF5C818D908EA08FB08F4
:1097C00029893A894B895C89C20ED31EE41EF51E95
:1097D000481859086A087B088D899E89AF89B88D19
:1097E000480E591E6A1E7B1EC6010E94A41DC2019E
:1097F0000E94C41D812C912C540191E9C91691E05D
:10980000D906E104F10414F40C943D404D855E85C5
:109810006F8578898BEC96E00E94C1A0B701A60104
:1098200087EC96E00E94C1A0B301A20183EC96E010
:109830000E94C1A0B501A4018FEB96E00E94C1A0D7
:109840000C949D3D80E396E00E94BF9F0C941843CA
:10985000C6A4D7A4E0A8F1A820E030E0A901C70180
:10986000B6010F94AF09882361F120E030E0A9012F
:10987000C701B6010F94E30B18165CF420E030E04A
:1098800040E251E4C701B6010F94AF091816B4F0D5
:109890000AC020E030E040E251ECC701B6010F946D
:1098A000E30B87FD0BC085E793E00E942F1D9B0112
:1098B000AC01C701B6010F944B094DC087E096E09B
:1098C000C3CF20E030E0A9016091E7077091E8077D
:1098D0008091E9079091EA070F94AF09811161C067
:1098E00020E030E0A9016091EB077091EC078091D6
:1098F000ED079091EE070F94AF09811152C080914E
:10990000BE0787FF2CC0C0907907D0907A07E090FF
:109910007B07F0907C0760910B0870910C08809198
:109920000D0890910E080F94800A9B01AC010F94D2
:10993000570C9B01AC01C701B6010F944A090F9463
:10994000C40C20913F08309140084091410850914B
:1099500042080F94570C0E945F1D0C941843C0904E
:109960007907D0907A07E0907B07F0907C076091B0
:109970000B0870910C0880910D0890910E089B01C6
:10998000AC010F941E0DC61AD70AE80AF90AC701DE
:10999000B6010E94EAD9BC0180E090E00F94800AF1
:1099A000D0CF84ED95E050CFCF93DF93EC01409181
:1099B000EA028881998144FF09C082FD2AC081FFA3
:1099C00005C02E813F812F36310519F582FF05C074
:1099D000CE01DF91CF910C949D3581FF05C0CE0162
:1099E000DF91CF910C94482491FF08C00E94261E5D
:1099F000CC5ADF4F8881DF91CF91E1C242FF13C083
:109A00008CE594E20E94859FCE01DF91CF910C946A
:109A10006F970F94E6036093811D7093821D80936E
:109A2000831D9093841DDF91CF9108958091BC0791
:109A300080FD1DC00E9462980E94EE92EC018CE6AF
:109A40009AE00E9474CA2097B1F08091830988231C
:109A500041F0888181FF12C08E819F814D9771F402
:109A600016C0CE01A1DFCE010E944D9804C08CE645
:109A70009AE00E9474CA0E94D979D8CFBE0188E1C9
:109A800099E00E948E9BCE010E943C98ECCF88E129
:109A900099E00E94039FF7CF0E946A8C0C94582390
:109AA000C5CFCF93DF93FC01E05CFF4F208121FD08
:109AB0001FC0DB014D915D916D917C91DC01AF5B2D
:109AC000BF4F4D935D936D937C931397EC01CB5BEC
:109AD000DF4FDC0117964D915D916D917C911A9746
:109AE000488359836A837B83822F897F8260808346
:109AF000DF91CF9108959F92AF92BF92CF92DF9264
:109B0000EF92FF920F931F93CF93DF93EC015B01D2
:109B10008C01005C1F4FF801908092FC32C0CB8416
:109B2000DC84ED84FE84A70196016F8178858985A8
:109B30009A850F944A099F7720E030E040E85FE380
:109B40000F944B0920E030E040EA51E40F94E30B1E
:109B50001816BCF0F50180819181A281B381FE01CC
:109B6000EF5BFF4F80839183A283B383CB5BDF4F97
:109B7000C882D982EA82FB82892D897F8460F801BC
:109B80008083DF91CF911F910F91FF90EF90DF9035
:109B9000CF90BF90AF909F9008958091BE07846052
:109BA0008093BE0708952F923F924F925F926F92DB
:109BB0007F928F929F92AF92BF92CF92DF92EF925D
:109BC000FF920F931F93CF93DF93CDB7DEB76497C8
:109BD0000FB6F894DEBF0FBECDBF382E292E7A8780
:109BE00069875A834983098B1A8B2B8B3C8B4AA438
:109BF0005BA46CA47DA423E333E948E853E4C501E6
:109C0000B4010F944B096D837E838F83988720E086
:109C100030E0A901C301B2010F94AF09882359F1C3
:109C20002EA53FA548A959A9C301B2010F944B091C
:109C30004B015C0120E030E040EA50E4C301B20196
:109C40000F94570CA50194010F94B6096D877E8778
:109C50008F87988BA30192016EA57FA588A999A9EA
:109C60000F94570CA50194010F94B6096EA77FA716
:109C700088AB99AB08C080E090E0A0EAB0E48D87A3
:109C80009E87AF87B88B2D813E814F81588569892A
:109C90007A898B899C8990580F94B6090F94230A6E
:109CA0009B01AC01C701B6010F94570C6D837E83F5
:109CB0008F83988769817A81A985BA856A1B7B0B16
:109CC000882777FD8095982F0F94820A20E030E056
:109CD00040E05DE30F94570C69877A878B879C87F8
:109CE000032D122D212C312C89819A81AA2797FDD1
:109CF000A095BA2F89839A83AB83BC83A895698189
:109D00007A818B819C810F94820A6B017C01B10165
:109D1000882777FD8095982F0F94820A29853A85A8
:109D20004B855C850F94570C9B01AC01C701B601B4
:109D30000F944A096B017C0123E333E548E853E4BF
:109D40000F944B099B01AC0169897A898B899C89A5
:109D50000F94B6090F94230A2D813E814F815885B7
:109D60000F94570C4B015C0120E030EC4FE755E4B9
:109D70000F94570C2D853E854F8558890F94570CAD
:109D80002B013C01A50194016EA57FA588A999A985
:109D90000F944B0920E030E040EA50E40F94570C58
:109DA0009B01AC01C301B2010F94B6090F944F0A95
:109DB0006D3F9FE0790714F06CEF7FE0D8016D9361
:109DC0007C9320E030E040E051E4C701B6010F94FD
:109DD000570C0F944F0AF80173836283FFEF2F1A19
:109DE0003F0A0C5F1F4F81E22816310409F086CF2D
:109DF00064960FB6F894DEBF0FBECDBFDF91CF9152
:109E00001F910F91FF90EF90DF90CF90BF90AF9098
:109E10009F908F907F906F905F904F903F902F908A
:109E20000895CF92DF92EF92FF92CF93DF93EC01F0
:109E30008B898130A9F5CE8CDF8CE8A0F9A020E0D9
:109E400030E0A901C701B6010F94AF09882341F1A1
:109E5000688D70E080E090E00F94800A20E030E0B0
:109E600040E251E40F94570CA70196010F94B609F4
:109E70006FA378A789A79AA7698D70E080E090E02A
:109E80000F94800A20E030E040E251E40F94570C38
:109E9000A70196010F94B6096BA77CA78DA79EA773
:109EA000DF91CF91FF90EF90DF90CF9008958EE0FB
:109EB00092E0B7CF7F928F929F92AF92BF92CF9254
:109EC000DF92EF92FF920F931F93CF93DF938BE577
:109ED00092E0909387038093860385E4782E7F92A7
:109EE000D2E9DF93C0EECF931F921F921F921F9271
:109EF0001F92812C912C98ECA92E91E4B92EC12CA3
:109F000020E5D22E23ECE22E27E4F22E00E010E131
:109F10002BE835E44CE251E06EEC7FEF8DE094E00D
:109F200042DE7F92DF93CF931F921F921F921F9268
:109F30001F9200E018E728E835E44CE251E06CEEAF
:109F40007FEF89E893E02FDE80910A01806480939F
:109F50000A013B9A809168022DB73EB7205F3F4FC0
:109F60000FB6F8943EBF0FBE2DBF87FD0CC061E059
:109F70000F94FA0480916902811105C061E080911B
:109F800068020F9433050F94E60360939502709373
:109F9000960280939702909398029D9AA59887DFE6
:109FA000DF91CF911F910F91FF90EF90DF90CF90B5
:109FB000BF90AF909F908F907F900C94DEDA4F927D
:109FC0005F926F927F92AF92BF92CF92DF92EF92A9
:109FD000FF920F931F93CF93DF93CDB7DEB72C97EC
:109FE0000FB6F894DEBF0FBECDBF8091FF079091F2
:109FF0000008A0910108B0910208E0918603F09159
:10A000008703838F948FA58FB68F2BE532E0309333
:10A010008703209386038093D7079093D807A09354
:10A02000D907B093DA0740906402509065026090BF
:10A03000660270906702409233035092340360923C
:10A04000350370923603A301920160E070E080E86E
:10A050009FE30F94B609609343087093440880937C
:10A06000450890934608C0906A02D0906B02E09039
:10A070006C02F0906D02C0922303D0922403E09210
:10A080002503F092260360916E0270916F02809119
:10A090007002909171026093F7027093F8028093BE
:10A0A000F9029093FA026093070370930803809378
:10A0B000090390930A03A30192010F94570C0F9484
:10A0C000540A609333087093340880933508909352
:10A0D0003608609323087093240880932508909392
:10A0E00026082091720230917302409174025091BF
:10A0F0007502C301B2010F94570C9B01AC0160E0E3
:10A1000074E284E798E40F94B6090F94BD0A0F94A3
:10A11000540A162F60934B08A3019201C701B601A0
:10A120000F94570C9B01AC0160E074E284E798E463
:10A130000F94B6090F94BD0A0F94540A603118F4B5
:10A1400060934A0803C08FE080934A0880914A08D0
:10A15000811710F010934A0860914A0870E080E07F
:10A1600090E00F94800AA30192010F94570C9B0179
:10A17000AC0160E074E284E798E40F94B6092B0127
:10A180003C01A70196010F94AF0987FF08C04092D8
:10A19000230350922403609225037092260386E8DD
:10A1A00092E03FDE2091E7073091E8074091E90710
:10A1B0005091EA072D833E834F8358874090EB07E9
:10A1C0005090EC076090ED077090EE078091EF07DC
:10A1D0009091F007A091F107B091F20789879A87D3
:10A1E000AB87BC872091F9063091FA064091FB06B7
:10A1F0005091FC0629833A834B835C83E09086036D
:10A20000F0908703F70181819281A381B4819C0141
:10A21000AD0166277727CB01621B730B840B950B6F
:10A220000F94820A209137083091380840913908FC
:10A2300050913A080F94570C6093ED067093EE0618
:10A240008093EF069093F006F70185819681A781B0
:10A25000B0859C01AD0166277727CB01621B730B8C
:10A26000840B950B0F94820A20913B0830913C0897
:10A2700040913D0850913E080F94570C6093E906B9
:10A280007093EA068093EB069093EC068091F506B6
:10A290009091F6060E94801F8091BD0780FF24C028
:10A2A00080910E038F9380910D038F9380910C0307
:10A2B0008F9380910B038F9330EFA32E33E2B32E55
:10A2C00034E7C32E39E4D32EE984FA840B851C8548
:10A2D000A30192016D817E818F8198850E942F7EDE
:10A2E0000F900F900F900F9089819A81AB81BC8164
:10A2F0008093F9069093FA06A093FB06B093FC06B0
:10A3000080E00E94EC802C960FB6F894DEBF0FBE62
:10A31000CDBFDF91CF911F910F91FF90EF90DF9014
:10A32000CF90BF90AF907F906F905F904F900C94C4
:10A33000D3DCE0910C02F0910D026781708581857C
:10A3400092850895E0918603F0918703858587FDC6
:10A3500006C061E09685911160E00D943305089583
:10A360008091680287FD07C061E0909169029111B8
:10A3700060E00D94330508952F923F924F925F92C3
:10A380006F927F928F929F92AF92BF92CF92DF9205
:10A39000EF92FF920F931F93CF93DF9300D01F9202
:10A3A000CDB7DEB79C838B83DC011196EC91E5334E
:10A3B00038F4E23348F5EE2369F0ED3090F50DC046
:10A3C000E43628F4E13648F4EC33F1F02AC0E43600
:10A3D000D9F027C049E150E026C0AB81BC8112967C
:10A3E0008C91A82FB0E0AA0FBB1FAF56BB4F4D9169
:10A3F0005C918CEF9FE0841B950BAB81BC81149624
:10A400009C938E93139715C0AB81BC8112968C914F
:10A41000A82FB0E0AA0FBB1FAF56BB4F4D915C9168
:10A4200002C04FEF5FE0AB81BC8114965C934E930A
:10A430001397AB81BC8113960D911C911497E53352
:10A4400038F5E23308F0A0C0EE2309F450C0ED3037
:10A4500008F081C1E1508E2F90E0FC01E45AF14FE9
:10A460004491440FFC01EE0FFF1FE859F14F859115
:10A470009491FC0185909490FC013296A590B49043
:10A480007CEF672E7FE0772E601A710A52E03CC0A5
:10A49000E436C0F4E13608F0DBC0EC3309F05BC110
:10A4A000B801882777FD8095982F0F94820A20E0C5
:10A4B00030E04AE754E40F94570C20E030E040E8E5
:10A4C00059E325C1E43609F046C1B801882777FD74
:10A4D0008095982F0F94820A20E030E04AEF53E4F1
:10A4E0000F94570C20E030E040E859E32CC180E0A5
:10A4F00090E0A8ECB1E4EB81FC8187839087A18791
:10A50000B28729C151014801541708F011C1FC015B
:10A51000E50FF11DE50FF11D05911491FC0161E0BE
:10A52000650FE60FF11D5E5FE60FF11D259034907B
:10A53000601671063CF7B501882777FD8095982F46
:10A540000F94820A6B017C01B3016819790988278D
:10A5500077FD8095982F0F94820A2B013C01B10161
:10A560006A197B09882777FD8095982F0F94820AB6
:10A570009B01AC01C301B2010F94570C2B013C01AC
:10A58000B80168197909ADC0EE528E2F90E0FC0138
:10A59000E45AF14F6491660FFC01EE0FFF1FE8597A
:10A5A000F14F85919491FC0125903490FC013296F5
:10A5B0008590949072E0761708F044C0FC01E70F94
:10A5C000F11DE70FF11DA590B490FC0121E0270FCC
:10A5D000E20FF11D7E5FE20FF11D259134910A1506
:10A5E0001B056CF5B401882777FD8095982F29838A
:10A5F0003A830F94820A6B017C01B80162197309D6
:10A60000882777FD8095982F0F94820A2B013C01B3
:10A6100029813A81B90168197909882777FD8095E0
:10A62000982F0F94820A9B01AC01C301B2010F94D1
:10A63000570C2B013C01B5016219730952C0490145
:10A640001501B9CFB901882777FD8095982F75C07E
:10A65000E23639F0A0900D04B0900E04EDE0F4E085
:10A6600006C0A0908903B0908A03E9E8F3E08280F5
:10A6700093804CEF642E4FE0742E601A710A82E0D2
:10A68000048115818E5F26803780601671060CF07C
:10A6900049C0B401882777FD8095982F0F94820ACE
:10A6A0006B017C01B3016A197B09882777FD8095CE
:10A6B000982F0F94820A2B013C01B1016819790986
:10A6C000882777FD8095982F0F94820A9B01AC0113
:10A6D000C301B2010F94570C2B013C01B8016A1958
:10A6E0007B09882777FD8095982F0F94820A9B011C
:10A6F000AC01C301B2010F94B6099B01AC01C701C3
:10A70000B6010F944B0920E030E040E05EE30F9487
:10A71000570CAB81BC8117966D937D938D939C9361
:10A720001A9719C03496823419F041015801A8CF04
:10A73000B101882777FD8095982F0F94820A20E039
:10A7400030E040E05EE30F94570CEB81FC816783BF
:10A750007087818792870F900F900F900F90DF91F5
:10A76000CF911F910F91FF90EF90DF90CF90BF900E
:10A77000AF909F908F907F906F905F904F903F90A1
:10A780002F9008958F929F92AF92BF92CF92DF92B7
:10A79000EF92FF920F931F93CF93DF93EC01CB01C6
:10A7A000BA016B877C878D879E87FE01E05CFF4F37
:10A7B0002081297F208320E030E040E051E40F94A5
:10A7C000570C0F944F0A4B012981253318F522337A
:10A7D00008F08AC0222309F448C02D3008F019C1BE
:10A7E000215030E0F901E45AF14FB490BB0CF9016B
:10A7F000EE0FFF1FE859F14F25913491F901E590D3
:10A80000F490F901329645915491C12CD12CB2E0CB
:10A81000AB2E30C02436B0F4213608F0B4C02C334F
:10A8200009F0F7C0882777FD8095982F2CE0660FF8
:10A83000771F881F991F2A95D1F728EE33E040E053
:10A8400050E09CC0243609F0E4C0882777FD80954D
:10A85000982F0CE0660F771F881F991F0A95D1F774
:10A8600024EF31E040E050E089C01E821D82D1C05B
:10A87000A8017D01AB1498F5F901EA0DF11DEA0D6F
:10A88000F11DA591B4916D01F90111E01A0DE10FCF
:10A89000F11DA394A394E10FF11D059114910815E6
:10A8A000190534F79A01261B370BC7018A1B9B0B2E
:10A8B000DC016CEFC62E6FE0D62ECE18DF080F94A9
:10A8C000A50D9A01201B310B442737FD4095542FCD
:10A8D0000F94830DC20ED31EDE82CD829AC08CEF00
:10A8E0009FE08C199D0993C02E5230E0F901E45A83
:10A8F000F14FA491AA0FF901EE0FFF1FE859F14F94
:10A9000025913491F90105911491F90132964591FF
:10A910005491C12CD12CB2E0BA1768F5F901EB0FB4
:10A92000F11DEB0FF11DA590B4906501F901FF2415
:10A93000F394FB0EEF0DF11DBE5FEF0DF11DE590E1
:10A94000F4908E149F04A4F49A01261B370BD801AF
:10A95000AA19BB090F94A50D9A012E193F09442786
:10A9600037FD4095542F0F94830D200F311F08C0E1
:10A97000A7018501D1CFCD82DE824BC00F94830D1C
:10A980003E832D8346C0223639F0E0900D04F090CE
:10A990000E04ADE0B4E006C0E0908903F0908A03B5
:10A9A000A9E8B3E012964D915C91139722E01496BA
:10A9B0000D911C9115972E5F1696ED91FC911797AE
:10A9C000E815F905D4F49A01261B370BD701A01B13
:10A9D000B10B0CEF1FE00E191F090F94A50D9A0182
:10A9E0002E1B3F0B442737FD4095542F0F94830DAA
:10A9F000020F131F1E830D830CC01496223419F00E
:10AA0000AF017801D4CF8CEF9FE0801B910B9E8328
:10AA10008D83DF91CF911F910F91FF90EF90DF9089
:10AA2000CF90BF90AF909F908F9008959F92AF92DC
:10AA3000BF92CF92DF92EF92FF920F931F93CF932B
:10AA4000DF936B017C01042F922EE0910A02F091BA
:10AA50000B02C1E020E030E040E751E463857485FB
:10AA6000858596850F94E30B18160CF0C0E011E075
:10AA70001C2720E030E041E953E4C701B6010F9400
:10AA8000E30B18166CF020E030E0A901C701B60115
:10AA90000F94AF0987FF0AC0C12CD12C760106C0E4
:10AAA000C12CD12C91E9E92E93E4F92EC02FD0E0EE
:10AAB000FE01EE0FFF1FE65FFD4FA080B180F501A4
:10AAC0008181811103C0C12CD12C7601B701A6016F
:10AAD000C50158DE992081F020E030E040EF51E4DC
:10AAE000C701B6010F94E30B181634F4F501E05CCE
:10AAF000FF4F80818160808320E030E040E252E4BB
:10AB0000C701B6010F94E30B87FD0EC023E82C9F0D
:10AB1000C0012D9F900D1124855A9D4FFC01E458D2
:10AB2000FF4F208131962083602F70E080E090E01D
:10AB30000F94800AAB01BC0120E084E292E20E9403
:10AB4000DAA120E0B701A60188E294E20E949DA16B
:10AB5000E0910A02F0910B0220E030E040E751E47E
:10AB600063857485858596850F94E30B18167CF0B4
:10AB7000111119C0DF91CF911F910F91FF90EF90AC
:10AB8000DF90CF90BF90AF909F900C9475D611231B
:10AB900051F00F94E6036093E3067093E40680930C
:10ABA000E5069093E606DF91CF911F910F91FF90FC
:10ABB000EF90DF90CF90BF90AF909F900895CF928D
:10ABC000DF92EF92FF92CF936B017C01C42F20E0C4
:10ABD00030E040EF52E40F94E30B18166CF020E0E5
:10ABE00030E0A901C701B6010F94AF0987FF0AC081
:10ABF000C12CD12C760106C0C12CD12C20EFE22E25
:10AC000022E4F22EA70196016091190270911A02B6
:10AC100080911B0290911C020F94AF09882341F18F
:10AC2000B701A6018EE092E0ADDDCC2379F020E003
:10AC300030E040EF51E4C701B6010F94E30B181662
:10AC40002CF480914E02816080934E024091190253
:10AC500050911A0260911B0270911C0220E089E160
:10AC600092E2CF91FF90EF90DF90CF900C949DA156
:10AC7000CF91FF90EF90DF90CF900895E0910A027E
:10AC8000F0910B021682158213861486158616869D
:10AC9000E081F0E0E958F24E1082E0910C02F09170
:10ACA0000D02168215821386148615861686E0819B
:10ACB000F0E0E958F24E10828FEF8093DE020895A3
:10ACC0002F923F924F925F926F927F928F929F92BC
:10ACD000AF92BF92CF92DF92EF92FF920F931F93AA
:10ACE000CF93DF93CDB7DEB7E5970FB6F894DEBF0D
:10ACF0000FBECDBF9DAB8CAB4E8B5F8B688F798FBA
:10AD00002E8F0BAB0F94E6036A8F7B8F8C8F9D8FFA
:10AD1000ACA9BDA996968C9190E0959587952C014C
:10AD2000662457FC6094762C86E092E20E94B59FE0
:10AD3000A5DFBE8DB093DE02ACA9BDA9EC91F0E019
:10AD4000E958F24E96968C918083BE8DB11104C065
:10AD50008091D7028093D802530142012A8D3B8D06
:10AD60004C8D5D8D2BA33CA34DA35EA32F8F38A3E9
:10AD700049A35AA319821F8630EA388B41E4498BD4
:10AD80001A8A1B8A50EA5C8B81E48D8B1BA61CA659
:10AD90001DA61EA61FA218A619A61AA6C12CD12C44
:10ADA00076011FA618AA19AA1AAA91E099871E86E9
:10ADB0001D86A8958CA99DA9DFDAACA9BDA9179617
:10ADC0003C90179718960C91189719961C91199703
:10ADD0001A962C900F94E6036D837E838F83988759
:10ADE000232D302F412F522D6A897B898C899D8993
:10ADF0000F94AF0987FF04C03A8A0B8B1C8B2D8AF6
:10AE0000232D302F412F522D69817F858889998983
:10AE10000F94AF0987FD04C039820F87188B298AE8
:10AE2000B985BB2309F449C02E893F89488D598DC6
:10AE3000632D702F812F922D0F94E30B18160CF0B9
:10AE400086C08D819E81AF81B8852BA13CA14DA18B
:10AE50005EA1821B930BA40BB50B3E8D311105C077
:10AE600044EC59E060E070E004C04CED55E060E077
:10AE700070E0481759076A077B0708F068C0ECA91B
:10AE8000FDA92081E22FF0E0E958F24E242D281987
:10AE900020838FA798ABA9ABBAABFE89FA8B2F8919
:10AEA0002B8B388D3C8B498D4D8B8D819E81AF8155
:10AEB000B8858F8F98A3A9A3BAA32E893F89488DFF
:10AEC000598D632D702F812F922D0F94AF0987FF1D
:10AED00011C28D819E81AF81B8852F8D38A149A186
:10AEE0005AA1821B930BA40BB50B3E8D3111EFC001
:10AEF00048E853E160E070E0481759076A077B07AC
:10AF000008F0F8C14D855E85452B09F0E5C0ACA978
:10AF1000BDA9EC91F0E0E958F24E882D840D8083B4
:10AF2000ED85FE853196FE87ED87FE89F9832F89B1
:10AF30002F87388D388B498D498B8D819E81AF81CC
:10AF4000B8858BA39CA3ADA3BEA391E0998720E015
:10AF500030E040E252E46E897F89888D998D0F94AC
:10AF60004B099B01AC01632D702F812F922D0F9403
:10AF7000E30B18161CF487E991E23BC08D819E819A
:10AF8000AF81B8852A8D3B8D4C8D5D8D821B930BD7
:10AF9000A40BB50B893E9340A105B10558F080E0A4
:10AFA0000E94E3238D819E81AF81B8858A8F9B8F1C
:10AFB000AC8FBD8F8D819E81AF81B885880F991F21
:10AFC000AA1FBB1F2BA13CA14DA15EA1821B930B0D
:10AFD000A40BB50B2F8D38A149A15AA1821B930B4D
:10AFE000A40BB50B81389F44A241B105E8F08AE774
:10AFF00091E20E94BF9FE5960FB6F894DEBF0FBEA8
:10B00000CDBFDF91CF911F910F91FF90EF90DF9017
:10B01000CF90BF90AF909F908F907F906F905F90F8
:10B020004F903F902F902ACE4D855E85463051053A
:10B030000CF443C08FE191E20E94B59F1FDE5BA933
:10B04000552309F459C1ACA9BDA95A96CD92DD92F8
:10B05000ED92FC925D972FA138A549A55AA55E9661
:10B060002D933D934D935C9391972BA53CA54DA5B6
:10B070005EA592962D933D934D935C93959781E0B9
:10B0800053968C9380E0E5960FB6F894DEBF0FBE22
:10B09000CDBFDF91CF911F910F91FF90EF90DF9087
:10B0A000CF90BF90AF909F908F907F906F905F9068
:10B0B0004F903F902F900C9457CF8CE69AE00E94CF
:10B0C00074CA61E08CE69AE00E9475CA72CE48EBC1
:10B0D0005BE060E070E010CF2FA538A949A95AA91C
:10B0E000280F391F4A1F5B1F29873A874B875C87C8
:10B0F0002FA538A949A95AA9281B390B4A0B5B0B64
:10B10000CA01B901A50194010F941E0D29853A8544
:10B110004B855C850F94830D240D351D461D571DF1
:10B120002431310541055105A4F0ACA9BDA996967D
:10B130008C9190E04497AA2797FDA095BA2F2901FA
:10B140003A0182179307A407B50744F42C013D0187
:10B1500005C044E1442E512C612C712CECA9FDA9B1
:10B1600026A1822F869590E0A0E0B0E08415950599
:10B17000A605B7056CF4822F90E001974C01AA2434
:10B1800097FCA094BA2C84189508A608B70802C0AA
:10B1900053014201B301A2018EEF91E20E94A9A0E6
:10B1A000B501A40189EF91E20E94A9A022E04981A2
:10B1B0005F856889798982EF91E20E94DAA122E0B5
:10B1C0004A895B896C897D898BEE91E20E949DA101
:10B1D0002D853E85233031050CF499CEC501B4018F
:10B1E0000F94820A20E030E040E850E40F94570CBE
:10B1F0006B017C0129813F85488959896A897B894E
:10B200008C899D890F944A0920ED3FE049E450E480
:10B210000F94570C9B01AC01C701B6010F94B609FE
:10B220006B017C0169857A858B859C850F94820AE8
:10B2300020E030E04AE754E40F94B60969837A834A
:10B240008B839C8322E0B701A60185EE91E20E94E8
:10B25000DAA122E049815A816B817C818FED91E2F4
:10B260000E949DA12AE939E949E15FE3C701B601DE
:10B270000F94570C6B017C019B01AC010F944B099F
:10B2800029813A814B815C810F94B6096FA378A71D
:10B2900089A79AA729813A814B815C81C701B601B0
:10B2A0000F94570C20E030E040E05EE30F94570C21
:10B2B0006BA77CA78DA79EA782ED91E20E949E9F1F
:10B2C00022E0B701A6018CEC91E20E949DA122E050
:10B2D0004FA158A569A57AA586EC91E20E949DA18F
:10B2E00022E04BA55CA56DA57EA580EC91E20E94B5
:10B2F0009DA10DCE19862BCEE5960FB6F894DEBF34
:10B300000FBECDBFDF91CF911F910F91FF90EF90B6
:10B31000DF90CF90BF90AF909F908F907F906F9075
:10B320005F904F903F902F900895CF93DF930F94AD
:10B33000E603AB01BC0188E191E20E94A9A0E09183
:10B34000E002F0E0EE0FFF1FE65FFD4FC081D1810C
:10B350004F81588569857A8522E085EB93E20E94CA
:10B36000DAA14B855C856D857E8520E085EB93E2D7
:10B370000E94DAA1E881F0E0E958F24E608170E0C5
:10B3800085EB93E2DF91CF910C9483A08091BE076F
:10B3900082FF3CC060E070E083E091E20E9477A011
:10B3A000E0910A02F0910B02678170858185928598
:10B3B0000F944F0A605171096D31714018F484EE99
:10B3C00090E202C08EEE90E20E949E9F8DE091E29C
:10B3D0000E94859FE0910C02F0910D0267817085BB
:10B3E000818592850F944F0A605171096D317140CA
:10B3F00018F08EEE90E202C084EE90E20E949E9FD2
:10B4000087EB90E20E94BF9F81E0089580E008955D
:10B410002F923F924F925F926F927F928F929F9264
:10B42000AF92BF92CF92DF92EF92FF920F931F9352
:10B43000CF93DF93CDB7DEB72B970FB6F894DEBF6F
:10B440000FBECDBFA8950F94E60369837A838B83E3
:10B450009C832AE032E03B872A8748ED52E05F83F5
:10B460004E8352E35987212C1D82AA85BB850D91FD
:10B470001D91BB87AA87211027C020E030E040E261
:10B4800052E4F80167817085818592850F94AF0938
:10B4900087FF13C020E030E040E252E4D8011B9661
:10B4A0006D917D918D919C911E970F94AF0987FFAF
:10B4B00004C0EE81FF81108207C0EE81FF813197C9
:10B4C0008081AE81BF818C938091DE02281609F4C1
:10B4D000B8C2C8010E94BC518091BE0782FD26C03F
:10B4E000F801C780D084E184F28420E030E040E8B5
:10B4F00051E4C701B6010F94AF0987FD0AC020E0EF
:10B5000030E046E953E4C701B6010F94E30B181687
:10B510006CF4809188038F5F809388038B3008F4EC
:10B52000C3C20E94CD4D32DFF1E0FD838091BE07A2
:10B5300082FD87C233243394D8011B962D913D910F
:10B540004D915C911E9717966D917D918D919C9177
:10B550001A970F94E30B87FD312CB1E03B2641F4A1
:10B560007801E0E4EE0EF11CD7018C9180FD9FC2C2
:10B57000C980DA80EB80FC80F801E75BFF4F4080F8
:10B580005180628073805801B1E4AB0EB11CF501AB
:10B5900080819181A281B381A7019601281B390B7B
:10B5A0004A0B5B0B421653066406750608F068C02A
:10B5B000480130E4830E911CD401BC91B8878B2FD5
:10B5C000867009F45DC08091BD0786FF59C0B885BB
:10B5D000B1FF81C27801E5E4EE0EF11CD7012D9197
:10B5E0003D914D915C91F8016781708581859285CF
:10B5F0000F944A0920E030E040E85FE30F94AF0980
:10B6000087FF5EC2809188038F5F809388038B30B1
:10B61000A8F10E94CD4D41E069E978E18CE69AE01D
:10B620000E9494AB82E598E10E94BF9FD7012D91C3
:10B630003D914D915C91F80167817085818592857E
:10B640000F944A09AB01BC0122E08CEE9DE00E9400
:10B65000DAA149815A816B817C81F50180819181D8
:10B66000A281B381481B590B6A0B7B0B84EE9DE0D2
:10B670000E94A9A080EE9DE00E949E9FF1E0FD83C4
:10B68000F80187A5C780D084E184F28424E0829FFA
:10B69000E00DF11D1124C0AAD1AAE2AAF3AA8F5F7E
:10B6A0008370D8019F968C939F9753968C91539754
:10B6B000813009F0CAC01B968D909D90AD90BC90D2
:10B6C0001E9720E030E040EA51E4C501B4010F9438
:10B6D000AF0987FDCCC0A7019601C501B4010F9445
:10B6E0004A094B015C0120E030E040EA51E40F944C
:10B6F000E30B18161CF4F801F6A0D3C020E030E0EC
:10B7000040EA51ECC501B4010F94AF0987FDDAC0DE
:10B71000BE016F5F7F4FC8010E947B4DD8015A96D2
:10B720002D913D914D915C915D97C501B4010F94B0
:10B73000570C6B017C01F8012489358946895789AA
:10B74000C501B4010F944B094B015C01D8019B96D4
:10B750005C909B979C966C909C979D967C909D97F7
:10B760009E964C90252D362D472D542D0F94AF09C4
:10B7700087FD13C0F80157A060A471A442A4252D31
:10B78000362D472D542DB401C5010F94E30B181627
:10B7900024F0582C692C7A2C4B2C852D962DA72D16
:10B7A000B42DF801848B958BA68BB78B268D378DA6
:10B7B00040A151A1652D762D872D942D0F94570C06
:10B7C0002DEC3CEC4CEC5DE30F94570C9B01AC0171
:10B7D000C701B6010F944B096B017C01D8019F96FC
:10B7E0008C91F801B4E08B9FE00DF11D1124D8017C
:10B7F00017962D913D914D915C911A9760A971A971
:10B8000082A993A90F944A09F80122A133A144A166
:10B8100055A10F94570C2FED3FE445E550E40F94EC
:10B82000570C9B01AC01C701B6010F944B090F9453
:10B830004F0A77FD47C0D80196962C9130E0261725
:10B8400037070CF4B901F62E98C0833009F09CC07C
:10B85000F80183849484A584B68420E030E040EA33
:10B8600051E4C501B4010F94AF0987FF07C0F80187
:10B87000E05CFF4F8081897F808324C0A70196010F
:10B88000C501B4010F944A096B017C0120E030E04E
:10B8900040EA51E40F94E30B181654F4D80196963D
:10B8A000FC90BE016F5F7F4FC8010E94514D65C083
:10B8B00020E030E040EA51ECC701B6010F94AF0937
:10B8C00087FF02C0F12C59C0BE016F5F7F4FC801D6
:10B8D0000E947B4DF801C780D084E184F28420E08F
:10B8E00030E040E450E464897589868997890F9433
:10B8F000570C4B015C01D8019F968C91F801B4E084
:10B900008B9FE00DF11D112420A931A942A953A953
:10B91000C701B6010F944A092FED3FE445E550E415
:10B920000F94570C9B01AC01C501B4010F944B0956
:10B9300020E030E040E85EE30F94570CF801648BA0
:10B94000758B868B978B228D338D448D558D0F94FF
:10B95000570C9B01AC01C701B6010F944B09D801EC
:10B960001B962D913D914D915C911E970F94E30B89
:10B9700018160CF4A7CFF801F08CD801EC91F0E088
:10B98000E958F24EF0823DC0823021F589819A81DA
:10B99000AB81BC81F80147855089618972896C014E
:10B9A0007D01C41AD50AE60AF70A29E8C21623E17E
:10B9B000D206E104F10428F12081E22FF0E0E958F9
:10B9C000F24E232D21952083F8018787908BA18B40
:10B9D000B28B08C0D801EC91F0E0E958F24E832D0B
:10B9E00081958083332039F0BE016F5F7F4FC8019E
:10B9F0000E94514D06C0F801E05CFF4F8081897FB5
:10BA0000808320E030E041E953E4F80167817085EC
:10BA1000818592850F94E30B181634F4D801EC91CC
:10BA2000F0E0E958F24E10828091860390918703EE
:10BA30008B960817190729F4332011F02F9A01C0AB
:10BA40002F982394B985BE5CB987EE81FF81ED57AD
:10BA5000FF4FFF83EE83F2E02F1207CDCD80C110A0
:10BA600007C080918803882319F081508093880350
:10BA70008091BE0782FF88C0E0910A02F0910B021C
:10BA8000E081F0E0E958F24E1082E0910C02F09172
:10BA90000D02E081F0E0E958F24E10828091EA0256
:10BAA00088608093EA0270C021E02D833FCD63E07F
:10BAB00089850E94B0A2D7018C918E7F8C9358CD3E
:10BAC0008885897FD4018C93BE016F5F7F4FC80149
:10BAD0000E94514DD5CDF801238534854585568585
:10BAE00067817085818592850F944A099F7720E050
:10BAF00030E040EA51E40F94E30B1816A4F580916E
:10BB000088038F5F809388038B3008F4B7CD0E9441
:10BB1000CD4D41E069E978E18CE69AE00E9494AB72
:10BB200082E598E10E94BF9FF801EB5BFF4F4081E7
:10BB300051816281738122E08EEB9DE00E94DAA147
:10BB4000D80117964D915D916D917C911A9722E0E5
:10BB500083EB9DE00E94DAA18BEA9DE00E949E9F0C
:10BB6000B1E0BD838DCDE8EECE0EE3E0DE1EE11C3C
:10BB7000F11CC418D508E608F708D501CD92DD926E
:10BB8000ED92FC9213977CCD2B960FB6F894DEBF06
:10BB90000FBECDBFDF91CF911F910F91FF90EF901E
:10BBA000DF90CF90BF90AF909F908F907F906F90DD
:10BBB0005F904F903F902F9008958FEF8EBD0DB402
:10BBC00007FEFDCF8EB50895DC01680F791F80E078
:10BBD00090E0A617B70779F02D91E92FFF27E2270C
:10BBE000EE0FFF1FEE51FD4E25913491982F8827BF
:10BBF00082279327EECF089522E090E0281728F4BB
:10BC0000963019F0220F9F5FF9CF209A289A219A37
:10BC1000229A2398809164008B7F80936400892FFF
:10BC2000806A86958CBD90FD03C081E0963009F452
:10BC300080E08DBD08958EBD0DB407FEFDCF089543
:10BC4000CF93FB0120E030E22F5F31932B30E1F7FF
:10BC5000DC0190E037E02A2FEB2F8D9181110AC093
:10BC6000DA012C931196EC9381E0FB0190819032E4
:10BC700041F526C08F32A1F3282F8E3219F0E2EE63
:10BC8000F4E108C03A30E1F098E03AE0E4CF3196D0
:10BC9000C817B1F0C491C111FACF391718F080520A
:10BCA0008F3508F02FE581E0890FFB01E90FF11DC9
:10BCB0009FE9920F9A3108F420522083982FCBCF1E
:10BCC00080E0CF9108959B01255F3F4F80E0FB010D
:10BCD0009191BF01482F4695F0E88F9F400D1124A8
:10BCE000842F890F6217730791F7089561E0FC01B3
:10BCF00080810F9433058FEF9ECFCF93DF93EC01BC
:10BD00008A817ADF60E08881DF91CF910D943305DD
:10BD1000CF92DF92EF92FF920F931F93CF93DF9317
:10BD2000EC018B017A010F94E6036B0146DF8B83F4
:10BD30008F3F49F40F94E6036C197D096D32714011
:10BD4000A8F381E131C08E3F11F08FE02DC0E114E6
:10BD5000F104D9F0C70101972FEF2EBDF8014FEF85
:10BD60009F01201B310B2817390738F40DB407FE4B
:10BD7000FDCF2EB521934EBDF3CF0DB407FEFDCF01
:10BD80002EB5F801E80FF91F20831B8216DFD82E8D
:10BD900014DFC82EB701C80117DF2C2D30E03D2974
:10BDA0002817390731F08BE18983CE019FDF80E0CE
:10BDB00003C0CE019BDF81E0DF91CF911F910F91F6
:10BDC000FF90EF90DF90CF9008950F931F93CF9344
:10BDD000DF931F921F92CDB7DEB78C0169837A8300
:10BDE0008CDF40E052E069817A81C8010F900F90AA
:10BDF000DF91CF911F910F918BCF0F931F93CF9313
:10BE0000DF93EB010F94E6038B01D7DE8F3F49F000
:10BE10000F94E603601B710B6C177D07B0F380E095
:10BE200001C081E0DF91CF911F910F910895BF92E2
:10BE3000CF92DF92EF92FF920F931F93CF93DF93F6
:10BE4000CDB7DEB72A970FB6F894DEBF0FBECDBFD1
:10BE50008C01B62E2F83388749875A874EDF6CE2D4
:10BE600071E0C801CADFFE01319686E0DF011D9254
:10BE70008A95E9F78B2D806489838A858A838985F1
:10BE80008B8388858C838F818D83CE010696DF011D
:10BE900020E059E04D9138E0220F642F622767FDC2
:10BEA0002527440F3150C1F7A817B90799F7220F7A
:10BEB00021602E837F016E01B7E0CB0ED11CF7010C
:10BEC00081917F01B8DEEC14FD04C9F7FCE0BF12DC
:10BED00001C073DEF12C71DED80113968C9387FFBD
:10BEE00005C0BFEFFB1611F0F394F5CF2A960FB6FD
:10BEF000F894DEBF0FBECDBFDF91CF911F910F91A0
:10BF0000FF90EF90DF90CF90BF900895BF92CF92B7
:10BF1000DF92EF92FF920F931F93CF93DF93EC0189
:10BF2000B62E1C82198248830F94E6038B0161E0D0
:10BF300088810F94FA0461E088810F943305239877
:10BF4000229A219A209A8BE08A8356DEE4E1FE2E23
:10BF50008FEF71DEFA94E1F720E030E0A90160E0B4
:10BF6000CE0165DF813049F00F94E603601B710B51
:10BF7000613D774088F381E057C021E030E040E048
:10BF800050E06BE3CE0153DF813011F08AE14CC009
:10BF90002AEA31E040E050E068E0CE0148DF853039
:10BFA00011F481E009C074E0F72E07DE8B83FA9468
:10BFB000E1F78A3A59F482E08C838C81823079F4FB
:10BFC000C12CD12CE12C60E4F62E0CC00F94E603BA
:10BFD000601B710B613D7740D8F282E025C0C12C17
:10BFE000D12C760120E030E0A90167E3CE011FDF0C
:10BFF000A701960169E2CE011ADF882349F00F9468
:10C00000E603601B710B613D774060F38AE00CC072
:10C010008C818230B1F420E030E0A9016AE3CE01E6
:10C0200006DF882329F088E08983CE015FDE14C013
:10C03000C4DD807C803C11F483E08C83BEDDBDDDFB
:10C04000BCDDCE0153DE8EE08B1518F488E18983C8
:10C0500003C0BA8281E001C080E0DF91CF911F91DF
:10C060000F91FF90EF90DF90CF90BF9008950F93C6
:10C070001F93CF93DF93EC0189018C81833039F0DA
:10C08000F9E0440F551F661F771FFA95D1F79A0103
:10C09000AB0161E1CE01CBDE811109C040E052E08D
:10C0A000B801CE01DF91CF911F910F9131CE84E085
:10C0B0008983CE011BDE80E0DF91CF911F910F912C
:10C0C0000895CF93DF93EC018C81833039F089E0C0
:10C0D000440F551F661F771F8A95D1F79A01AB0150
:10C0E00062E1CE01A4DE882331F085E08983CE01B0
:10C0F000FDDD80E003C0CE01F9DD81E0DF91CF916D
:10C100000895CF93DF93EC01F8DD20E030E0A90142
:10C110006CE0CE018CDE882331F083E08983CE0190
:10C12000E5DD80E003C0CE01E1DD81E0DF91CF916C
:10C130000895CF92DF92EF92FF920F931F93CF93C8
:10C14000DF931F92CDB7DEB78C01E62E6A0160E067
:10C1500072E0CA0139DDF82E8E2D99836CDDF6016F
:10C1600080818EBD418122E030E099810DB407FECF
:10C17000FDCF4EBD2115F2E03F0739F0F601E20F89
:10C18000F31F40812F5F3F4FF1CF0DB407FEFDCF6E
:10C19000892F51DD8F2D4FDD10DDF80183838F71E5
:10C1A000853031F083E18183C801A0DD80E001C0EA
:10C1B00081E00F90DF91CF911F910F91FF90EF9051
:10C1C000DF90CF9008950F931F93CF93DF93EC01EF
:10C1D00089018C81833039F039E0440F551F661F87
:10C1E000771F3A95D1F79A01AB0168E1CE011FDEC6
:10C1F000882311F086E01EC0A8016EEFCE0199DF02
:10C200008823C9F068E572E0CE01F7DD182F8111AF
:10C2100002C087E10FC020E030E0A9016DE0CE014F
:10C2200006DE811106C0C9DC811103C0CE015EDDCE
:10C2300005C086E18983CE0159DD10E0812FDF91B1
:10C24000CF911F910F9108950F931F93CF93DF9379
:10C25000EC018B0152DD68E572E0CE01CEDD882372
:10C2600051F0A8016CEFCE0164DF182F882319F07C
:10C27000CE013CDD05C085E18983CE0137DD10E0CC
:10C28000812FDF91CF911F910F9108958F929F92EF
:10C29000AF92BF92CF92DF92EF92FF920F931F93D4
:10C2A000CF93DF93EC016A017B014801590120E043
:10C2B00030E0A90167E3BBDDA501940167E1CE0190
:10C2C000B6DD882311F089E012C08C81833039F00B
:10C2D00049E0CC0CDD1CEE1CFF1C4A95D1F7A701F0
:10C2E000960169E1CE01A3DD882331F087E08983DF
:10C2F000CE01FCDC80E003C0CE01F8DC81E0DF9100
:10C30000CF911F910F91FF90EF90DF90CF90BF9052
:10C31000AF909F908F9008951F93CF93DF93EC0180
:10C32000ECDC68E572E0CE0168DD882361F08DEF1A
:10C3300082DC68E572E0CE0160DD182F882319F0F9
:10C34000CE01D4DC05C082E18983CE01CFDC10E0D0
:10C35000812FDF91CF911F9108950F931F93CF935A
:10C360008091A50480FF41C04091A6045091A7048C
:10C370006091A8047091A9042AEA34E080919F0496
:10C380009091A00420DFC82F811102C0C0E02EC010
:10C390008091A50481FD06C08091A5048E7F8093C5
:10C3A000A50424C00091A1041091A2042091A3042B
:10C3B0003091A404011511052105310569F340915F
:10C3C000A6045091A7046091A8047091A904400F9D
:10C3D000511F621F731F2AEA34E080919F049091DD
:10C3E000A004F1DE8111D8CFD1CFC1E08C2FCF9145
:10C3F0001F910F910895CF92DF92EF92FF92CF930A
:10C400006B017C01C42F8091A6049091A704A09198
:10C41000A804B091A9048C159D05AE05BF05F9F0DF
:10C420009CDF811103C080E090E021C0C2FF0BC0FF
:10C430001092A504C092A604D092A704E092A8048A
:10C44000F092A9040CC02AEA34E0B701A601809159
:10C450009F049091A0040BDE8111EACFE4CFC3705A
:10C460008091A5048C2B8093A5048AEA94E0CF9157
:10C47000FF90EF90DF90CF900895CF93DF93EC0182
:10C48000462F6F85788989899A89B5DF009739F0B9
:10C490002C8130E2239F800D911D112402C080E089
:10C4A00090E0DF91CF9108950F931F93CF93DF9387
:10C4B000EC018B818823D1F1898187FF32C061E053
:10C4C000CE01DBDF8C01009789F1FC018081853E84
:10C4D00069F18B81823040F44B895C896D897E895A
:10C4E000448F558F668F778F4F89588D698D7A8DE0
:10C4F000F801538F428F758B648BE091AA06F091FF
:10C50000AB06309759F0B8016A5E7F4FC801489674
:10C510001995F801808D918D938B828B89818F770E
:10C520008983DF91CF911F910F9117CF81E088838D
:10C5300080E0DF91CF911F910F910895CF93DF930A
:10C54000EC01B2DF1B82DF91CF9108958FEF9FEF57
:10C55000DC018093A6049093A704A093A804B09351
:10C56000A9041092A50408958F929F92AF92BF9252
:10C57000CF92DF92EF92FF920F931F93CF93DF93AF
:10C58000EC016A017B0189014230510561057105A9
:10C5900008F454C089859A85AB85BC850196A11D98
:10C5A000B11D84179507A607B70708F447C08F8900
:10C5B000803129F49927872F762F652F0BC0803281
:10C5C000E9F5CB01BA0127E09695879577956795B0
:10C5D0002A95D1F78B889C88AD88BE88680D791D17
:10C5E0008A1D9B1D42E007DF009741F12F89203112
:10C5F00069F4DD24EE24FF24F601EE0FFF1FE80F9F
:10C60000F91F80819181A0E0B0E011C0E894C7F8E3
:10C61000DD24EE24FF24F601EE0FFF1FEE0FFF1FB7
:10C62000E80FF91F80819181A281B381BF70F80169
:10C6300080839183A283B38381E001C080E0DF9196
:10C64000CF911F910F91FF90EF90DF90CF90BF900F
:10C65000AF909F908F9008952F923F924F925F924C
:10C660007F928F929F92AF92BF92CF92DF92EF9282
:10C67000FF920F931F93CF93DF93EC017B016A012D
:10C680008B81811103C08FEF9FEF17C1898180FFDC
:10C69000FACF4B895C896D897E898B859C85AD85B8
:10C6A000BE854601A12CB12C8A019B01081B190BE8
:10C6B0002A0B3B0B80169106A206B30618F06A01FE
:10C6C000C81AD90A86014E0127E0820E911C011575
:10C6D000110509F46EC02B843C844D845E845101A5
:10C6E00081E0B8228D819E81B201A101E9E07695B9
:10C6F000679557954795EA95D1F7FC0174807A9430
:10C7000074222B81223049F4228C338C448C558C3A
:10C71000240E351E461E571E37C0A114B104C1F4A5
:10C72000711016C023282428252849F48F89988D54
:10C73000A98DBA8D8F839887A987BA8709C04F8141
:10C74000588569857A8594010FDF882309F49BCF8A
:10C75000ED81FE81A4812F81388549855A8522503B
:10C76000310941095109B0E00F94C00D1B012C01A2
:10C7700086859785A089B189280E391E4A1E5B1EC1
:10C78000270C311C411C511CA114B104A1F401154A
:10C79000F2E01F0780F08091A6049091A704A09179
:10C7A000A804B091A904281639064A065B06D9F4F4
:10C7B00002C0C60182C040E0C201B1011CDE009788
:10C7C00009F461CF20E032E02A193B092801201743
:10C7D000310708F42901BC016A0D7B1DA201C701C4
:10C7E0000F94C8112AC00115E4E01E07B8F1B12E5C
:10C7F000B6942B81223009F040C0281639064A062B
:10C800005B0608F043C0B201A10180919F049091A2
:10C81000A00457DC882309F436CF1701412C8091FE
:10C820009F049091A0044B103BC06BDC882309F45B
:10C830002ACF512C542C4424550CE40CF51C8B8528
:10C840009C85AD85BE85840D951DA11DB11D8B8771
:10C850009C87AD87BE870419150939CF9701B201AE
:10C86000A10180919F049091A00401DC882309F428
:10C870000ACF412C42E0542EE0CFED81FE8124818D
:10C8800027192B1508F0B9CFB22EB7CF8B0D911DFC
:10C89000A11DB11D281639064A065B0650F0B3CF1C
:10C8A000B10193DA2EEF321A882309F4ECCE4394C7
:10C8B000B6CF53DD8111A7CFE6CEDF91CF911F9187
:10C8C0000F91FF90EF90DF90CF90BF90AF909F902F
:10C8D0008F907F905F904F903F902F900895CF93CF
:10C8E000DF931F92CDB7DEB741E050E0BE016F5F2E
:10C8F0007F4FB2DE019719F4898190E002C08FEF7B
:10C900009FEF0F90DF91CF9108951F93CF93DF9307
:10C91000EC018B81823018F480E090E023C04B85DD
:10C920005C856D857E85A5E07695679557954795DD
:10C93000AA95D1F7142F1F70CE01D1DF97FDECCF50
:10C940004B855C856D857E85415E5F4F6F4F7F4F68
:10C950004B875C876D877E8720E2129FC001112480
:10C9600086559B4FDF91CF911F910895AF92BF9253
:10C97000CF92DF92EF92FF920F931F93CF93DF93AB
:10C980001F92CDB7DEB77C018A014115510511F028
:10C99000DA011C9241E0BDE0CB2EA895C701498386
:10C9A000B4DF5C014981009709F47AC0FC01208161
:10C9B000222309F475C0253009F467C0253E09F427
:10C9C00064C0FC018385982F9F739F3009F054C089
:10C9D0000115110511F3828D938D892BF1F62F71BD
:10C9E000E1F22330D4F6332727FD30952150310969
:10C9F000C29EF001C39EF00D1124E00FF11FD5017E
:10CA000011968C911197808313968C911397818343
:10CA100015968C911597828317968C91179783831F
:10CA200019968C91199784831E968C911E978583F5
:10CA300050968C915097868352968C91529787830B
:10CA400054968C915497808756968C9156978187EF
:10CA500058968C91589782875C968C915C978387C7
:10CA60005E968C915E978487442309F496CF1D9639
:10CA7000DC90158640E091CF982F967031F42E32DD
:10CA800061F4F50191819E3241F00115110511F417
:10CA900041E083CFD8011C92FBCF83FD7ECF03C042
:10CAA00080E090E011C00115110569F0411105C049
:10CAB000B501C70108D9D81631F0A501B80188E140
:10CAC00099E00E94639DC5010F90DF91CF911F9166
:10CAD0000F91FF90EF90DF90CF90BF90AF900895AF
:10CAE0004F925F926F927F92AF92BF92CF92DF92FE
:10CAF000EF92FF920F931F93CF93DF93EC016A01A4
:10CB00007B012B81222349F08B899C89AD89BE89C9
:10CB100084179507A607B70710F480E073C022308A
:10CB200049F4CB86DC86ED86FE861F821886198640
:10CB30001A8667C0C114D104E104F10449F41F82CC
:10CB4000188619861A861B861C861D861E8659C065
:10CB50008B859C85AD85BE85ED81FE81E585F0E008
:10CB60003996AC01BD0141505109610971090E2E80
:10CB700004C076956795579547950A94D2F7970123
:10CB80008601015011092109310904C03695279504
:10CB900017950795EA95D2F7041715072607370763
:10CBA00020F0892B8A2B8B2B49F48F89988DA98DA6
:10CBB000BA8D8F839887A987BA8704C0041B150B89
:10CBC000260B370B280139015E0187E0A80EB11C46
:10CBD000411451046104710481F04F8158856985C5
:10CBE0007A8595018D819E81BFDC91E0491A5108BB
:10CBF000610871088111ECCF05C0CB86DC86ED861B
:10CC0000FE8681E0DF91CF911F910F91FF90EF9011
:10CC1000DF90CF90BF90AF907F906F905F904F90DC
:10CC2000089540E050E0BA015BCFAF92BF92CF923F
:10CC3000DF92EF92FF920F931F93CF93DF936C01DC
:10CC4000A42E7901E801FC018381823008F43DC003
:10CC5000C601E7DFB12CA895C60157DE0097B9F1F0
:10CC6000FC012081222399F1253011F0253E91F716
:10CC7000FC0183858F738F3031F1209721F11A14D5
:10CC800014F5BA1404F1088119812A813B81012B22
:10CC9000022B032BC1F4F60183859485A585B68507
:10CCA0008097A109B109FB2D40E2F4029001112403
:10CCB000821B930BA109B10988839983AA83BB8343
:10CCC000F701B08202C0B394C6CF81E001C080E01A
:10CCD000DF91CF911F910F91FF90EF90DF90CF9058
:10CCE000BF90AF900895AF92BF92CF92DF92EF9234
:10CCF000FF920F931F93CF93DF9300D01F92CDB776
:10CD0000DEB78C01FC018789908DA18DB28D89835E
:10CD10009A83AB83BC83A12CB12C49815A816B814E
:10CD20007C819E012F5F3F4FD80115968D919C917C
:10CD300016971ADC8823C1F1D8011596ED91FC9164
:10CD400016978481A80EB11CA114B0E1BB0658F55A
:10CD5000C980DA80EB80FC808789803149F481E0EA
:10CD6000E8EFCE16EFEFDE06E104F10450F4D5CF84
:10CD700081E0F8EFCF16FFEFDF06EF06FFE0FF06DA
:10CD800060F2A50160E070E099E0440F551F661F56
:10CD9000771F9A95D1F7D80153964D935D936D9374
:10CDA0007C93569701C080E00F900F900F900F90EA
:10CDB000DF91CF911F910F91FF90EF90DF90CF9077
:10CDC000BF90AF900895CF93DF93EC01FB018B816F
:10CDD000882311F080E03BC07E836D83878980319A
:10CDE00001F18032B9F783E08B83428D538D648DDE
:10CDF000758D4F8B588F698F7A8FCE0174DF8823A2
:10CE000049F381E089831F82188619861A861B865A
:10CE10001C861D861E861F86188A198A1A8A1C82FD
:10CE200016C082E08B831F8A188E198E1A8E408D51
:10CE3000518D60E070E025E0440F551F661F771F9D
:10CE40002A95D1F74B8B5C8B6D8B7E8BDACFDF9184
:10CE5000CF9108950F931F93CF93DF938C01EC0133
:10CE6000A396662321F0D093AD06C093AC06F801DB
:10CE700086A1882311F0CE0161DBB8016B5F7F4F83
:10CE8000CE01DF91CF911F910F919DCF8F929F92F5
:10CE9000AF92BF92CF92DF92EF92FF920F931F93C8
:10CEA000CF93DF93EC016A017B01480159014230C5
:10CEB00051056105710508F44DC049855A856B859A
:10CEC0007C854F5F5F4F6F4F7F4F4C155D056E0543
:10CED0007F0508F43FC08F89803129F499278F2D71
:10CEE0007E2D6D2D0BC08032A9F5C701B60157E02C
:10CEF00096958795779567955A95D1F70B891C89F3
:10CF00002D893E89600F711F821F931F43E073DAE2
:10CF1000009701F12F89203159F4DD24EE24FF24FC
:10CF2000F601EE0FFF1FE80FF91F9182808210C0FB
:10CF3000E894C7F8DD24EE24FF24F601EE0FFF1F6E
:10CF4000EE0FFF1FE80FF91F80829182A282B38249
:10CF500081E001C080E0DF91CF911F910F91FF90A0
:10CF6000EF90DF90CF90BF90AF909F908F900895FB
:10CF70002F923F924F925F926F927F928F929F92E9
:10CF8000AF92BF92CF92DF92EF92FF920F931F93D7
:10CF9000CF93DF93CDB7DEB72F970FB6F894DEBFF0
:10CFA0000FBECDBF1C014C875D876E877F873B8797
:10CFB0002A87DC0119960D911D912D913C911C97AA
:10CFC0000F5F1F4F2F4F3F4F0D831E832F833887D7
:10CFD000EA85FB8580809180A280B38081149104D2
:10CFE000A104B10431F0FFEF8F1A9F0AAF0ABF0A04
:10CFF00010C0DC018D909D90AD90BC90B1E0B987E0
:10D000000C851D852E853F850130110521053105D3
:10D0100009F0198675016401412C512C3201F1018E
:10D0200081859285A385B485481659066A067B06D4
:10D0300008F04EC00D811E812F8138850C151D050D
:10D040002E053F0550F472E0C72ED12CE12CF12CB7
:10D05000E2E08E2E912CA12CB12C9E012F5F3F4F30
:10D06000B701A601C10180DA882391F149815A8173
:10D070006B817C81D701C6010196A11DB11D452B95
:10D08000462B472B19F04C015D010FC0AC01BD01CF
:10D09000481959096A097B090C851D852E853F852C
:10D0A000401751076207730741F01FEF411A510AF9
:10D0B000610A710A6C017D01B2CF0FEF1FEF2FEFF4
:10D0C0003FE0B701A601C101E1DE8D83811113C0EC
:10D0D0001D823DC02601370121E0421A5108610836
:10D0E000710897018601B301A201C101CFDE882337
:10D0F00079F3730162018C149D04AE04BF0450F3F4
:10D10000AA85BB854D915D916D917C91411551052D
:10D1100061057105A9F4EA85FB8580829182A2826E
:10D12000B382F985FF2399F00FEF801A900AA00AC5
:10D13000B00AD1018D929D92AD92BC92139707C017
:10D1400095018401C101A2DE8111E5CFC1CF8D819E
:10D150002F960FB6F894DEBF0FBECDBFDF91CF91F3
:10D160001F910F91FF90EF90DF90CF90BF90AF9005
:10D170009F908F907F906F905F904F903F902F90F7
:10D180000895CF93DF93EC019C01295F3F4F41E06D
:10D1900050E060E070E08D819E81EADE882399F0A6
:10D1A0004F89588D698D7A8D452B462B472B59F425
:10D1B0004F81588569857A854F8B588F698F7A8F13
:10D1C000998190689983DF91CF9108952F923F9232
:10D1D0004F925F926F927F928F929F92AF92BF9287
:10D1E000CF92DF92EF92FF920F931F93CF93DF9333
:10D1F000CDB7DEB728970FB6F894DEBF0FBECDBF10
:10D200007C015B014A01DC0111968C9181FFB0C168
:10D2100082FD02C064018DC0F7014389548965898C
:10D22000768983859485A585B68584179507A60795
:10D23000B70781F3C70154DC8111ECCF99C1D70145
:10D2400015968D919C911697FC0134803A94B90102
:10D25000A80129E076956795579547952A95D1F7C6
:10D2600034221170332009F470C0D70113968C91C9
:10D2700013971596ED91FC911697823009F0A9C08D
:10D280001B964D905D906D907C901E9789E07694F2
:10D290006794579447948A95D1F7828D938DA48D86
:10D2A000B58D480E591E6A1E7B1E0115110509F425
:10D2B000AFC080E092E0801B910B16018C159D059C
:10D2C00008F41C010115110509F0A7C0F7014385F9
:10D2D00054856585768583899489A589B68948179B
:10D2E00059076A077B0708F498C045E0C301B201FB
:10D2F00082D8009709F43CC1A101B501800F911FAC
:10D300000F94C811020D131D0115124009F487C0B6
:10D31000F70183859485A585B685820D931DA11D92
:10D32000B11D83879487A587B687A20CB31CC2184A
:10D33000D308D7011B960D911D912D913C911E97FD
:10D34000C114D10409F07BCFE7C00115110509F024
:10D350008CCF17964D915D916D917C911A974115E7
:10D3600051056105710509F19E012F5F3F4FFCD802
:10D37000882309F4FDC089819A81AB81BC81F701C2
:10D3800025813681F9012789203139F4883FFFEF63
:10D390009F07A105B10590F416C0883F2FEF9207B3
:10D3A000A2072FE0B20778F009C0F7018789908DB6
:10D3B000A18DB28D0097A105B10529F4C701E1DE69
:10D3C000811153CFD5C0F70187839087A187B2879A
:10D3D0004CCF8481D70117962D913D914D915C9151
:10D3E0001A972250310941095109A82FB0E00F9432
:10D3F000C00D2B013C0186859785A089B189480E17
:10D40000591E6A1E7B1E430C511C611C711C4DCFA2
:10D41000C114B2E0DB0640F44CCF41E067CF0E947C
:10D42000AD61811175CFA4C0C11424E0D206F0F41F
:10D430008091A6049091A704A091A804B091A9049A
:10D4400084159505A605B70509F480D89501B301A3
:10D45000A20180919F049091A0040E94E360882320
:10D4600009F486C0212CA2E03A2E52CF8481831980
:10D470003D2C3694831508F4382E032D10E020E05F
:10D4800030E0B301A20180919F049091A0040E941A
:10D490004661882309F46CC085014D825E826F82EB
:10D4A00078868D818419831548F58091A604909122
:10D4B000A704A091A804B091A9042D813E814F81B9
:10D4C0005885281739074A075B0709F43FD8B80180
:10D4D00080919F049091A0040E9424611E5F2D8181
:10D4E0003E814F8158852F5F3F4F4F4F5F4F2D83B8
:10D4F0003E834F8358878111D4CF3AC080919F04D7
:10D500009091A0040E948C61882391F1232C312CEE
:10D51000322C2224330CFCCE53968D919D910D908C
:10D52000BC91A02DF701418180179107A207B30795
:10D5300038F4038B148B258B368B406841830CC0E9
:10D540008091AA069091AB06892B31F08114910449
:10D5500019F04068F7014183D70111968C9183FD42
:10D5600002C0C4010AC0C7010E9454628111F9CFF0
:10D5700081E0F70180838FEF9FEF28960FB6F89434
:10D58000DEBF0FBECDBFDF91CF911F910F91FF90F6
:10D59000EF90DF90CF90BF90AF909F908F907F9053
:10D5A0006F905F904F903F902F900895AF92BF92F1
:10D5B000CF92DF92EF92FF920F931F93CF93DF935F
:10D5C00000D01F92CDB7DEB75C016A017B0182E01B
:10D5D00090E0A0E0B0E0F50180839183A283B38363
:10D5E0009E012F5F3F4FB701A601C5010E94B462A3
:10D5F000811102C080E023C000E010E09801B70173
:10D60000A601C50143DC8823A9F3C980DA80EB8039
:10D61000FC80F5018789803149F481E0F8EFCF166D
:10D62000FFEFDF06E104F10450F4DACF81E098EF78
:10D63000C9169FEFD906E9069FE0F90688F20F9018
:10D640000F900F900F90DF91CF911F910F91FF904E
:10D65000EF90DF90CF90BF90AF9008954F925F9280
:10D660006F927F92AF92BF92CF92DF92EF92FF9232
:10D670000F931F93CF93DF9300D01F92CDB7DEB7E8
:10D680005C016A017B01FC0183818130E9F48181C5
:10D6900081FF1AC0F50183899489A589B689841709
:10D6A0009507A607B70780F0892B8A2B8B2B09F4E7
:10D6B00074C0F5014384548465847684B701A6015F
:10D6C000C5010EDA811102C080E068C0F5018581D4
:10D6D0009681C114D104E104F10469F44789508DA5
:10D6E000618D728D63DF882379F3F501178A108EBF
:10D6F000118E128E38C0F501478150856185728583
:10D700009E012F5F3F4F0E94B4628823E9F2498156
:10D710005A816B817C81F50185819681FC01278985
:10D72000203139F4483FFFEF5F0761057105D8F4F8
:10D7300007C0483F2FEF520762072FE0720798F4A7
:10D7400035DF882309F4C0CFF50147815085618515
:10D7500072850FEF1FEF2FEF3FE08581968196DBFB
:10D76000882309F4B1CFF501C38AD48AE58AF68A01
:10D77000818180688183C5010E945462882309F4F5
:10D78000A3CFB701A6014C145D046E047F0410F40E
:10D79000B301A201C501A4D901C081E00F900F908F
:10D7A0000F900F90DF91CF911F910F91FF90EF900D
:10D7B000DF90CF90BF90AF907F906F905F904F9031
:10D7C0000895BF92CF92DF92EF92FF920F931F9333
:10D7D000CF93DF93EC01B42E80E2689FF001112417
:10D7E000E655FB4F8091A6049091A704A091A80450
:10D7F000B091A9048F87988BA98BBA8B6C8304890D
:10D80000158920E030E0980111270027C28CD38CC5
:10D81000E12CF12C0C291D292E293F290F8B188F63
:10D82000298F3A8F8385887151F4048D158D268D4B
:10D83000378D0B8B1C8B2D8B3E8B81E00BC0803189
:10D84000F1F4CE0150DA811104C01B8A1C8A1D8AB2
:10D850001E8A84E08B838B2D8F7089831F821886AC
:10D8600019861A861B861C861D861E86B4FE0AC073
:10D8700040E050E0BA01CE01F1DE811103C01B820D
:10D8800080E012C0B5FE0FC04B895C896D897E892E
:10D89000CE01DF91CF911F910F91FF90EF90DF901C
:10D8A000CF90BF901DC981E0DF91CF911F910F9163
:10D8B000FF90EF90DF90CF90BF900895DF92EF92AE
:10D8C000FF920F931F93CF93DF938C01EB017A01AB
:10D8D000D22E8D819E81F80196838583838181116B
:10D8E00028C0209731F127FD24C0A70165E0440F2F
:10D8F000551F6A95E1F760E070E0CE01F1D888230A
:10D90000C1F0CE0102D80097A1F0FC0180818823EC
:10D9100081F0853E71F08E3261F06E2D6F704D2D6D
:10D92000C801DF91CF911F910F91FF90EF90DF9091
:10D9300048CF80E0DF91CF911F910F91FF90EF9042
:10D94000DF9008952F923F924F925F926F927F9255
:10D950008F929F92AF92BF92CF92DF92EF92FF92FF
:10D960000F931F93CF93DF93CDB7DEB7C454D10984
:10D970000FB6F894DEBF0FBECDBF4C017B016A012C
:10D98000422E302E1EAA1FAA18AE19AEDB01159624
:10D990008D919C911697F40196838583CB0141D993
:10D9A00046FE1AC0F60101900020E9F73197EC1904
:10D9B00077247394E9300CF0712C8E2F6DE00F9466
:10D9C0002D0D21E0911101C020E08E2F6DE00F940C
:10D9D0002D0D582E520E03C055245A94712C8E01D1
:10D9E0000A5C1F4F252D4AED59E0B501C7010E9481
:10D9F000B6645C01009779F1A895D7011B968D91CB
:10DA00009D910D90BC91A02D23968CAF9DAFAEAF94
:10DA1000BFAF2397B6018AED99E00E947A9D8111EC
:10DA2000DECF47FE02C080E08FC123968CAD9DAD56
:10DA3000AEADBFAD23974F97A109B109F5E0B695FB
:10DA4000A79597958795FA95D1F7682F6F70442D14
:10DA5000C401B7DE79C1842D8274823421F79E011E
:10DA6000265C3F4F452DFE0131965F01BF01C70186
:10DA7000DCD88EA99FA9A8ADB9AD892B8A2B8B2B99
:10DA8000A9F4D70113962C9113971B968D919D9114
:10DA90000D90BC91A02D223009F046C18115E0E423
:10DAA0009E07A105B10508F0BECF3EC122242394F4
:10DAB000D70111968C911197826011968C934EA983
:10DAC0005FA968AD79ADC7010BD8711037C06EE2A0
:10DAD00070E0C6010F94DC113C0186010A5F1F4F04
:10DAE000009761F044E050E0BC01CE01C1960F9474
:10DAF000F7111DAA0615170518F401C019AA380157
:10DB00006C187D087724A301B601CE0181960F948D
:10DB1000C811E1E2F0E0EC0FFD1FE60DF71D1082E9
:10DB200069E573E0CE0181960F94D111BE016F5C5F
:10DB30007F4FCE0181960F94D11105C0B601CE0161
:10DB400081960F94F011AE014F5C5F4FB501CE018D
:10DB500081960E94205EB501C4010E94635E782E0A
:10DB6000F60101900020E9F78F01015011090C190D
:10DB70001D09652C252D332727FD309525963FAFB0
:10DB80002EAF259711279E01215F3F4F3CAF2BAF52
:10DB9000225F3F4F3EAF2DAF662009F460C0862D57
:10DBA00090E0BC01615071093DE0639F602D11243C
:10DBB000D501E0E21D92EA95E9F72FE02C87259642
:10DBC0002EAD3FAD25978217930711F480E401C075
:10DBD00080E08629898340E050E0FE01329670E0C3
:10DBE000C601860F971F21969FAF8EAF2197CF0159
:10DBF00002969A01260F371F0217130734F49C016F
:10DC0000AFEFBFEFB183A0830DC09C012196AEADF5
:10DC1000BFAD2197A40FB51F8C91992787FD9095D3
:10DC200091838083443029F04A3029F42DAD3EADF4
:10DC300002C02BAD3CAD4F5F5F4F4D30510511F031
:10DC4000F901D5CF7E8640E250E0B501C701BEDACA
:10DC500097FDE9CEC7010E9454626A949DCF80E28D
:10DC6000F50111928A95E9F7AE014F5C5F4FB5015E
:10DC7000CE0181960E94205E332011F080E101C028
:10DC800080E28C8781E298E29A8B898B20E038E0F1
:10DC9000388B2F879C8B8B8B9A8F898F388F2F8B0C
:10DCA00040E250E0B501C70191DA97FDBCCEC70153
:10DCB0000E94546280E2D5011D928A95E9F72220E4
:10DCC00011F085EE8983D12C052D112707FD1095C4
:10DCD0008AAD992787FD9095801B910B2D2D3327B9
:10DCE00027FD30952817390764F440E250E0B5016C
:10DCF000C7016CDA97FD97CEC7010E945462D39496
:10DD0000E7CF242D2F774EA95FA968AD79ADE5E067
:10DD10007695679557954795EA95D1F7400F511F2E
:10DD2000B701C401CBDD10C021E0250D2AAF00975B
:10DD3000A105B10539F08097A109B1098EAB9FAB60
:10DD4000A8AFB9AF212CB4CECC5BDF4F0FB6F8949F
:10DD5000DEBF0FBECDBFDF91CF911F910F91FF901E
:10DD6000EF90DF90CF90BF90AF909F908F907F907B
:10DD70006F905F904F903F902F900895BF92CF92F9
:10DD8000DF92EF92FF920F931F93CF93DF93CDB764
:10DD9000DEB7A0970FB6F894DEBF0FBECDBF7C01F3
:10DDA0006B01FB018381823088F101E023ECC70124
:10DDB000C9DDB82E882351F18E010F5F1F4F80E21D
:10DDC000F80111928A95E9F721E238E23A8B298B22
:10DDD00080E098E0988B8F873C8B2B8B3A8F298F34
:10DDE000988F8F8B8EE2898380E18C87FE0132963B
:10DDF000CE010C9620E22193E817F907E1F740E203
:10DE000050E0B801C701E2D997FF02C0B12C37C07A
:10DE1000C7010E9454628EE28A83F6018381825098
:10DE2000823028F41C8E1B8E1E8A1D8A09C0F601C2
:10DE30004789508D618D728D5C8F4B8F7E8B6D8B82
:10DE400040E250E0B801C701C1D997FDDFCFC7015B
:10DE50000E94546280E2F80111928A95E9F740E24B
:10DE600050E0B801C701B2D997FDD0CFC7010E94D9
:10DE7000546284E0F70183838181806881838B2DE4
:10DE8000A0960FB6F894DEBF0FBECDBFDF91CF9145
:10DE90001F910F91FF90EF90DF90CF90BF9008956A
:10DEA0002F923F924F925F926F927F928F929F92AA
:10DEB000AF92BF92CF92DF92EF92FF920F931F9398
:10DEC000CF93DF93CDB7DEB7C154D1090FB6F89425
:10DED000DEBF0FBECDBF4B016A0139011801EFAEA5
:10DEE0001E8E19A219821C82F9011082611571051A
:10DEF00011F480E08AC0FC0183818111FACFFA011C
:10DF000080818F3261F4CA016C010196F601208193
:10DF10002F32D1F3F40183818250823010F4540106
:10DF20000CC0F40165817681CE0101960E94E36602
:10DF30008823F9F2CE0101965C017E019EE1E90E93
:10DF4000F11CFCAEEBAEFE013196FEAFEDAF2196BB
:10DF5000EFAE21972296FFAE229734C092012C1982
:10DF60003D09022F112707FD1095A801B601C30135
:10DF70000F94C811F301E00FF11F1082F2018181AB
:10DF80008823D9F100E021E0A301B501C701DADC63
:10DF9000882309F1A814B90419F0C5010E949E62F2
:10DFA0008BAD9CADE816F90609F121969FAD21973E
:10DFB00022968FAD22976201EFEFCE1ADE0A57014B
:10DFC000E92EF82E6FE270E0C6010F94DC112C01EF
:10DFD000009721F60EC0FFADFF2309F48ACFA301FD
:10DFE000B501C701CBDE8111D5CF83CF9DAD8EADFD
:10DFF000E2CFB601C3010F94F0118DE1F501D1011B
:10E0000001900D928A95E1F781E0CF5BDF4F0FB66B
:10E01000F894DEBF0FBECDBFDF91CF911F910F915E
:10E02000FF90EF90DF90CF90BF90AF909F908F9038
:10E030007F906F905F904F903F902F900895CF9278
:10E04000DF92EF920F931F93CF93DF93CDB7DEB79D
:10E05000E9970FB6F894DEBF0FBECDBF6C011982F1
:10E060001C82E22E8E010F5F1F4F9E01225E3F4FEA
:10E0700017DF882339F0AE01425E5F4FB801C60159
:10E080007DDE01C080E0E9960FB6F894DEBF0FBEDA
:10E09000CDBFDF91CF911F910F91EF90DF90CF9087
:10E0A0000895CF93DF93CDB7DEB76D970FB6F89491
:10E0B000DEBF0FBECDBF242F19821C828396AB0119
:10E0C000BC01CE010196BBDF6D960FB6F894DEBFA2
:10E0D0000FBECDBFDF91CF910895CF92DF92EF9227
:10E0E000FF920F931F93CF93DF93CDB7DEB7E997DE
:10E0F0000FB6F894DEBF0FBECDBF6C01F22E1982B1
:10E100001C82E12C8E010F5F1F4F9E01225E3F4F4C
:10E11000C7DE882371F08E8D882369F000E02F2DF3
:10E12000AE01425E5F4FBE016F5F7F4FC6010ADCEA
:10E1300003C080E001C081E0E9960FB6F894DEBF2D
:10E140000FBECDBFDF91CF911F910F91FF90EF9048
:10E15000DF90CF900895FF920F931F93CF93DF939B
:10E16000CDB7DEB76D970FB6F894DEBF0FBECDBF4B
:10E17000FB01F42E19821C8220812F3239F4218177
:10E18000211104C0642F0E942A671EC08C010D5DFE
:10E190001F4F21E0AF01B801CE0101969EDF882319
:10E1A00099F09C81923078F09DE1FE013196D80182
:10E1B00001900D929A95E1F7FF2031F01093AD0692
:10E1C0000093AC0601C080E06D960FB6F894DEBFF8
:10E1D0000FBECDBFDF91CF911F910F91FF9008959A
:10E1E000FB01242F6091AC067091AD06AF0175CF95
:10E1F000CF93DF93EC0140E050E0BA012FDA88239F
:10E2000071F061E0CE010E943D62009741F025EE81
:10E21000FC0120831B82DF91CF910C94AD6180E0E3
:10E22000DF91CF910895CF93DF93CDB7DEB76D9790
:10E230000FB6F894DEBF0FBECDBFAB0119821C82B2
:10E2400022E0BC01CE01019648DF882319F0CE01FF
:10E250000196CEDF6D960FB6F894DEBF0FBECDBF30
:10E26000DF91CF9108958396DECF0F931F93CF93C5
:10E27000DF93EC018B81843061F5CE010E94116641
:10E280000B851C852D853E854B895C896D897E8932
:10E29000041715072607370748F4CE010E94856446
:10E2A0000097B9F0FC01208121110BC081E08B8324
:10E2B000898182608983CE01DF91CF911F910F9177
:10E2C00097CF253EE9F22E32D9F2FC01838583FDFA
:10E2D000D7CF80E0DF91CF911F910F910895CF9319
:10E2E000DF93CDB7DEB76D970FB6F894DEBF0FBEE4
:10E2F000CDBF19821C8241E0CE01019671DF8823D7
:10E3000019F0CE010196B1DF6D960FB6F894DEBF1D
:10E310000FBECDBFDF91CF9108954F925F926F9264
:10E320007F92AF92BF92CF92DF92EF92FF920F93C4
:10E330001F93CF93DF93EC01142F7093A00460938D
:10E340009F041F8A82E090E0A0E0B0E08883998378
:10E35000AA83BB831092A5048FEF9FEFDC0180930B
:10E36000A6049093A704A093A804B093A9041092C4
:10E37000A1041092A2041092A3041092A4044423B6
:10E3800061F1453008F0D6C040E060E070E0CB01BC
:10E390000E94FB61009709F4CDC0FC0120E1129FAF
:10E3A000E00DF11D1124E255FE4F80818F7709F0B9
:10E3B000C1C044855585668577854436510561051C
:10E3C000710508F4B7C0C084D184E284F384C11419
:10E3D000D104E104F10421F4ADC0C12CD12C7601AB
:10E3E00040E0C701B6010E94FB61FC01009709F4FF
:10E3F000A1C0838594858115924009F09BC0208936
:10E40000222309F497C086859785892B09F492C049
:10E410008585882309F48EC02A8B25852C831D864B
:10E4200030E041E050E06D85062FCA01062E02C0A3
:10E43000880F991F0A94E2F72817390731F081E015
:10E44000860F8D87683078F375C026893789211546
:10E45000310519F040E050E004C024A135A146A1E7
:10E4600057A12D833E834F8358872093A104309377
:10E47000A2044093A3045093A404868597852601A3
:10E480003701480E591E611C711C4B8A5C8A6D8ACB
:10E490007E8AA188B288B98EA88EA089B0E00F9438
:10E4A000C00D640D751D861D971D6A8F7B8F8C8F27
:10E4B0009D8F15E0AA0CBB1C1A95E1F741E0A41A48
:10E4C0004EEFB40AAB2CBB24A694DC01CB018A0D21
:10E4D0009B1DA11DB11D8E879F87A88BB98B43887B
:10E4E00054884114510419F0612C712C04C040A0CF
:10E4F00051A062A073A0A7019601281B390B4A0BFB
:10E500005B0BDA01C901840D951DA61DB71D04C062
:10E51000B695A795979587950A95D2F789879A8793
:10E52000AB87BC87853F3FE09307A105B10520F489
:10E530008CE08F8B80E012C0853F9F4FA105B10515
:10E5400010F480E109C084A595A5A6A5B7A58A8F7A
:10E550009B8FAC8FBD8F80E28F8B81E0DF91CF915D
:10E560001F910F91FF90EF90DF90CF90BF90AF90F1
:10E570007F906F905F904F9008950F931F93CF936C
:10E58000DF93EC01842F462F682FCE010E94865F17
:10E590008823B9F08E010B5F1F4F41E0BE01C80117
:10E5A000BCDE882341F061E0CE01DF91CF911F9165
:10E5B0000F910C942A6740E0BE01C801AEDE8111C4
:10E5C000F2CF80E0DF91CF911F910F9108950C94CD
:10E5D000E668682F8FE29BE00C9478D92F923F92E7
:10E5E0004F925F926F927F928F929F92AF92BF9263
:10E5F000CF92DF92EF92FF920F931F93CF93DF930F
:10E60000CDB7DEB76D970FB6F894DEBF0FBECDBFA6
:10E610007B01342E59014801CB010E941166C12CA7
:10E62000D12C22242394230C00E010E020E04AEDBA
:10E6300059E0B601C7010E94B6646C01009739F039
:10E64000A895D6011B961C9113FF03C0EDCF80E067
:10E65000C2C06EE573E08AED99E00F94E711892B53
:10E6600019F31871103109F067C0B1E0B315E0F289
:10E67000A114B10491F4332041F081EA99E00E94A1
:10E68000C99F86E294E20E94859F8AED99E00E94EC
:10E69000C99F86E294E20E949E9F19821C823320C9
:10E6A00031F06CE573E081EA99E00F94D1116AEDE5
:10E6B00079E081EA99E00F94D111F7014384548401
:10E6C00065847684FFE14F1A51086108710845E0BE
:10E6D00076946794579447944A95D1F721E0A20124
:10E6E000B701CE010196EAD8882351F08401950143
:10E6F000422DBE016F5F7F4FCB0170DF81116AC079
:10E700008FEF481A580A35E0440C551C3A95E1F74A
:10E71000A20160E070E0C7010E9470656FE270E0E6
:10E7200081EA99E00F940612009719F0DC011C921F
:10E730007BCF1092A10978CFA114B10489F1E1EA4D
:10E74000F9E0DF010D900020E9F78D01015011097A
:10E75000015A1940702E402F552747FD5095B5019D
:10E76000CF010E94B79D81115FCF10161CF4772452
:10E770007394700EB501670D711D77FC7A958AED63
:10E7800099E00E947A9D81114FCF8114910411F17B
:10E790008DE1F701D40101900D928A95E1F71AC03D
:10E7A000332041F081EA99E00E94C99F86E294E219
:10E7B0000E94859F8AED99E00E94C99FF601448DD1
:10E7C000558D668D778D85EB93E20E94A9A00E94FE
:10E7D000D9232ACF81E06D960FB6F894DEBF0FBE25
:10E7E000CDBFDF91CF911F910F91FF90EF90DF9000
:10E7F000CF90BF90AF909F908F907F906F905F90E1
:10E800004F903F902F900895EF92FF920F931F9398
:10E81000CF93DF93CDB7DEB76D970FB6F894DEBF19
:10E820000FBECDBF7C0119821C820E941166E1EAF5
:10E83000F9E01082D7015C96FC93EE935B978DE133
:10E84000F701DE01119601900D928A95E1F700E043
:10E8500010E020E030E040E0BE016F5F7F4FC70175
:10E86000BDDE6D960FB6F894DEBF0FBECDBFDF9153
:10E87000CF911F910F91FF90EF900895882321F081
:10E8800080910B018D7F03C080910B01826080938A
:10E890000B010895882321F080910B018E7F03C026
:10E8A00080910B01816080930B010895882321F0F2
:10E8B00080910B018B7F03C080910B01846080935A
:10E8C0000B010895FB01DC0180914708882349F082
:10E8D00023E333E34BEC51E4CD010F94570CFB01E0
:10E8E000DC01BF01CD010895CF93DF931F92CDB717
:10E8F000DEB79091BE0790FF02C0811146C0209103
:10E90000BD0723FD42C091609093BE07179A169AE7
:10E91000159A89830E94B0518981811128C020E015
:10E9200040E060E070E0CB010E94165520E041E03D
:10E9300060E070E0CB010E94165540E060E070E0BE
:10E94000CB010E94DF5540E069E877E18CE69AE070
:10E950000E9494AB8CE69AE00E94E8AE9B9AA39A40
:10E960008091BD078F7B88608093BD070EC040E01B
:10E9700068E777E18CE69AE00E9494AB8CE69AE037
:10E980000F90DF91CF910C94E8AE0F90DF91CF9173
:10E990000895CF93C091BE07CD7FC093BE0720E0FE
:10E9A00030E0A90160918002709181028091820221
:10E9B000909183020F94AF09882319F0C260C0932D
:10E9C000BE07CF9108952F923F924F925F926F9220
:10E9D0007F928F929F92AF92BF92CF92DF92EF92EF
:10E9E000FF920F931F93CF93DF93CDB7DEB76D9751
:10E9F0000FB6F894DEBF0FBECDBF8BE793E00F9448
:10EA00002E12909344078093430789E793E00F9475
:10EA10002E129093420780934107C0902F03D0900D
:10EA20003003E0903103F0903203C0922B03D09278
:10EA30002C03E0922D03F0922E03C0922703D09274
:10EA40002803E0922903F0922A0380910303909116
:10EA50000403A0910503B09106038093FF029093F5
:10EA60000003A0930103B09302038093FB029093F1
:10EA7000FC02A093FD02B093FE02809113039091DB
:10EA80001403A0911503B091160380930F03909384
:10EA90001003A0931103B093120380930B03909380
:10EAA0000C03A0930D03B0930E0380911F0390916C
:10EAB0002003A0912103B091220380931B03909324
:10EAC0001C03A0931D03B0931E0380931703909320
:10EAD0001803A0931903B0931A038091F302909145
:10EAE000F402A091F502B091F6028093EF029093A8
:10EAF000F002A093F102B093F2028093EB029093A4
:10EB0000EC02A093ED02B093EE0220910107309148
:10EB100002074091030750910407C701B6010F9403
:10EB2000570C0F944F0A609321077093220780932C
:10EB300023079093240720910D0730910E074091F1
:10EB40000F0750911007C701B6010F94570C0F948F
:10EB50004F0A60931D0770931E0780931F079093C1
:10EB60002007209105073091060740910707509133
:10EB70000807C701B6010F94570C0F944F0A609312
:10EB8000190770931A0780931B0790931C07209115
:10EB9000FD063091FE064091FF0650910007C70127
:10EBA000B6010F94570C0F944F0A6093150770939A
:10EBB00016078093170790931807C0906D07D090A1
:10EBC0006E07E0906F07F090700781E993E00E9474
:10EBD0002F1D9B01AC01C701B6010F944B092B01FE
:10EBE0003C01C0906D07D0906E07E0906F07F090E9
:10EBF000700785E993E00E942F1D9B01AC01C701BE
:10EC0000B6010F944B094B015C01C0906D07D09089
:10EC10006E07E0906F07F090700789E993E00E941B
:10EC20002F1D9B01AC01C701B6010F944B096B016D
:10EC30007C0185E893E00E942F1D2BED3FE049E425
:10EC400050E40F94570C20E030E044E353E40F9479
:10EC5000B6090F94B3099B01AC01C301B2010F9433
:10EC6000570C20912F033091300340913103509184
:10EC700032030F94570C20E030E040E05FE30F9444
:10EC80004B090F94BD0A0F944F0A60936507709368
:10EC90006607809367079093680785E893E00E9472
:10ECA0002F1D2BED3FE049E450E40F94570C20E07A
:10ECB00030E044E353E40F94B6090F94BA0C9B017F
:10ECC000AC01C301B2010F94570C20912F03309176
:10ECD000300340913103509132030F94570C20E0E0
:10ECE00030E040E05FE30F944B090F94BD0A0F94AE
:10ECF0004F0A609361077093620780936307909354
:10ED0000640789E893E00E942F1D2BED3FE049E462
:10ED100050E40F94570C20E030E044E353E40F94A8
:10ED2000B6090F94B3099B01AC01C501B4010F945E
:10ED3000570C20912F0330913003409131035091B3
:10ED400032030F94570C20E030E040E05FE30F9473
:10ED50004B090F94BD0A0F944F0A60935D0770939F
:10ED60005E0780935F079093600789E893E00E94B5
:10ED70002F1D2BED3FE049E450E40F94570C20E0A9
:10ED800030E044E353E40F94B6090F94BA0C9B01AE
:10ED9000AC01C501B4010F94570C20912F033091A1
:10EDA000300340913103509132030F94570C20E00F
:10EDB00030E040E05FE30F944B090F94BD0A0F94DD
:10EDC0004F0A6093590770935A0780935B0790939B
:10EDD0005C078DE893E00E942F1D2BED3FE049E496
:10EDE00050E40F94570C20E030E044E353E40F94D8
:10EDF000B6090F94B3099B01AC01C701B6010F948A
:10EE0000570C20912F0330913003409131035091E2
:10EE100032030F94570C20E030E040E05FE30F94A2
:10EE20004B090F94BD0A0F944F0A609355077093D6
:10EE3000560780935707909358078DE893E00E94F8
:10EE40002F1D2BED3FE049E450E40F94570C20E0D8
:10EE500030E044E353E40F94B6090F94BA0C9B01DD
:10EE6000AC01C701B6010F94570C20912F033091CC
:10EE7000300340913103509132030F94570C20E03E
:10EE800030E040E05FE30F944B090F94BD0A0F940C
:10EE90004F0A6093510770935207809353079093E2
:10EEA000540785EA93E00E942F1D6B017C0181E7E6
:10EEB00093E00E942F1D9B01AC01C701B6010F9486
:10EEC0004B0920912F033091300340913103509131
:10EED00032030F94570C0F94540A60937D0770937C
:10EEE0007E0780937F079093800789EA93E00E94D2
:10EEF0002F1D6B017C0181E793E00E942F1D9B0178
:10EF0000AC01C701B6010F944B0920912F0330913A
:10EF1000300340913103509132030F94570C0F94FA
:10EF2000540A6093790770937A0780937B079093D4
:10EF30007C078DEA93E00E942F1D6B017C0181E725
:10EF400093E00E942F1D9B01AC0140902F03509035
:10EF500030036090310370903203C701B6010F9403
:10EF60004B09A30192010F94570C0F94540A4B01C3
:10EF70005C01C0907D07D0907E07E0907F07F09005
:10EF800080071091BE078FEFC816D806E104F10480
:10EF9000C0F460916D0770916E0780916F0790913A
:10EFA00070079B01AC010F944B09A30192010F94D0
:10EFB000570C20E03EEF4FE757E40F94E30B181691
:10EFC000D4F510681093BE07C701B6010F94800AEC
:10EFD0009B01AC010F94570C60937D0770937E07E3
:10EFE00080937F07909380076091790770917A07EB
:10EFF00080917B0790917C070F94800A9B01AC0164
:10F000000F94570C6093790770937A0780937B076E
:10F0100090937C07C501B4010F94800A9B01AC0159
:10F020000F94570C6093750770937607809377075A
:10F030009093780733C01F771093BE07A7019601FE
:10F04000C701B6010F941E0D60937D0770937E0774
:10F0500080937F07909380076091790770917A077A
:10F0600080917B0790917C079B01AC010F941E0D52
:10F070006093790770937A0780937B0790937C075E
:10F08000A5019401C501B4010F941E0D609375078D
:10F090007093760780937707909378078DE993E0D4
:10F0A0000E942F1D9B01AC010F94570C60937107B8
:10F0B000709372078093730790937407198A1A8A62
:10F0C0001B8A1C8A1D861E861F86188A809121072E
:10F0D00090912207A0912307B09124078D8B9E8BDE
:10F0E000AF8BB88FBE016F5F7F4FCE010D960E9430
:10F0F000F3EC89819A81AB81BC81809381079093E5
:10F100008207A0938307B093840780912107909191
:10F110002207A0912307B09124078093250790939D
:10F120002607A0932707B093280780932907909379
:10F130002A07A0932B07B0932C0710921507109263
:10F1400016071092170710921807109219071092BD
:10F150001A0710921B0710921C0710921D0710929D
:10F160001E0710921F071092200740902F03509007
:10F170003003609031037090320320E030E040E7CC
:10F1800051E4C301B2010F94570C0F944F0A6093DE
:10F19000690770936A0780936B0790936C0787E207
:10F1A000882E83E0982E97E3A92E98E0B92E0BEFD6
:10F1B00012E027E2222E28E0322EEBEEF2E0FD8F65
:10F1C000EC8F87E198E09B8F8A8F198EF401C190B4
:10F1D000D190E190F1904F01A701960160E070E0BD
:10F1E00080E89FE30F94B609F501619371938193D1
:10F1F00091935F01F80161917191819191918F01DA
:10F20000A70196010F94570C0F94540AF1016193D2
:10F210007193819391931F01EC8DFD8D619171919B
:10F2200081919191FD8FEC8FA70196010F94570C5E
:10F230000F94540AEA8DFB8D61937193819391939E
:10F24000FB8FEA8FF98DFF5FF98FF43009F0BECFA5
:10F25000A090EB02B090EC02C090ED02D090EE02D4
:10F26000E090FB02F090FC020091FD021091FE0282
:10F270009501A601B701C8010F94AF0987FF02C02D
:10F2800075018601209127033091280340912903BD
:10F2900050912A03B701C8010F94570C9B01AC0190
:10F2A00060E070E080E090E40F94B6090F94C40C25
:10F2B0009B01AC01B701C8010F94570C6093310753
:10F2C000709332078093330790933407A090F30232
:10F2D000B090F402C090F502D090F602E0900303E3
:10F2E000F090040300910503109106039501A60117
:10F2F000B701C8010F94AF0987FF02C075018601ED
:10F300009701A801C301B2010F94570C9B01AC01F6
:10F3100060E070E080E090E40F94B6090F94C40CB4
:10F320009B01AC01B701C8010F94570C60932D07E6
:10F3300070932E0780932F07909330072ADB6D96EA
:10F340000FB6F894DEBF0FBECDBFDF91CF911F91F6
:10F350000F91FF90EF90DF90CF90BF90AF909F9074
:10F360008F907F906F905F904F903F902F90089577
:10F37000EF92FF920F931F936093BF077093C007A4
:10F380008093C1079093C2072093C3073093C407AB
:10F390004093C5075093C607E092C707F092C8078D
:10F3A0000093C9071093CA071F910F91FF90EF9028
:10F3B0000895CF92DF92EF92FF9281E00E94041EA7
:10F3C0008CE69AE00E9474CA0F94E6032091210C07
:10F3D000211148C02091BB0722FD44C0C090811D6F
:10F3E000D090821DE090831DF090841D9B01AC01A4
:10F3F0002C193D094E095F0969017A018091420388
:10F4000090914303A0914403B09145030097A10557
:10F41000B10541F08C159D05AE05BF0518F480E0DF
:10F4200063DA05C08091BD07877F8093BD07809117
:10F430003E0390913F03A0914003B0914103009798
:10F44000A105B10539F08C159D05AE05BF0510F479
:10F4500081E04ADA88E199E0FF90EF90DF90CF9069
:10F460000C94F79A6093811D7093821D8093831D85
:10F470009093841DEFCFAF92BF92CF92DF92EF9225
:10F48000FF920F931F93CF93DF93EB01D82EC92EDA
:10F490001092F3071092F4071092F5071092F607F6
:10F4A0001092F7071092F8071092F9071092FA07D6
:10F4B0001092FB071092FC071092FD071092FE07B6
:10F4C00067E078E083EF97E00E94F3EC609121071A
:10F4D0007091220780912307909124070F94820A4C
:10F4E00020E030E040EC5FE30F94570C0F944F0A9C
:10F4F0007B018C0121E02F932F93CF92DF92DF933A
:10F50000CF93A12CB12C650120E030E0A90160E08F
:10F5100070E0CB010E9407F81092ED061092EE0603
:10F520001092EF061092F0061092E9061092EA0689
:10F530001092EB061092EC060F900F900F900F9028
:10F540000F900F90DF91CF911F910F91FF90EF904F
:10F55000DF90CF90BF90AF9008954F925F926F92DF
:10F560007F928F929F92AF92BF92CF92DF92EF9253
:10F57000FF920F931F93CF93DF9300D01F92CDB7CD
:10F58000DEB760911303709114038091150390917D
:10F59000160371DF60912F03709130038091310366
:10F5A000909132039B01AC010F944B0920E030E0B5
:10F5B00040EA50EC0F94570C0F944F0A2B013C017A
:10F5C0001F92992493949F9220E030E040E05FE303
:10F5D00060911303709114038091150390911603A9
:10F5E0000F94570C9F938F937F936F93A12CB12C03
:10F5F00065018301720120E030E0A90160E070E064
:10F60000CB010E9407F820E030E040E05FE360912A
:10F6100013037091140380911503909116030F94B6
:10F62000570C29DF20E030E040EA50EC60912F03D6
:10F630007091300380913103909132030F94570CF5
:10F640000F944F0A1F929F92209116032F9320919F
:10F6500015032F93209114032F93209113032F93BD
:10F660007B018C0120E030E0A90160E070E0CB017B
:10F670000E9407F88DE793E00F942E1280901D07EB
:10F6800090901E07A0901F07B0902007B094A09400
:10F6900090948094811C911CA11CB11CAA2797FDF9
:10F6A000A095BA2F881A990AAA0ABB0A8FE793E095
:10F6B0000F942E12C0901907D0901A07E0901B07E4
:10F6C000F0901C07F094E094D094C094C11CD11C1D
:10F6D000E11CF11CAA2797FDA095BA2FC81AD90AD8
:10F6E000EA0AFB0A81E893E00F942E124091150775
:10F6F00050911607609117077091180770956095E3
:10F70000509541955F4F6F4F7F4FAA2797FDA0956A
:10F71000BA2F481B590B6A0B7B0B0FB6F894DEBF50
:10F720000FBECDBF2A013B018C149D04AE04BF0463
:10F7300044F484169506A606B70654F42401350150
:10F7400007C0C416D506E606F70614F426013701ED
:10F7500084189508A608B708C418D508E608F7085D
:10F76000DB01CA0184199509A609B70989839A831F
:10F77000AB83BC831092F3071092F4071092F50745
:10F780001092F6071092F7071092F8071092F907F7
:10F790001092FA078091210790912207A0912307E8
:10F7A000B09124078093FB079093FC07A093FD077B
:10F7B000B093FE0767E078E083EF97E00E94F3ECF8
:10F7C0008091070890910808A0910908B0910A0853
:10F7D00088199909AA09BB0980930708909308081A
:10F7E000A0930908B0930A0880910B0890910C0827
:10F7F000A0910D08B0910E088C199D09AE09BF09A2
:10F8000080930B0890930C08A0930D08B0930E08FA
:10F8100080910F0890911008A0911108B0911208E2
:10F8200029813A814B815C81821B930BA40BB50B20
:10F8300080930F0890931008A0931108B0931208BA
:10F840001F9281E08F93809116038F93809115030F
:10F850008F93809114038F93809113038F93A12C26
:10F86000B12C65018301720120E030E0A90160E064
:10F8700070E0CB010E9407F81092F3071092F40792
:10F880001092F5071092F6071092F7071092F807FA
:10F890001092F9071092FA078091210790912207A0
:10F8A000A0912307B09124078093FB079093FC0756
:10F8B000A093FD07B093FE071092BF071092C007F8
:10F8C0001092C1071092C2071092C3071092C4078A
:10F8D0001092C5071092C6071092C7071092C8076A
:10F8E0001092C9071092CA0767E078E083EF97E0AB
:10F8F0000E94F3EC8091070890910808A0910908F4
:10F90000B0910A088093450790934607A093470754
:10F91000B093480780910B0890910C08A0910D08B6
:10F92000B0910E088093490790934A07A0934B0724
:10F93000B0934C0780910F0890911008A091110886
:10F94000B091120880934D0790934E07A0934F07F4
:10F95000B09350076091810770918207809183076F
:10F96000909184070F94820A6B017C0120E030E0C3
:10F9700040EA50E460912F0370913003809131038D
:10F98000909132030F94570C9B01AC01C701B60153
:10F990000F944B090F944F0A60938107709382076D
:10F9A00080938307909384070F900F900F900F9090
:10F9B0000F900F90E0918603F091870380810F9064
:10F9C0000F900F900F90DF91CF911F910F91FF90AB
:10F9D000EF90DF90CF90BF90AF909F908F907F90EF
:10F9E0006F905F904F900C94DF4F0F931F93CF93C6
:10F9F000DF9380910508C1E018161CF0C0E08F5F0E
:10FA000001C0815080930508179816981598809129
:10FA1000BE078E7F8093BE070091090110910901F6
:10FA2000D09109018C2F0E943E748C2F0E944A7441
:10FA30008C2F0E94567481E090E00F943A04409A13
:10FA4000419A429A82E090E00F943A04409841989B
:10FA50004298C1E001FB882780F98C270E943E7400
:10FA6000812F81708C270E944A74D2FB882780F9ED
:10FA70008C27DF91CF911F910F910C9456744F9268
:10FA80005F926F927F928F929F92AF92BF92CF922E
:10FA9000DF92EF92FF920F931F93CF93DF93CDB737
:10FAA000DEB728970FB6F894DEBF0FBECDBF2B018F
:10FAB0003C0129833A834B835C83ED82FE820F8372
:10FAC0001887850174012091930730919407409124
:10FAD0009507509196070F94570C4B015C012091AC
:10FAE0009F073091A0074091A1075091A20769811B
:10FAF0007A818B819C810F94570C9B01AC01C501CD
:10FB0000B4010F944B094B015C012091AB0730917C
:10FB1000AC074091AD075091AE076D817E818F811A
:10FB200098850F94570C9B01AC01C501B4010F944B
:10FB30004B09F60160837183828393832091970739
:10FB4000309198074091990750919A07C301B201EB
:10FB50000F94570C4B015C012091A3073091A4072F
:10FB60004091A5075091A60769817A818B819C817C
:10FB70000F94570C9B01AC01C501B4010F944B09C4
:10FB80004B015C012091AF073091B0074091B10764
:10FB90005091B2076D817E818F8198850F94570CAB
:10FBA0009B01AC01C501B4010F944B09F8016083BE
:10FBB00071838283938320919B0730919C074091AE
:10FBC0009D0750919E07C301B2010F94570C4B0142
:10FBD0005C012091A7073091A8074091A907509197
:10FBE000AA0769817A818B819C810F94570C9B01B4
:10FBF000AC01C501B4010F944B094B015C0120918C
:10FC0000B3073091B4074091B5075091B6076D81A5
:10FC10007E818F8198850F94570C9B01AC01C501A3
:10FC2000B4010F944B09F70160837183828393833E
:10FC300028960FB6F894DEBF0FBECDBFDF91CF91EF
:10FC40001F910F91FF90EF90DF90CF90BF90AF90FA
:10FC50009F908F907F906F905F904F9008954F92FC
:10FC60005F926F927F928F929F92AF92BF92CF924C
:10FC7000DF92EF92FF920F931F93CF93DF93CDB755
:10FC8000DEB764970FB6F894DEBF0FBECDBF6983B1
:10FC90007A838B839C832D833E834F835887E986A9
:10FCA000FA860B871C8725013601E62EF72E082FD2
:10FCB000192F20EF33E244E759E4B701C8010F944C
:10FCC000AF0981110DC08091E7079091E807A091DD
:10FCD000E907B091EA0789839A83AB83BC830AC0A2
:10FCE000C701D8018093E7079093E807A093E9073D
:10FCF000B093EA07CD80DE80EF80F88420EF33E216
:10FD000044E759E4C701B6010F94AF0981110DC052
:10FD10008091EB079091EC07A091ED07B091EE0771
:10FD20008D839E83AF83B88708C0C092EB07D092C3
:10FD3000EC07E092ED07F092EE07C984DA84EB84D9
:10FD4000FC8420EF33E244E759E4C701B6010F9485
:10FD5000AF0981110DC08091EF079091F007A0913C
:10FD6000F107B091F20789879A87AB87BC8708C0F3
:10FD7000C092EF07D092F007E092F107F092F207FD
:10FD80008091BE0785FF3DC029853A854B855C85FE
:10FD90002D873E874F87588B2091E9063091EA06E0
:10FDA0004091EB065091EC066D817E818F819885A4
:10FDB0000F944B09698B7A8B8B8B9C8B2091ED0672
:10FDC0003091EE064091EF065091F00669817A81FC
:10FDD0008B819C810F944B09AE01475F5F4F4A01B5
:10FDE000DE0115965D019E012F5F3F4F6901ED8495
:10FDF000FE840F85188929893A894B895C893FDE01
:10FE000024C02091ED063091EE064091EF0650910E
:10FE1000F00669817A818B819C810F944B096983FB
:10FE20007A838B839C832091E9063091EA06409186
:10FE3000EB065091EC066D817E818F8198850F9441
:10FE40004B096D837E838F839887209127033091A0
:10FE500028034091290350912A0369817A818B817B
:10FE60009C810F94570C20E030E040E05FE30F945A
:10FE70004B090F94BD0A0F944F0A6093CB07709300
:10FE8000CC078093CD079093CE0720912B03309120
:10FE90002C0340912D0350912E036D817E818F8123
:10FEA00098850F94570C20E030E040E05FE30F941A
:10FEB0004B090F94BD0A0F944F0A6093CF077093BC
:10FEC000D0078093D1079093D20720912F033091D0
:10FED0003003409131035091320369857A858B85D7
:10FEE0009C850F94570C20E030E040E05FE30F94D6
:10FEF0004B090F94BD0A0F944F0A6093D307709378
:10FF0000D4078093D5079093D60720EF33E244E7D8
:10FF100059E4C301B2010F94AF098823C1F0809165
:10FF2000EA0283FD14C0E0918603F091870320E08C
:10FF300030E046E153E462A973A984A995A90F941E
:10FF4000E30B18165CF18091BD0787FD27C020EFF9
:10FF500033E244E759E468A579A58AA59BA50F94E7
:10FF6000AF09882361F088A599A5AAA5BBA58093B0
:10FF7000F9069093FA06A093FB06B093FC0641E0C5
:10FF800061E081E00E94D7F2811106C088E297E12A
:10FF90000E94AB9F80E019C081E017C0209133031D
:10FFA000309134034091350350913603C301B201BF
:10FFB0000F94570C0F944F0A6093D7077093D8078C
:10FFC0008093D9079093DA07C2CF64960FB6F8945E
:10FFD000DEBF0FBECDBFDF91CF911F910F91FF907C
:10FFE000EF90DF90CF90BF90AF909F908F907F90D9
:10FFF0006F905F904F9008954F925F926F927F92B3
:020000021000EC
:100000008F929F92AF92BF92CF92DF92EF92FF9228
:100010000F931F93CF93DF93CDB7DEB728970FB61B
:10002000F894DEBF0FBECDBF2B013C0129833A837C
:100030004B835C83ED82FE820F83188785017401F8
:10004000209193073091940740919507509196071E
:100050000F94570C4B015C01209197073091980742
:100060004091990750919A0769817A818B819C818F
:100070000F94570C9B01AC01C501B4010F944B09BF
:100080004B015C0120919B0730919C0740919D079B
:1000900050919E076D817E818F8198850F94570CBA
:1000A0009B01AC01C501B4010F944B09F6016083BB
:1000B00071838283938320919F073091A0074091A1
:1000C000A1075091A207C301B2010F94570C4B0135
:1000D0005C012091A3073091A4074091A50750919E
:1000E000A60769817A818B819C810F94570C9B01B3
:1000F000AC01C501B4010F944B094B015C01209187
:10010000A7073091A8074091A9075091AA076D81D0
:100110007E818F8198850F94570C9B01AC01C5019E
:10012000B4010F944B09F801608371838283938338
:100130002091AB073091AC074091AD075091AE07CD
:10014000C301B2010F94570C4B015C012091AF0722
:100150003091B0074091B1075091B20769817A811F
:100160008B819C810F94570C9B01AC01C501B4019C
:100170000F944B094B015C012091B3073091B407F8
:100180004091B5075091B6076D817E818F8198852A
:100190000F94570C9B01AC01C501B4010F944B099E
:1001A000F701608371838283938328960FB6F89456
:1001B000DEBF0FBECDBFDF91CF911F910F91FF909A
:1001C000EF90DF90CF90BF90AF909F908F907F90F7
:1001D0006F905F904F9008953F924F925F926F9211
:1001E0007F928F929F92AF92BF92CF92DF92EF92C7
:1001F000FF920F931F93CF93DF9300D01F92CDB741
:10020000DEB7382E6091F3077091F4078091F507FF
:100210009091F6070F94820A2091370830913808A0
:100220004091390850913A080F94570C2B013C012A
:100230006093E7077093E8078093E9079093EA07D4
:100240006091F7077091F8078091F9079091FA078C
:100250000F94820A20913B0830913C0840913D0860
:1002600050913E080F94570C69837A838B839C834B
:100270006093EB077093EC078093ED079093EE0784
:100280006091FB077091FC078091FD079091FE073C
:100290000F94820A20913F08309140084091410814
:1002A000509142080F94570C6093EF077093F0073A
:1002B0008093F1079093F2072091BE0725FF15C0A8
:1002C0004FEE842E47E0942E5BEEA52E57E0B52E20
:1002D000E7EECE2EE7E0DE2E7B018C0129813A810C
:1002E0004B815C81C301B20187DE2091ED06309124
:1002F000EE064091EF065091F0066091E70770918D
:10030000E8078091E9079091EA070F944A092B01C9
:100310003C016093E7077093E8078093E9079093A7
:10032000EA072091E9063091EA064091EB065091E8
:10033000EC066091EB077091EC078091ED079091CE
:10034000EE070F944A096093EB077093EC078093D4
:10035000ED079093EE07332001F14092DB075092B6
:10036000DC076092DD077092DE076093DF07709311
:10037000E0078093E1079093E2078091EF07909167
:10038000F007A091F107B091F2078093E3079093F3
:10039000E407A093E507B093E6070F900F900F9046
:1003A0000F90DF91CF911F910F91FF90EF90DF9011
:1003B000CF90BF90AF909F908F907F906F905F9005
:1003C0004F903F9008954F925F926F927F928F92DD
:1003D0009F92AF92BF92CF92DF92EF92FF920F93D4
:1003E0001F93CF93DF932B013C0149015A01670111
:1003F00078018091BD0785FD53C020E030E048ECD6
:1004000052ECC701B6010F94E30B87FD1DC02DEC24
:100410003CEC4CE45DE36091010770910207809130
:100420000307909104070F944B0920E030E040EA65
:1004300050E40F944B099B01AC01C1E0C701B60128
:100440000F94AF0918160CF4C0E0A3019201C30188
:10045000B2010F94570C6B017C01A5019401C501F9
:10046000B4010F94570C9B01AC01C701B6010F9466
:100470004B09D1E0209171073091720740917307C9
:10048000509174070F94AF0918160CF4D0E0CD23E7
:1004900041F481E0A1DE80E997E10E94341E01C0B1
:1004A000C1E08C2FDF91CF911F910F91FF90EF90C2
:1004B000DF90CF90BF90AF909F908F907F906F9084
:1004C0005F904F9008952F923F924F925F926F925C
:1004D0007F928F929F92AF92BF92CF92DF92EF92D4
:1004E000FF920F931F93CF93DF93CDB7DEB7609743
:1004F0000FB6F894DEBF0FBECDBF1C01809104087B
:10050000F1011081811169C013FF20C062857385DC
:10051000848595850E9462742091BF073091C00741
:100520004091C1075091C2070F944A096093E707B1
:100530007093E8078093E9079093EA076093DB07DD
:100540007093DC078093DD079093DE0714FF21C0D2
:10055000F10166857785808991890E946274209176
:10056000C3073091C4074091C5075091C6070F9447
:100570004A096093EB077093EC078093ED07909323
:10058000EE076093DF077093E0078093E107909395
:10059000E20715FF8BC0F10162897389848995890F
:1005A0000E9462742091C7073091C8074091C90723
:1005B0005091CA070F944A096093EF077093F007B0
:1005C0008093F1079093F2076093E3077093E40739
:1005D0008093E5079093E60769C013FF21C0F101FE
:1005E00062857385848595850E9462742091DB07FE
:1005F0003091DC074091DD075091DE070F944B09E5
:100600006093DB077093DC078093DD079093DE0730
:100610006093E7077093E8078093E9079093EA07F0
:1006200014FF21C0F10166857785808991890E9438
:1006300062742091DF073091E0074091E10750910B
:10064000E2070F944B096093DF077093E0078093F4
:10065000E1079093E2076093EB077093EC078093B8
:10066000ED079093EE0715FF21C0F10162897389B0
:10067000848995890E9462742091E3073091E40790
:100680004091E5075091E6070F944B096093E3070B
:100690007093E4078093E5079093E6076093EF0774
:1006A0007093F0078093F1079093F2078091BE0753
:1006B0004090E3075090E4076090E5077090E607EC
:1006C00085FF3BC02091E9063091EA064091EB0698
:1006D0005091EC066091DF077091E0078091E1078F
:1006E0009091E2070F944B096D877E878F87988BD7
:1006F0002091ED063091EE064091EF065091F00604
:100700006091DB077091DC078091DD079091DE0737
:100710000F944B099E012F5F3F4F4901AE014B5F84
:100720005F4F5A01FE0139966F01830172012D85D9
:100730003E854F855889A3D930C02091ED06309170
:10074000EE064091EF065091F0066091DB07709144
:10075000DC078091DD079091DE070F944B096987D4
:100760007A878B879C872091E9063091EA06409131
:10077000EB065091EC066091DF077091E0078091E5
:10078000E1079091E2070F944B096D837E838F837D
:10079000988749825A826B827C822091270330910C
:1007A00028034091290350912A0369857A858B8516
:1007B0009C850F94570C20E030E040E05FE30F94FD
:1007C0004B090F94BD0A0F944F0A6093CB077093A7
:1007D000CC078093CD079093CE0720912B033091C7
:1007E0002C0340912D0350912E036D817E818F81CA
:1007F00098850F94570C20E030E040E05FE30F94C1
:100800004B090F94BD0A0F944F0A6093CF07709362
:10081000D0078093D1079093D20720912F03309176
:100820003003409131035091320369817A818B8189
:100830009C810F94570C20E030E040E05FE30F9480
:100840004B090F94BD0A0F944F0A6093D30770931E
:10085000D4078093D5079093D607F10100811181C9
:1008600006FF35C18091EA0283FD31C1F101C688DE
:10087000D788E08CF18C8090330390903403A09063
:100880003503B0903603A5019401C701B6010F945A
:10089000570C0E9462740F944F0A2B013C01809107
:1008A0000408E0918603F0918703811104C08091D0
:1008B00003088823B1F120E030E046E153E462A967
:1008C00073A984A995A90F94AF0987FF08C08091E7
:1008D000BD0787FD04C0412C512C320115C0C70152
:1008E000B6019F772091E5023091E6024091E70240
:1008F0005091E8020F94570C20E030E04AE754E4AE
:100900000F94E30B18163CF38091FF0790910008B9
:10091000A0910108B0910208840D951DA61DB71D78
:10092000DEC020E030E046E153E462A973A984A967
:1009300095A90F94AF0987FF04C08091BD0787FF79
:10094000D7C08091FF0790910008A0910108B09155
:100950000208A3019201281B390B4A0B5B0BCA0149
:10096000B9010F94820A9F772091E5023091E60247
:100970004091E7025091E8020F94570C6B017C0103
:1009800020E030E04AE754E4C501B4010F94570C6D
:100990009B01AC01C701B6010F94E30B18160CF4D0
:1009A000A7C04092D7075092D8076092D90770929B
:1009B000DA0710FF3DC0809147080091F7061091BB
:1009C000F8068823C9F02FE737EB4AE85BE3F1012B
:1009D000628D738D848D958D0F94570C6B017C0106
:1009E000B801882777FD8095982F0F94820A9B0184
:1009F000AC01C701B60112C0B801882777FD809508
:100A0000982F0F94820AF101228D338D448D558DDC
:100A10000F94570C2EE333EC4EE259E30F94570C2E
:100A20006093F9067093FA068093FB069093FC0698
:100A3000E090E307F090E4070091E5071091E607E6
:100A40002091DF073091E0074091E1075091E207E4
:100A50006091DB077091DC078091DD079091DE07E4
:100A6000B2DC811111C08091D7079091D807A09175
:100A7000D907B091DA078093FF0790930008A093FD
:100A80000108B09302080AC0F101808191819C01A4
:100A900028733327232BC9F486FD02C080E031C0C0
:100AA0004091D7075091D8076091D9077091DA0724
:100AB0008091FF0790910008A0910108B091020871
:100AC000481759076A077B0749F381E01AC08091EC
:100AD000FF0790910008A0910108B091020880934F
:100AE000D7079093D807A093D907B093DA0761CFBF
:100AF0004092FF075092000860920108709202082D
:100B000050CF60960FB6F894DEBF0FBECDBFDF9119
:100B1000CF911F910F91FF90EF90DF90CF90BF90FA
:100B2000AF909F908F907F906F905F904F903F908D
:100B30002F9008954F925F926F927F92AF92BF92E3
:100B4000CF92DF92EF92FF920F931F93CF93DF9399
:100B5000CDB7DEB728970FB6F894DEBF0FBECDBF76
:100B600069837A838B839C8329013A01ED82FE821B
:100B70000F83188720EF33E244E759E40F94AF095D
:100B8000882311F12091ED063091EE064091EF0699
:100B90005091F00669817A818B819C810F944B0979
:100BA00020912703309128034091290350912A0373
:100BB0000F94570C0F944F0A6093CB077093CC0798
:100BC0008093CD079093CE0720EF33E244E759E4BA
:100BD000C301B2010F94AF09882301F12091E90606
:100BE0003091EA064091EB065091EC06C301B20148
:100BF0000F944B0920912B0330912C0340912D032E
:100C000050912E030F94570C0F944F0A6093CF0707
:100C10007093D0078093D1079093D20720EF33E2EF
:100C200044E759E46D817E818F8198850F94AF09E7
:100C30008823C1F020912F0330913003409131037C
:100C4000509132036D817E818F8198850F94570C6E
:100C50000F944F0A6093D3077093D4078093D507FE
:100C60009093D60720EF33E244E759E4C601B5017B
:100C70000F94AF098823B1F02091330330913403EE
:100C80004091350350913603C601B5010F94570CBE
:100C90000F944F0A6093D7077093D8078093D907B2
:100CA0009093DA0720EF33E244E759E46A8D7B8DB5
:100CB0008C8D9D8D0F94AF09882361F08A8D9B8D5B
:100CC000AC8DBD8D8093F9069093FA06A093FB0638
:100CD000B093FC0640E061E081E00E94D7F2811110
:100CE00006C082E597E10E94AB9F80E003C080E0F0
:100CF00073DA81E028960FB6F894DEBF0FBECDBF41
:100D0000DF91CF911F910F91FF90EF90DF90CF90E7
:100D1000BF90AF907F906F905F904F9008950E942A
:100D2000261E80E059DA8091E7079091E807A091AC
:100D3000E907B091EA078093DA069093DB06A09367
:100D4000DC06B093DD068091EB079091EC07A09153
:100D5000ED07B091EE078093D6069093D706A09347
:100D6000D806B093D9068091EF079091F007A09133
:100D7000F107B091F2078093D2069093D306A09327
:100D8000D406B093D5066091FF077091000880915A
:100D90000108909102080F94820A20914308309133
:100DA000440840914508509146080F94570C6093B1
:100DB000CE067093CF068093D0069093D106809193
:100DC000F9069091FA06A091FB06B091FC0680937B
:100DD000E1029093E202A093E302B093E40208954B
:100DE0008F929F92AF92BF92CF92DF92EF92FF923B
:100DF0000F931F93CF93DF93982EC62FD42FC22E1D
:100E000020E030E0A9016091E1027091E20280915E
:100E1000E3029091E4020F94AF0987FDA7C09110FF
:100E200005C0C11103C0E1E0ED2701C0E0E0CC2026
:100E300049F0A090CE06B090CF06C090D006D090DA
:100E4000D10608C0F0EFAF2EF3E2BF2EF4E7CF2EAD
:100E5000F9E4DF2EE11102C0DD23B9F05091D20692
:100E60004091D3063091D4062091D506852F942F3A
:100E7000A32FB22F8093E3079093E407A093E50795
:100E8000B093E607E11107C004C050EF43E234E736
:100E900029E4CC23B9F0D091D606C091D706709141
:100EA000D8066091D9068D2F9C2FA72FB62F80933F
:100EB000DF079093E007A093E107B093E207E11109
:100EC00007C004C0D0EFC3E274E769E49920B1F031
:100ED0008090DA069090DB06F091DC06E091DD066A
:100EE000C401AF2FBE2F8093DB079093DC07A09344
:100EF000DD07B093DE07B82DA92D04C0B0EFA3E243
:100F0000F4E7E9E41F930F93FF92EF92E52EF42E9E
:100F1000032F122F2D2F3C2F472F562F6B2F7A2F59
:100F20008F2F9E2F0E942F7E8091E1029091E202EE
:100F3000A091E302B091E4028093F9069093FA063F
:100F4000A093FB06B093FC060F900F900F900F90AC
:100F500080E0DF91CF911F910F91FF90EF90DF9094
:100F6000CF90BF90AF909F908F9036C9DF91CF9177
:100F70001F910F91FF90EF90DF90CF90BF90AF90B7
:100F80009F908F9008959091BE0795FB222720F99E
:100F9000821791F0882311F0906201C09F7D909399
:100FA000BE07882319F082E190E202C08CEF9FE136
:100FB0000E94B59F80E010C90895AF92BF92CF9272
:100FC000DF92EF92FF920F931F93CF93E82E062F9D
:100FD000F42EC091BE07C5FBCC27C0F980E0D3DF5B
:100FE0009091BD0791609093BD07EE2021F0002302
:100FF00039F01F2D06C0011103C011E01F2501C0EB
:1010000010E040E06DE077E18CE69AE00E9494AB5E
:101010008CE69AE00E94E8AE111102C0FF2019F0A0
:101020000E94AD7A1FC0EE2041F01092CB071092C3
:10103000CC071092CD071092CE07002341F01092FA
:10104000CF071092D0071092D1071092D20740E03C
:1010500060E081E00E94D7F2811104C085EE96E144
:101060000E94AB9FE0900107F090020700910307F8
:1010700010910407809116038F93809115038F932D
:10108000809114038F93809113038F93A0EFAA2E66
:10109000A3E2BA2EA4E7CA2EA9E4DA2E20E030E0BB
:1010A000A901CA01B9010E942F7E81E095D8109252
:1010B000D50A8BED96E10E94341E0F900F900F9091
:1010C0000F908C2FCF911F910F91FF90EF90DF9099
:1010D000CF90BF90AF9057CF2F923F924F925F9299
:1010E0006F927F928F929F92AF92BF92CF92DF9238
:1010F000EF92FF920F931F93CF93DF93CDB7DEB79D
:101100002B970FB6F894DEBF0FBECDBF6A874D8315
:101110004091ED065091EE066091EF067091F00659
:1011200049835A836B837C834090E9065090EA069A
:101130006090EB067090EC06882309F4AEC0222381
:1011400021F08FE390E20E942896C090EF07D090A4
:10115000F007E090F107F090F20781EA93E00E9437
:101160002F1D9B01AC01C701B6010F94E30B1816AC
:101170001CF5E09013031091140300911503F090F7
:10118000160381EA93E00E942F1DFF920F931F9395
:10119000EF9210EFA12E13E2B12E14E7C12E19E445
:1011A000D12E7B018C01A6019501C601B501C2DCDF
:1011B0000F900F900F900F9080E293E00E942F1DF0
:1011C000DC01CB01B0588093ED069093EE06A0931E
:1011D000EF06B093F00684E293E00E942F1DDC013D
:1011E000CB01B0588093E9069093EA06A093EB06F2
:1011F000B093EC0688E493E00E942F1DE62E172F93
:10120000082FF92EA30192016091E9067091EA0678
:101210008091EB069091EC060F944A0920912B03E4
:1012200030912C0340912D0350912E030F94570CB5
:101230000F944F0A2B013C0129813A814B815C813B
:101240006091ED067091EE068091EF069091F006A8
:101250000F944A09209127033091280340912903D4
:1012600050912A030F94570C0F944F0A21E02F93AB
:101270002F93FF920F931F93EF92A12CB12C650136
:10128000E12CF12C8701A30192010E9407F80F9035
:101290000F900F900F900F900F900E94261E20E04D
:1012A00030E040E251E460912F037091300380916F
:1012B0003103909132030F94570C0F944F0A6E83B1
:1012C0007F83888799876091FB077091FC078091E5
:1012D000FD079091FE0769837A838B839C838091BD
:1012E0000F0890911008A0911108B09112088093F6
:1012F0004D0790934E07A0934F07B09350071B865E
:10130000412C512C32017D81272E312C7B85872E5B
:10131000992487FC9094821493040CF01FC1C09010
:101320002107D0902207E0902307F09024078091B6
:10133000150790911607A0911707B0911807C81AC2
:10134000D90AEA0AFB0ACC0CDD1CEE1CFF1C8FEF4D
:101350009FEFDC0180933D0790933E07A0933F07EA
:10136000B093400780E293E00E942F1D84E293E057
:101370000E942F1D8091BE0780648093BE070E944B
:10138000C3230E94C3230AE010E08091000181FF83
:1013900038C08CE293E00E942F1DA7019601EE2435
:1013A000FF248701E21AF30A040B150B31E03F9387
:1013B0003F939F938F937F936F93A12CB12C6501E3
:1013C00020E030E0A90160E070E0CB010E9407F866
:1013D0000F900F900F900F900F900F9080913D07FE
:1013E00090913E07A0913F07B0914007B7FF18C00A
:1013F00086ED9FE10E94BF9F812C912C30E82FEB5E
:10140000FAC18EEC96E10E949E9F64E670E080E057
:1014100090E00F9415040150110909F0B6CFB9CF2F
:101420008091BE078F7B8093BE0700914D0710917E
:101430004E0720914F073091500780910F089091EF
:101440001008A0911108B0911208B901A801481B19
:10145000590B6A0B7B0BDB01CA0140933D0750938C
:101460003E0760933F0770934007409107085091F3
:1014700008086091090870910A08480F591F6A1FEF
:101480007B1F4093070850930808609309087093E6
:101490000A0840910B0850910C0860910D0870915A
:1014A0000E08480F591F6A1F7B1F40930B0850936B
:1014B0000C0860930D0870930E0800930F081093AA
:1014C000100820931108309312084091FB075091A7
:1014D000FC076091FD077091FE07480F591F6A1FB6
:1014E0007B1F4093FB075093FC076093FD077093AD
:1014F000FE0789819A81AB81BC81841B950BA60B69
:10150000B70B480E591E6A1E7B1EC4010196821538
:10151000930504F58CE293E00E942F1D1F9251E089
:101520005F939F938F937F936F93A12CB12C650151
:10153000EE80FF800885198520E030E0A90160E099
:1015400070E0CB010E9407F80F900F900F900F9062
:101550000F900F906B856F5F6B87D8CEC301B20180
:101560000F94820A20913F08309140084091410831
:10157000509142080F94570C6B017C01AD816A2F8A
:1015800070E080E090E00F94800A9B01AC01C701FD
:10159000B6010F94B6096B017C0188E293E00E94CA
:1015A0002F1D9B01AC01C701B6010F944B094B01E4
:1015B0008E839D8322E0AB01BC018EEA90E20E9403
:1015C000DAA120E030E040EA52E4B4018E819D814E
:1015D0000F94570C20E030E048EC54E40F944A0993
:1015E000AB01BC0122E082E890E20E94DAA14091C6
:1015F000E7075091E8076091E9077091EA0722E058
:101600008BE494E20E94DAA14091EB075091EC0741
:101610006091ED077091EE0722E087E494E20E946A
:101620009DA180E00E94EC8088EC96E10E94341E2F
:101630008CE293E00E942F1D9B014091FB0750918B
:10164000FC076091FD077091FE07E980FA800B812D
:101650001C81E41AF50A060B170B1F9241E04F9309
:101660009F938F933F932F93A12CB12C650120E082
:1016700030E0A90160E070E0CB010E9407F80F9014
:101680000F900F900F900F900F90BA85BB2309F425
:10169000B0C0C090ED06D090EE06E090EF06F0905E
:1016A000F0062090E9063090EA064090EB06509054
:1016B000EC068EE390E20E9428966090860370907C
:1016C00087036114710409F444C0F301818192819C
:1016D000A381B4819C01AD0166277727CB01621BF2
:1016E000730B840B950B0F94820A2091370830916D
:1016F00038084091390850913A080F94570C60937C
:10170000ED067093EE068093EF069093F006F301DA
:1017100085819681A781B0859C01AD0166277727D9
:10172000CB01621B730B840B950B0F94820A2091E3
:101730003B0830913C0840913D0850913E080F9481
:10174000570C6093E9067093EA068093EB0690933A
:10175000EC0688E493E00E942F1D5B01182F092FEF
:10176000A20191016091E9067091EA068091EB0671
:101770009091EC060F944A0920912B0330912C0391
:1017800040912D0350912E030F94570C0F944F0A44
:101790002B013C01A70196016091ED067091EE06C8
:1017A0008091EF069091F0060F944A09209127034B
:1017B000309128034091290350912A030F94570C2C
:1017C0000F944F0A21E02F932F930F931F93BF92F3
:1017D000AF92A12CB12C6501E12CF12C8701A30162
:1017E00092010E9407F80F900F900F900F900F90AA
:1017F0000F903E812D81B401832F922F2B960FB62F
:10180000F894DEBF0FBECDBFDF91CF911F910F9136
:10181000FF90EF90DF90CF90BF90AF909F908F9010
:101820007F906F905F904F903F902F90089540E091
:1018300050E060E87FE34093B3075093B4076093B0
:10184000B5077093B6074093A3075093A40760931E
:10185000A5077093A607409393075093940760934E
:101860009507709396071092AF071092B0071092E9
:10187000B1071092B2071092AB071092AC0710920A
:10188000AD071092AE071092A7071092A80710920A
:10189000A9071092AA0710929F071092A007109212
:1018A000A1071092A20710929B0710929C0710921A
:1018B0009D0710929E07109297071092980710921A
:1018C000990710929A07811104C087E290E20C9464
:1018D000B59F089588E10FB6F89480936000109248
:1018E00060000FBE9B9AA3988091BD07806480938F
:1018F000BD07809104018E7F8093040180910501D2
:10190000816080930501389A399A3A9A80910A0148
:10191000826080930A0180910A01816080930A01AC
:1019200080910A01846080930A010F9A179A0E9A97
:10193000169A0D9A159A3F98479A0A98129A0998FA
:10194000119A809101018D7F8093010180910201A4
:101950008260809302018091010180628093010185
:10196000809102018F7D809302016D9A75980E948B
:101970007E210E949F2281E05ADF80E090E0A8E46F
:10198000B2E48093F9069093FA06A093FB06B09315
:10199000FC0684E690E09093F8068093F706909317
:1019A000F6068093F5061092E3071092E407109272
:1019B000E5071092E6071092DF071092E0071092F9
:1019C000E1071092E2071092DB071092DC071092F9
:1019D000DD071092DE07109286071092850710929D
:1019E000771D1092781D1092791D10927A1D80E05B
:1019F00090E0A0EEB1E48093F1069093F206A093FC
:101A0000F306B093F4061092E9061092EA061092DB
:101A1000EB061092EC061092ED061092EE06109274
:101A2000EF061092F00688E893E1A0E0B0E0809322
:101A30008F0790939007A0939107B093920781E04E
:101A40008093E9021092E3061092E4061092E506F4
:101A50001092E6061092DF061092E0061092E10660
:101A60001092E2068093BE0780E090E0AAE7B3E41C
:101A70008093110790931207A0931307B093140754
:101A80008093090790930A07A0930B07B0930C0764
:101A900080E090E0A6E6B3E480930107909302070C
:101AA000A0930307B093040710920D0710920E073E
:101AB00010920F0710921007109205071092060758
:101AC00010920707109208071092FD061092FE066A
:101AD0001092FF061092000782EC95EFA1EBB2E4A2
:101AE00080936D0790936E07A0936F07B093700774
:101AF0001092DE0610924908109248080E9421CFE9
:101B000040913A0350913B0360913C0370913D0337
:101B10008FE29BE00E9488DD82EB94E20E949E9F10
:101B20008CE69AE00E94BFAB0E94A1DA0E945A4F55
:101B30000E9439D61092F3071092F4071092F5071D
:101B40001092F6071092E7071092E8071092E90743
:101B50001092EA071092F7071092F8071092F9070F
:101B60001092FA071092EB071092EC071092ED0713
:101B70001092EE071092FB071092FC071092FD07DF
:101B80001092FE071092EF071092F0071092F107E3
:101B90001092F2071092FF071092000810920108AD
:101BA000109202081092F3071092F4071092F507B2
:101BB0001092F6070E94E3740E94DD220E94EB223D
:101BC0000E9481DA67E078E083EF97E00E94F3EC0F
:101BD0008AEF93E00F9421129091BC07882311F0B3
:101BE000926001C09D7F9093BC07682F70E085ECE8
:101BF00093E00E9483A088E197E10E94341E80E078
:101C00000E94DF4F88E199E00E94AA9A2EE088E1C5
